:100000000C94EC100C94E5130C9410140C943B1409
:100010000C9466140C9491140C94BC140C94E71476
:100020000C9412150C941C110C941C110C941C11A2
:100030000C941C110C941C110C941C110C941C118C
:100040000C941C110C9465320C941C110C941C1112
:100050000C941C110C941C110C94A2260C941E11CF
:100060000C941C110C9435170C94E1170C941C1172
:100070000C941C110C941C110C941C110C941C114C
:100080000C941C110C941C110C941C110C941C113C
:100090000C941C110C941C110C941C110C941C112C
:1000A0000C941C110C941C110C941C110C941C111C
:1000B0000C941C110C941C110C941C110C941C110C
:1000C0000C941C110C941C110C941C110C941C11FC
:1000D0000C941C110C941C110C941C110C941C11EC
:1000E0000C941C115B12601265126F127912F212DD
:1000F00083128B1293129D12A712B112C012CA1250
:10010000F212D412DE12E8121613191308130C138C
:10011000121350131D13211327132B132F133513F1
:1001200039133D135013431347134B1368176E17BE
:100130007F178A179217A7179617A7179A179E1750
:10014000A717A4174C1F4A1F731F701F6E1FAA1FEB
:10015000A71FA51F0320D11FCE1FCC1F084AD73BC6
:100160003BCE016E84BCBFFDC12F3D6C74319ABD86
:1001700056833DDA3D00C77F11BED9E4BB4C3E91AA
:100180006BAAAABE000000803F05A84CCDB2D44E99
:10019000B93836A9020C50B9918688083CA6AAAA9B
:1001A0002ABE000000803F004E414E494E4954593E
:1001B000494E46CDCCCC3D0AD7233C17B7D1387732
:1001C000CC2B329595E6241FB14F0A000020410048
:1001D00000C84200401C4620BCBE4CCA1B0E5AAE92
:1001E000C59D7400000A0B02090C0D0E08070304DC
:1001F00001000000000000000000000000000000FE
:1002000000000000000000000000000000000012DC
:1002100011100000000000000000000000000000BD
:10022000000000000000000000010210202008086B
:100230001020401020408002010201080402010148
:100240000204081020408080402010080402018031
:100250000402018040201008040201080402010188
:10026000020408102040800102040810204080058C
:10027000050505070508080808020202020A0A081F
:100280000804040404010101010101010103030345
:100290000303030303040707070C0C0C0C0C0C0CE2
:1002A0000C0202020206060606060606060B0B0BE9
:1002B0000B0B0B0B0B000020002300260029002C49
:1002C000002F0032000001000003010601090100B7
:1002D000002200250028002B002E003100340002EF
:1002E000010000050108010B010000210024002786
:1002F000002A002D00300033000101000004010736
:10030000010A014F4646004F4E006563686F3A0090
:100310004572726F723A004572726F72207772691D
:1003200074696E6720746F20454550524F4D210A05
:100330000063616E63656C00706F7765726F6666EF
:10034000002F2F616374696F6E3A0020573A0020C6
:10035000573A00202F002042403A0020403A0054F3
:100360006865726D616C2052756E617761790045C8
:100370003120544845524D414C2052554E41574131
:10038000590042656400202D20496E76616C6964D5
:10039000206578747275646572206E756D62657221
:1003A00020210A0048656174696E67206661696C86
:1003B0006564004265640048656174696E67206623
:1003C00061696C65640045312048656174696E67D8
:1003D000206661696C6564004D494E54454D50205E
:1003E0007472696767657265640045312045727291
:1003F0003A204D494E54454D5000426564004D41F0
:100400005854454D50207472696767657265640081
:100410004531204572723A204D415854454D5000A7
:1004200042656400626564002C2073797374656DA5
:100430002073746F70706564212048656174657203
:100440005F49443A200023646566696E652044452F
:100450004641554C545F004B6420004B6920004BD3
:100460007020000062656400504944204175746F3B
:1004700074756E652066696E6973686564212050C5
:10048000757420746865206C617374204B702C2027
:100490004B6920616E64204B6420636F6E737461DE
:1004A0006E74732066726F6D2062656C6F77206961
:1004B0006E746F20436F6E66696775726174696FE1
:1004C0006E2E680A00504944204175746F74756E31
:1004D00065206661696C6564212074696D656F755E
:1004E000740A00546865726D616C2052756E617794
:1004F000617900453120544845524D414C205255B8
:100500004E41574159004265640048656174696E07
:1005100067206661696C65640045312048656174D7
:10052000696E67206661696C6564004265640050AD
:100530004944204175746F74756E65206661696CFD
:100540006564212054656D706572617475726520F3
:10055000746F6F20686967680A00204B643A200056
:10056000204B693A2000204B703A20000A20436C4F
:10057000617373696320504944200A002054753A1E
:100580002000204B753A2000206D61783A20002031
:100590006D696E3A200020643A2000206269617320
:1005A0003A2000504944204175746F74756E65207F
:1005B00073746172740A00504944204175746F74F9
:1005C000756E65206661696C6564212054656D7087
:1005D0006572617475726520746F6F2068696768F1
:1005E0000A001000AD0330016A0150022B017003B4
:1005F0000A019004F500B005E500D006D800F00728
:10060000CE001009C500300ABE00500BB700700CB8
:10061000B100900DAB00B00EA600D00FA200F010FC
:100620009D0010129900301395005014920070151F
:100630008E0090168B00B0178700D0188400F01938
:100640008100101B7E00301C7B00501D7900701E45
:100650007600901F7300B0207000D0216E00F02251
:100660006B00102469003025660050266300702757
:10067000610090285E00B0295C00D02A5900F02B60
:100680005600102D5400302E5100502F4E00703067
:100690004B0090314800B0324500D0334200F03476
:1006A0003E0010363B003037370050383300703989
:1006B0002E00903A2900B03B2300D03C1B00F03DB7
:1006C0001100103F0100F03F00001000C9021001AE
:1006D0002C014001220170011801B0010E01F0014E
:1006E00004015002FA00B002F0003003E600D0032B
:1006F000DC009004D2007005C800A006BE0000080F
:10070000B400B009AA00D00BA000600E96006011E2
:100710008C000015820020197800C01D6E00A022F8
:100720006400B0275A00902C500000314600E0349D
:100730003C0010383200903A2800603C1E00A03D7A
:100740001400803E0A00203F00006F70656E005468
:100750005249474745524544003A20007A5F6D614F
:1007600078007A5F6D696E00795F6D617800795FFE
:100770006D696E00785F6D617800785F6D696E00FD
:100780005265706F7274696E6720656E6473746F02
:1007900070207374617475730A00205A3A002059EE
:1007A0003A0020583A00656E6473746F7073206865
:1007B00069743A2000486F6D696E67206661696CE4
:1007C000656400496E76616C696420657874727541
:1007D0006465720A0045303A20005A3A2000593ABE
:1007E00020004D53312C4D53322C4D533320506942
:1007F0006E730A583A20004D6963726F73746570A6
:100800007320756E617661696C61626C650A0020A7
:100810005A3A0020593A0020436F756E7420583AB6
:1008200000C23100001C260000F4190000D80F009F
:1008300000EB080000C00400007502000040010049
:100840000024F4D43050C38E20C2A24017828B7093
:1008500011127A910D816CD90AA861E108C7586616
:1008600007615143061E4B5D05C145A7041A41119E
:1008700004093D9803713931034036DB0265339139
:1008800002D4305402802E1D02632CEE01752AC55D
:1008900001B028A001102781018F2564012B244B72
:1008A00001E0223401AC211F018D200D01801FFCCD
:1008B00000841EED00971DDF00B81CD200E61BC6A9
:1008C00000201BBC00641AB200B219A8000A19A0CB
:1008D000006A189900D117910040178B00B5168453
:1008E0000031167E00B31579003A157300C7146FF6
:1008F0000058146A00EE1366008813630025135E27
:1009000000C7125B006C12570015125400C1115140
:100910000070114F0021114B00D61049008D104777
:10092000004610440002104200C00F4000800F3EFD
:1009300000420F3C00060F3B00CB0E3800930E37F1
:10094000005C0E3500270E3400F30D3200C10D316E
:1009500000900D3000600D2E00320D2D00050D2C85
:1009600000D90C2B00AE0C2900850C29005C0C274B
:1009700000350C27000E0C2600E80B2400C40B24C5
:1009800000A00B23007D0B23005A0B2100390B2103
:1009900000180B2000F80A1F00D90A1E00BB0A1E0F
:1009A000009D0A1D00800A1D00630A1C00470A1BE7
:1009B000002C0A1B00110A1A00F7091A00DD091998
:1009C00000C4091900AB091900920917007B091826
:1009D00000630917004C0916003609160020091695
:1009E000000A091500F5081500E0081400CC0814E9
:1009F00000B8081400A4081400900813007D081221
:100A0000006B081300580812004608120034081141
:100A100000230811001208110001081100F007104E
:100A200000E0071000D0071000C0071000B0070F4B
:100A300000A107100091070E0083070F0074070F35
:100A40000065070E0057070E0049070E003B070D13
:100A5000002E070E0020070D0013070D0006070DDE
:100A600000F9060C00ED060D00E0060C00D4060CA3
:100A700000C8060C00BC060C00B0060C00A4060B57
:100A80000099060C008D060B0082060B0077060B02
:100A9000006C060B0061060A0057060B004C060AA4
:100AA0000042060A0038060A002E060A0024060A3A
:100AB000001A060A001006090007060A00FD0509CB
:100AC00000F4050900EB050900E2050900D9050954
:100AD00000D0050900C7050900BE050900B50508D5
:100AE00000AD050800A50509009C0508009405084F
:100AF000008C050800840508007C050800740508C2
:100B0000006C050700650508005D0507005605082F
:100B1000004E050700470507004005080038050797
:100B200000310507002A050700230507001C0506FC
:100B300000160507000F0507000805060002050757
:100B400000FB040600F5040700EE040600E80406B6
:100B500000E2040700DB040600D5040600CF04060B
:100B600000C9040600C3040600BD040600B704065D
:100B700000B1040500AC040600A6040600A00405AC
:100B8000009B04060095040500900406008A0405F5
:100B90000085040500800406007A0405007504053C
:100BA00000700405006B040500660405006104057F
:100BB000005C04050057040500520405004D0405BF
:100BC0000048040500430405003E0404003A0405FF
:100BD0000035040500300404002C0405002704043B
:100BE00000230405001E0404001A04040016040572
:100BF00000110404000D04040009040500040404A9
:100C00000000040400FC030400F8030400F40304DF
:100C100000F0030400EC030400E8030400E4030410
:100C200000E0030400DC030400D8030400D4030440
:100C300000D0030400CC030400C8030300C5030371
:100C40000024F404D9201BC40C5C0E9804C4095F72
:100C50000265077101F405F900FB04B3004804873D
:100C600000C10369005803550003034500BE023A62
:100C7000008402310053022A0029022500040220C8
:100C800000E4011C00C8011900AF0117009801140D
:100C90000084011300710110006101100051010E68
:100CA0000043010D0036010B002B010B0020010B4E
:100CB00000150109000C01090003010800FB0008F0
:100CC00000F3000800EB000700E4000600DE000669
:100CD00000D8000600D2000600CC000500C70005C1
:100CE00000C2000500BD000400B9000400B5000406
:100CF00000B1000400AD000400A9000400A5000339
:100D000000A20003009F0004009B00030098000362
:100D1000009500020093000300900003008D000284
:100D2000008B00030088000200860002008400039C
:100D300000810002007F0002007D0002007B0002B3
:100D400000790002007700010076000200740002C2
:100D50000072000100710002006F0002006D0001CE
:100D6000006C0002006A00010069000200670001D7
:100D700000660001006500010064000200620001DD
:100D80000061000100600001005F0002005D0001E1
:100D9000005C0001005B0001005A000100590001E5
:100DA00000580001005700010056000100550001E5
:100DB00000540001005300000053000100520001E4
:100DC0000051000100500001004F0001004E0000E2
:100DD000004E0001004D0001004C0001004B0000DE
:100DE000004B0001004A00010049000100480000DA
:100DF00000480001004700010046000000460001D5
:100E000000450000004500010044000100430000CF
:100E100000430001004200000042000100410000C8
:100E20000041000100400001003F0000003F0001C0
:100E3000003E0000003E0001003D0000003D0001BA
:100E4000003C0000003C0000003C0001003B0000B2
:100E5000003B0001003A0000003A000100390000A8
:100E6000003900010038000000380000003800019F
:100E70000037000000370001003600000036000097
:100E8000003600010035000000350000003500018B
:100E90000034000000340000003400010033000082
:100EA0000033000000330001003200000032000077
:100EB000003200010031000000310000003100016B
:100EC000003000000030000000300001002F000062
:100ED000002F0000002F0000002F0001002E000056
:100EE000002E0000002E0001002D0000002D00004B
:100EF000002D0000002D0001002C0000002C00003F
:100F0000002C0000002C0001002B0000002B000032
:100F1000002B0000002B0001002A0000002A000026
:100F2000002A0000002A000100290000002900001A
:100F3000002900000029000000290001002800000D
:100F40000028000000280000002800000028000100
:100F500000270000002700000027000000270000F5
:100F600000270001002600000026000000260000E7
:100F700000260000002600010025000000250000DA
:100F800000250000002500000025000000250001CC
:100F900000240000002400000024000000240000C1
:100FA00000240001002300000023000000230000B3
:100FB00000230000002300000023000000230001A4
:100FC0000022000000220000002200000022000099
:100FD000002200000022000100210000002100008A
:100FE000002100000021000000210000002100007D
:100FF000002100010020000000200000002000006F
:101000000020000000200000002000000020000060
:1010100000200001001F0000001F0000001F000052
:10102000001F0000001F0000001F0000001F000143
:10103000001E0000001E0000001E0000001E000038
:10104000003A0A0020286D6D2900204500205A0032
:1010500020204D3930372058005374657070657208
:10106000206D6F746F722063757272656E74733A5F
:101070000A0020204D393030204B004C696E6561EC
:101080007220416476616E63653A0A0020204D3813
:101090003531205A005A2D50726F6265204F6666B6
:1010A0007365740020440020490020204D33303403
:1010B00020500020440020490020204D33303120B2
:1010C00050005049442073657474696E67733A0A1E
:1010D0000020204D3432302053004175746F20427F
:1010E0006564204C6576656C696E673A0A00204538
:1010F00000205A002059002058002054002053009E
:1011000020204D32303520420020453C6D61785F13
:10111000655F6A65726B3E0020583C6D61785F7850
:101120005F6A65726B3E20593C6D61785F795F6ADA
:1011300065726B3E205A3C6D61785F7A5F6A6572BA
:101140006B3E00416476616E6365643A20423C6D9B
:10115000696E5F7365676D656E745F74696D655FF9
:1011600075733E20533C6D696E5F666565647261A0
:1011700074653E20543C6D696E5F74726176656C77
:101180005F66656564726174653E0020540020529C
:101190000020204D323034205000416363656C657F
:1011A000726174696F6E2028756E6974732F733263
:1011B000293A20503C7072696E745F616363656C9C
:1011C0003E20523C726574726163745F6163636553
:1011D0006C3E20543C74726176656C5F616363653C
:1011E0006C3E0A00204500205A0020590020204D66
:1011F0003230312058004D6178696D756D20416342
:1012000063656C65726174696F6E2028756E6974B0
:10121000732F7332293A0A00204500205A002059C2
:101220000020204D3230332058004D6178696D75B3
:101230006D206665656472617465732028756E69DA
:1012400074732F73293A0A005374657073207065A4
:101250007220756E69743A0A0020204732312020CE
:1012600020203B20556E69747320696E206D6D00DF
:1012700048617264636F6465642044656661756C7F
:10128000742053657474696E6773204C6F61646574
:10129000640A00282300002823000064000000E8FE
:1012A0000300000000964300009643000000410048
:1012B0000020420000C9420000C9420000C84400AA
:1012C00000D243290A002062797465733B2063725F
:1012D0006320002073746F72656420736574746991
:1012E0006E67732072657472696576656420280084
:1012F000202863616C63756C6174656429210A0040
:1013000020213D2000454550524F4D20435243205F
:101310006D69736D61746368202D202873746F721A
:1013200065642920002053697A653A2000496E647B
:1013300065783A2000204D61726C696E3D563634F6
:10134000290A00454550524F4D2076657273696FEA
:101350006E206D69736D6174636820284545505235
:101360004F4D3D00290A002062797465733B20636C
:101370007263200053657474696E67732053746FD1
:10138000726564202800454550524F4D20646174B9
:101390006173697A65206572726F722E0A005072ED
:1013A0006F62696E67206661696C65640A005761E7
:1013B000726E696E673A20486F6D696E672042757C
:1013C0006D702044697669736F72203C20310A0089
:1013D0000202042066697273740A00486F6D65200A
:1013E0000020746F6F206C6F6E6720657874727563
:1013F00073696F6E2070726576656E7465640A003D
:1014000020636F6C6420657874727573696F6E20E9
:1014100070726576656E7465640A0020453A002036
:101420005A3A0020593A00583A000000F0410000B2
:10143000F04100000041FF01010000A0400000A0B9
:10144000400000004000002543000045430000210B
:1014500043000040C000003E4300001F4300002244
:101460004300003E4300001F43000040C00000E076
:10147000C0000000C020746F6F206C6F6E67206525
:101480007874727573696F6E2070726576656E74AC
:1014900065640A0020636F6C6420657874727573EC
:1014A000696F6E2070726576656E7465640A00629D
:1014B0007573793A2070617573656420666F722068
:1014C000696E7075740A00627573793A207061757F
:1014D00073656420666F7220757365720A006275A9
:1014E00073793A2070726F63657373696E670A006F
:1014F0004D3131372050726F6265207375636365BB
:10150000737366756C0A0020496E76616C6964209D
:1015100065787472756465722000205A3A20002044
:10152000593A200042656420583A200050726F6298
:1015300065205A204F66667365743A20003F5A2032
:101540006F7574206F662072616E676520282D327A
:1015500020746F2035290A00220A00556E6B6E6FC9
:10156000776E20636F6D6D616E643A202200454591
:1015700050524F4D204F4B0A004543484F00494EB3
:10158000464F004552524F52530044525952554E05
:1015900000434F4D4D554E49434154494F4E006F06
:1015A00066660079157E1583158A159115444542A6
:1015B00055473A00205A00205900580020204D611C
:1015C000783A2000205A00205900580020204D6908
:1015D0006E3A2000536F667420656E6473746F708A
:1015E000733A20002569730025696D202569730011
:1015F0002569682025696D202569730025696420A7
:101600002569682025696D20256973002569792081
:10161000256964202569682025696D202569730086
:101620005072696E742074696D653A20004D3131D5
:10163000332053002F2F20004361703A004D4F5448
:10164000494F4E5F4D4F44455300544845524D411C
:101650004C5F50524F54454354494F4E00415554EE
:101660004F5245504F52545F53445F535441545569
:10167000530050524F4D50545F535550504F525499
:1016800000454D455247454E43595F5041525345E1
:101690005200434153455F4C494748545F425249C9
:1016A0004748544E45535300544F47474C455F4CB1
:1016B000494748545300534F4654574152455F5091
:1016C0004F574552004255494C445F50455243459F
:1016D0004E54004C4556454C494E475F4441544199
:1016E000005A5F50524F4245004155544F4C4556A9
:1016F000454C005052494E545F4A4F420050524FA1
:101700004752455353004155544F5245504F525440
:101710005F54454D5000564F4C554D45545249432A
:1017200000454550524F4D0042494E4152595F4687
:10173000494C455F5452414E534645520053455221
:1017400049414C5F584F4E5F584F464600464952FC
:101750004D574152455F4E414D453A4D61726C695E
:101760006E20204649524D574152455F56455253CF
:10177000494F4E3A322E302E302E313033204558DC
:101780005452554445525F545950453A4861726429
:10179000656E6564537465656C506C757320534F4A
:1017A000555243455F434F44455F55524C3A687428
:1017B0007470733A2F2F636F64652E616C65706867
:1017C0006F626A656374732E636F6D2F64696666FA
:1017D0007573696F6E2F4D41524C494E2050524FD8
:1017E000544F434F4C5F56455253494F4E3A312E5A
:1017F00030204D414348494E455F545950453A4C7D
:10180000756C7A426F74204D696E69204558545248
:10181000554445525F434F554E543A312055554932
:10182000443A33353134383762362D636139612DAE
:10183000346331612D383736352D643636386231B0
:101840006461363538350A0020284E6F742079657A
:1018500074206D656173757265642900202041767E
:101860006572616765206D6561737572656420627C
:1018700061636B6C61736820286D6D293A002020CC
:10188000536D6F6F7468696E6720286D6D293A20FB
:101890002020202020202020202020202020202048
:1018A000530020204261636B6C617368204469734C
:1018B00074616E636520286D6D293A2020202020F8
:1018C0002020200020202020202846312E30203DBE
:1018D0002066756C6C2C2046302E30203D206E6FBB
:1018E0006E65290A002020436F7272656374696F08
:1018F0006E20416D6F756E742F466164652D6F7536
:10190000743A202020202046006163746976653A8D
:101910000A00696E004261636B6C61736820636FDB
:101920007272656374696F6E2069732000205A00BB
:1019300020506F736974696F6E616C204572726FAD
:10194000723A0A004E6F7A7A6C6520546970204FA3
:10195000757465722044696D656E73696F6E733A54
:101960000A002020546F703A2000202046726F6ECB
:10197000743A200020204C6566743A20004261636E
:101980006B6C6173683A0A00205A0043656E746597
:10199000723A0A00202046726F6E743A20002020AE
:1019A0004C6566743A20002020546F703A20005332
:1019B000696465733A0A00426564204C6576656C1B
:1019C000696E6720004661696C656420746F2065EC
:1019D0006E61626C6520426564204C6576656C6959
:1019E0006E670A00426564204C6576656C20436F23
:1019F0007272656374696F6E204D61747269783AB2
:101A0000000A0A426564204C6576656C20436F725B
:101A100072656374696F6E204D61747269783A0003
:101A2000202B000A436F72726563746564204265FF
:101A300064204865696768742076732E2042656467
:101A400020546F706F6C6F67793A0A00202B000A80
:101A50004265642048656967687420546F706F67D9
:101A600072617068793A0A2020202B2D2D2D20429A
:101A700041434B202D2D2B0A2020207C202020208C
:101A8000202020202020207C0A204C207C20202088
:101A900020282B29202020207C20520A2045207C31
:101AA00020202020202020202020207C20490A20C7
:101AB00046207C20282D29204E20282B29207C20E0
:101AC000470A2054207C2020202020202020202075
:101AD000207C20480A2020207C20202020282D291E
:101AE000202020207C20540A2020207C2020202020
:101AF000202020202020207C0A2020204F2D2D2057
:101B000046524F4E54202D2D2B0A2028302C3029A0
:101B10000A003474682070726F626520706F696E9D
:101B2000742C2064697374616E63652066726F6DD6
:101B300020706C616E653A2000202844525952553D
:101B40004E2900473239204175746F204265642068
:101B50004C6576656C696E67003F20284C2C522CD2
:101B6000462C4229206F7574206F6620626F756E57
:101B700064732E0A003F50726F626520706F696E49
:101B800074732028592920697320696D706C617500
:101B90007369626C652028322D32292E0A003F506D
:101BA000726F626520706F696E74732028582920E7
:101BB000697320696D706C61757369626C6520284A
:101BC000322D32292E0A003F2856296572626F7322
:101BD00065206C6576656C20697320696D706C6139
:101BE000757369626C652028302D34292E0A0041F6
:101BF0006476616E6365204B3D003F4B2076616CDF
:101C00007565206F7574206F662072616E67652040
:101C100028302D3130292E0A004D31313720486FC0
:101C20007420456E642048656174696E672E2E2E9F
:101C30000A4D31303420533137302054300A473286
:101C400038204F310A473120593235205A3130205F
:101C500046353030300A4D3130392052313730205E
:101C600054300A4D313137205265776970696E679B
:101C7000206E6F7A7A6C650A54300A4731205834E6
:101C80003520593137322046353030300A4731203F
:101C90005A310A4D31303920523137300A4731201C
:101CA00058343520593137322046343030300A47E5
:101CB00031205834352059313732204634303030D5
:101CC0000A473120583435205931373220463430D4
:101CD00030300A47312058343520593137322046C8
:101CE000343030300A4731205834352059313732BA
:101CF0002046343030300A473120583435205931AD
:101D000037322046343030300A47312058343520BD
:101D1000593137322046343030300A473120583478
:101D20003520593137322046343030300A4731209F
:101D300058343520593137322046343030300A4754
:101D40003120583435205931373220463430303044
:101D50000A47312058343520593137322046343043
:101D600030300A4731205834352059313732204637
:101D7000343030300A4731205A31350A4D3130364F
:101D80002053323535200A47302058302059300A48
:101D90004D31303920523136302054300A4D3130F7
:101DA000370A0020466C6F773A200020643A002002
:101DB000693A0020703A00204500205A002059005E
:101DC000204D393220580043290A0061626C656455
:101DD00020286D696E2074656D7020006469730041
:101DE000656E00436F6C642065787472756465730A
:101DF0002061726520002054002052004163636519
:101E00006C65726174696F6E3A205000496E76613C
:101E10006C69642065787472756465720A00206468
:101E20003A0020693A0020703A0047322F473320A9
:101E300062616420706172616D65746572730A001D
:101E40005072696E7465722073746F70706564206F
:101E500064756520746F206572726F72732E2046F0
:101E6000697820746865206572726F7220616E6493
:101E700020757365204D39393920746F2072657370
:101E8000746172742E202854656D7065726174756A
:101E900072652069732072657365742E20536574B2
:101EA0002069742061667465722072657374617252
:101EB00074696E67290A004E6F20436865636B730F
:101EC000756D2077697468206C696E65206E756D1C
:101ED0006265722C204C617374204C696E653A20E7
:101EE00000636865636B73756D206D69736D6174F4
:101EF00063682C204C617374204C696E653A200035
:101F00004C696E65204E756D626572206973206E36
:101F10006F74204C617374204C696E65204E756D32
:101F20006265722B312C204C617374204C696E6594
:101F30003A20004D31313000526573656E643A20AD
:101F4000002042002050006F6B00220A00656E7175
:101F500075657565696E672022005049442041759A
:101F6000746F74756E65206661696C6564212042CA
:101F70006164206578747275646572206E756D6237
:101F800065720A006F6B002020506C616E6E657286
:101F900042756666657242797465733A2000204620
:101FA000726565204D656D6F72793A2000436F6DE3
:101FB00070696C65643A204D617220323220323093
:101FC00031390A00207C20417574686F723A2028EC
:101FD000416C657068204F626A6563747320496E56
:101FE000632E2C204C756C7A426F742047697420E4
:101FF0005265706F7369746F7279290A0000204C02
:1020000061737420557064617465643A2000322EE7
:10201000302E302E3130330A004D61726C696E0003
:1020200020536F6674776172652052657365740A18
:1020300000205761746368646F672052657365742C
:102040000A002042726F776E206F7574205265739C
:1020500065740A002045787465726E616C20526563
:102060007365740A00506F77657255700A00737457
:102070006172740A005072696E7465722068616CD6
:102080007465642E206B696C6C28292063616C6C0C
:102090006564210A004B494C4C206361757365648B
:1020A00020627920746F6F206D75636820696E619E
:1020B00063746976652074696D65202D206375727F
:1020C00072656E7420636F6D6D616E643A20004DB1
:1020D0003132310A4730205A31300A4732382058DD
:1020E000302059300A4731320A4D313039205231CF
:1020F00036300A4D3131372050726F62696E672079
:102100006265640070726F62655F726577697065A1
:102110000050726F62696E67206661696C65640069
:102120004D31313720426564206C6576656C696E8F
:1021300067206661696C65642E0A4730205A313029
:102140000A47302045300A4D333030205032352098
:10215000533838300A4D333030205035302053302A
:102160000A4D3330302050323520533838300A4D44
:10217000333030205035302053300A4D333030204A
:1021800050323520533838300A47342053310070EC
:10219000726F62655F6661696C65640050726F742E
:1021A00065637465642050696E0A0025301D0C1E3D
:1021B000282924311C0B184527232F1B0A174443B9
:1021C000222B1A4142043803FF3604080606000198
:1021D000651A1A30CD6B0A9211241FBECFEFD1E2DF
:1021E000DEBFCDBF00E00CBF13E0A0E0B2E0ECE04A
:1021F000FFE601E00BBF02C007900D92A03AB107C5
:10220000D9F72EE0A0EAB3E001C01D92AD3EB207BF
:10221000E1F710E1CCEED0E100E006C02197010922
:10222000802FFE010E941BB0C83ED10780E0080746
:10223000A9F766D40C9484B70C9400001F920F92F7
:102240000FB60F9211242F933F938F939F93AF93C9
:10225000BF938091A1039091A203A091A303B09199
:10226000A4033091A00323E0230F2D3720F401961F
:10227000A11DB11D05C026E8230F0296A11DB11DA9
:102280002093A0038093A1039093A203A093A303A0
:10229000B093A4038091A5039091A603A091A703F6
:1022A000B091A8030196A11DB11D8093A503909341
:1022B000A603A093A703B093A803BF91AF919F91EA
:1022C0008F913F912F910F900FBE0F901F901895F7
:1022D0002FB7F8946091A1037091A2038091A3039A
:1022E0009091A4032FBF08953FB7F8948091A50360
:1022F0009091A603A091A703B091A80326B5A89B2F
:1023000005C02F3F19F00196A11DB11D3FBFBA2F87
:10231000A92F982F8827820F911DA11DB11DBC01E7
:10232000CD0142E0660F771F881F991F4A95D1F7AC
:1023300008958F929F92AF92BF92CF92DF92EF92C9
:10234000FF926B017C01D0DF4B015C01C114D10411
:10235000E104F104F1F091D3C7DFDC01CB0188196E
:102360009909AA09BB09883E9340A105B10570F3FC
:1023700021E0C21AD108E108F10888EE880E83E056
:10238000981EA11CB11CC114D104E104F10421F771
:10239000DDCFFF90EF90DF90CF90BF90AF909F90F8
:1023A0008F900895789484B5826084BD84B58160EF
:1023B00084BD85B5826085BD85B5816085BDEEE64D
:1023C000F0E0808181608083E1E8F0E0108280812C
:1023D00082608083808181608083E0E8F0E080819A
:1023E00081608083E1EBF0E0808184608083E0EBBA
:1023F000F0E0808181608083E1E9F0E080818260AB
:102400008083808181608083E0E9F0E08081816069
:102410008083E1EAF0E08081826080838081816056
:102420008083E0EAF0E0808181608083E1E2F1E096
:10243000808182608083808181608083E0E2F1E03E
:10244000808181608083EAE7F0E08081846080831E
:1024500080818260808380818160808380818068C8
:1024600080831092C10008951F93CF93DF93182F9C
:10247000EB0161E016D1209711F460E004C0CF3F7A
:10248000D10531F461E0812FDF91CF911F9145C1DA
:10249000E12FF0E0ED51FE4FE4914E2F50E0FA01B4
:1024A0003197E231F10508F09DC08827EE58FF4FC3
:1024B0008F4F0C941BB084B5806884BDC7BD97C096
:1024C00084B5806284BDC8BD92C080918000806860
:1024D00080938000D0938900C093880088C0809149
:1024E0008000806280938000D0938B00C0938A002C
:1024F0007EC080918000886080938000D0938D00A2
:10250000C0938C0074C08091B00080688093B0004C
:10251000C093B3006CC08091B00080628093B00023
:10252000C093B40064C08091900080688093900054
:10253000D0939900C09398005AC080919000806217
:1025400080939000D0939B00C0939A0050C08091DC
:102550009000886080939000D0939D00C0939C0071
:1025600046C08091A00080688093A0008091A00068
:102570008F7B8093A000D093A900C093A80037C0A0
:102580008091A00080628093A000D093AB00C093A4
:10259000AA002DC08091A00088608093A000D093F5
:1025A000AD00C093AC0023C080912001806880936F
:1025B0002001D0932901C093280119C080912001E6
:1025C000806280932001D0932B01C0932A010FC019
:1025D00080912001886080932001D0932D01C093C9
:1025E0002C0105C0C038D1050CF04CCF46CFDF918F
:1025F000CF911F91089590E0FC013197E231F105F0
:1026000008F04EC08827EC57FF4F8F4F0C941BB03B
:10261000809180008F7703C0809180008F7D8093B0
:102620008000089580918000877FF9CF84B58F77EF
:1026300002C084B58F7D84BD08958091B0008F77EE
:1026400003C08091B0008F7D8093B0000895809189
:1026500090008F7707C0809190008F7D03C080919C
:102660009000877F8093900008958091A0008F77DD
:1026700007C08091A0008F7D03C08091A000877F5C
:102680008093A0000895809120018F7707C08091EA
:1026900020018F7D03C080912001877F80932001DE
:1026A0000895CF93DF9390E0FC01E75DFD4F249107
:1026B000FC01E159FD4F8491882361F190E0880F7E
:1026C000991FFC01E751FD4FC591D491FC01E153E5
:1026D000FD4FA591B491611109C09FB7F89488810D
:1026E000209582238883EC912E230BC0623061F405
:1026F0009FB7F8943881822F809583238883EC914B
:102700002E2B2C939FBF06C08FB7F894E8812E2BF9
:1027100028838FBFDF91CF9108951F93CF93DF93CD
:10272000282F30E0F901ED51FE4F8491F901E75D6A
:10273000FD4FD491F901E159FD4FC491CC23C1F073
:10274000162F811158DFEC2FF0E0EE0FFF1FE15341
:10275000FD4FA591B4918FB7F894111105C09C91CC
:10276000ED2FE095E92302C0EC91ED2BEC938FBFA8
:10277000DF91CF911F910895CF93DF93282F30E001
:10278000F901ED51FE4F8491F901E75DFD4FD491C0
:10279000F901E159FD4FC491CC2389F081112BDF60
:1027A000EC2FF0E0EE0FFF1FEB54FD4FA591B4911D
:1027B000EC91ED2381E090E021F480E002C080E024
:1027C00090E0DF91CF91089508951F920F920FB678
:1027D0000F9211240BB60F922F933F934F935F9359
:1027E0006F937F938F939F93AF93BF93EF93FF93D9
:1027F000E0910402F09105021995FF91EF91BF91CC
:10280000AF919F918F917F916F915F914F913F9188
:102810002F910F900BBE0F900FBE0F901F90189529
:102820001F920F920FB60F9211240BB60F922F9397
:102830003F934F935F936F937F938F939F93AF9348
:10284000BF93EF93FF93E0910602F0910702199571
:10285000FF91EF91BF91AF919F918F917F916F9178
:102860005F914F913F912F910F900BBE0F900FBE34
:102870000F901F9018951F920F920FB60F92112470
:102880000BB60F922F933F934F935F936F937F936A
:102890008F939F93AF93BF93EF93FF93E0910802C1
:1028A000F09109021995FF91EF91BF91AF919F911E
:1028B0008F917F916F915F914F913F912F910F90E9
:1028C0000BBE0F900FBE0F901F9018951F920F9286
:1028D0000FB60F9211240BB60F922F933F934F9385
:1028E0005F936F937F938F939F93AF93BF93EF9378
:1028F000FF93E0910A02F0910B021995FF91EF917D
:10290000BF91AF919F918F917F916F915F914F9107
:102910003F912F910F900BBE0F900FBE0F901F9005
:1029200018951F920F920FB60F9211240BB60F92AB
:102930002F933F934F935F936F937F938F939F93C7
:10294000AF93BF93EF93FF93E0910002F0910102E8
:102950001995FF91EF91BF91AF919F918F917F91C9
:102960006F915F914F913F912F910F900BBE0F9000
:102970000FBE0F901F9018951F920F920FB60F92D7
:1029800011240BB60F922F933F934F935F936F9346
:102990007F938F939F93AF93BF93EF93FF93E091B8
:1029A0000202F09103021995FF91EF91BF91AF914F
:1029B0009F918F917F916F915F914F913F912F9157
:1029C0000F900BBE0F900FBE0F901F9018951F9287
:1029D0000F920FB60F9211240BB60F922F933F93C5
:1029E0004F935F936F937F938F939F93AF93BF9317
:1029F000EF93FF93E0910C02F0910D021995FF9176
:102A0000EF91BF91AF919F918F917F916F915F9166
:102A10004F913F912F910F900BBE0F900FBE0F90D3
:102A20001F9018951F920F920FB60F9211240BB69C
:102A30000F922F933F934F935F936F937F938F9357
:102A40009F93AF93BF93EF93FF93E0910E02F091AA
:102A50000F021995FF91EF91BF91AF919F918F91C7
:102A60007F916F915F914F913F912F910F900BBE8E
:102A70000F900FBE0F901F90189508954F925F9280
:102A80006F927F92AF92BF92CF92DF92EF92FF92BE
:102A90000F931F93CF93DF93CDB7DEB729013A0190
:102AA0009B01AC0124193509460957098A899B897C
:102AB000AC89BD89BC01CD016A197B098C099D09CE
:102AC0000E94BAAFA8019701241935094609570990
:102AD0000E94FFAFCA01B9016A0D7B1D8C1D9D1DAF
:102AE000DF91CF911F910F91FF90EF90DF90CF90EA
:102AF000BF90AF907F906F905F904F900895089532
:102B000051DCFDDF0E944DABC0E0D0E00E94CCABB9
:102B10002097E1F30E940000F9CFCF93C82F0E94C5
:102B20007C30CC2349F024982C9A65E070E080E05A
:102B300090E0FFDB149A03C0249A2C981498CF914C
:102B4000089580E0EACFCF92DF92EF92FF926B017F
:102B50007C0183E3C816D104E104F10468F082E348
:102B6000C81AD108E108F10862E370E080E090E063
:102B7000E0DB0E94C724EDCFC701B601DADBFF908E
:102B8000EF90DF90CF900C94C724DC01FB01460F3F
:102B9000571FE417F507C1F081912D913C911197D2
:102BA000382798E0B901660F771F37FF06C09B01F1
:102BB00081E2282780E1382701C09B01915091F7DD
:102BC00011963C932E93E5CF0895CF93DF93FC01AC
:102BD0008491EF012196882319F087D2FE01F8CF66
:102BE000DF91CF9108958AE093E0EFCF80E193E009
:102BF000ECCF0F931F93CF93DF931F921F92CDB70C
:102C0000DEB769837A83E1DF6981062F7A81172F26
:102C1000F80181918F01882311F067D2F9CF0F90CD
:102C20000F90DF91CF911F910F910895CF93DF9374
:102C3000EB01CBDF6AE070E0CE01DF91CF9148C3BA
:102C4000CF92DF92EF92FF926A017B01BEDF4AE0F2
:102C500050E0C701B601FF90EF90DF90CF9027C3FF
:102C6000CF92DF92EF92FF926A017B01AEDF42E0EA
:102C700050E0C701B601FF90EF90DF90CF90B3C353
:102C8000CF92DF92EF92FF926A017B019EDF42E0DA
:102C900050E0C701B601FF90EF90DF90CF90A3C343
:102CA000CF93DF93EB0191DF6AE070E0CE01DF911B
:102CB000CF9123C3CF92DF92EF92FF926A017B0103
:102CC00084DF4AE050E0C701B601FF90EF90DF904B
:102CD000CF900DC3811103C083E093E002C087E071
:102CE00093E073CFF7DF8AE000C2CF93DF931F92A8
:102CF0001F92CDB7DEB72091E70E3091E80ECE01DE
:102D000001962115310519F48D5E9E4002C0821B8B
:102D1000930B9A83898389819A810F900F90DF9119
:102D2000CF91089581E0089581E008958F929F9258
:102D3000AF92BF92CF92DF92EF92FF920F931F93C9
:102D4000CF93DF931F921F92CDB7DEB76C0159016D
:102D50008B017B01E40EF51E0E151F0561F1F601D6
:102D600080809180F80161918F016983C4016A8339
:102D70000E946EB76A81681779F0C4010E9476B725
:102D8000C4010E946EB79981891731F02CDF87E169
:102D900093E01BDF81E010C041E050E0BE016F5FB7
:102DA0007F4FC501F2DEF601408151814F5F5F4FD9
:102DB00051834083D1CF80E00F900F90DF91CF916E
:102DC0001F910F91FF90EF90DF90CF90BF90AF9049
:102DD0009F908F9008958F929F92AF92BF92CF92C3
:102DE000DF92EF92FF920F93CF93DF931F92CDB7B5
:102DF000DEB75C016B017A014901F50180819181A7
:102E00000E946EB78983002311F0F601808341E0B0
:102E100050E0BE016F5F7F4FC401B7DEF501408116
:102E200051814F5F5F4F51834083FFEFCF1ADF0A1D
:102E300081E0E81AF10809F780E00F90DF91CF9167
:102E40000F91FF90EF90DF90CF90BF90AF909F9049
:102E50008F90089598E288E10FB6F894A895809332
:102E600060000FBE9093600008951F920F920FB6FE
:102E70000F9211240BB60F920F931F932F933F9332
:102E80004F935F936F937F938F939F93AF93BF9372
:102E9000CF93DF93EF93FF930091CF03D091CE03B5
:102EA00011E01D0F1F77C091C6009091AA03492F12
:102EB000092E000C550B660B770B4C30510508F0B2
:102EC00046C0FA018827EA56FF4F8F4F0C941BB07B
:102ED000CD3441F0CE34B9F481E005C0CA3330F0CE
:102EE000CD3471F582E08093AA034AC0C03308F064
:102EF00047C0C03209F444C0CD3211F541C0C133DE
:102F000029F0C43329F0C032D9F43AC083E0EBCFC2
:102F100088E0E9CFC03321F0C13391F486E0E3CFFC
:102F200084E0E1CFC83361F485E0DDCFC23341F402
:102F300087E0D9CFC13321F489E0D5CFC03311F078
:102F40008BE0D1CF8AE0CFCFCA30D1F417C0CA30DE
:102F5000B9F480915904882389F0973049F09A3068
:102F600059F0953059F410926F021092E60E06C097
:102F700081E080935A0402C00E9407AA1092AA031B
:102F8000101731F0ED2FF0E0E253FC4FC283D12F48
:102F9000D093CE03FF91EF91DF91CF91BF91AF918D
:102FA0009F918F917F916F915F914F913F912F9161
:102FB0001F910F910F900BBE0F900FBE0F901F909F
:102FC00018951F920F920FB60F9211240BB60F9205
:102FD0002F938F939F93EF93FF938091AD03209155
:102FE000AC03281791F0E82FF0E0E455FC4F9281F4
:102FF0008F5F8F719093C6008093AD039091C00056
:1030000090649093C000281305C08091C1008F7D0B
:103010008093C100FF91EF919F918F912F910F901D
:103020000BBE0F900FBE0F901F9018959B01AC0127
:103030001092C000211581EE380741055105C1F0FD
:103040008091C00082608093C00060E079E08DE3F1
:1030500090E00E94FFAFCA01B90161507109810976
:10306000910922E030E040E050E00E94FFAF02C052
:1030700020E130E03093C5002093C4008091C1006E
:1030800080618093C1008091C10088608093C100FD
:103090008091C10080688093C1008091C1008F7DC4
:1030A0008093C1001092AB0308958091CE0390915C
:1030B000CF03891759F0E92FF0E0E253FC4F8281EA
:1030C0009F5F9F779093CF0390E008958FEF9FEFDE
:1030D0000895EEECF3E0808181830895EEECF3E057
:1030E00080819181891B8F77089591E09093AB0344
:1030F0009091C10095FD04C09091C00095FD40C025
:103100002091AC032F5F2F710FB607FC34C0909154
:10311000AD03291322C09091C00095FF1DC090916E
:10312000AD034091AC03491791F0E92FF0E0E4556D
:10313000FC4F32819F5F9F713093C6009093AD0327
:103140003091C00030643093C000491305C09091A5
:10315000C1009F7D9093C100DACFE091AC03F0E015
:10316000E455FC4F82832093AC038091C1008062C0
:103170008093C10008959091AD032913EECFFBCF4A
:103180008093C6008091C00080648093C000089541
:103190008DE0ABDF8AE0A9CFCF93DF93EC0189917B
:1031A000882311F0A2DFFBCFDF91CF91F1CF8F9277
:1031B0009F92AF92BF92EF92FF921F93CF93DF93B4
:1031C000CDB7DEB7A0970FB6F894DEBF0FBECDBF68
:1031D000611571058105910579F110E0842E912C1E
:1031E000A12CB12CEE24E394F12CEC0EFD1EE10E8B
:1031F000F11C17FDFA94A50194010E94DDAFF701BF
:103200006083B901CA011F5F6115710581059105D0
:1032100049F7115010F1E1E0F0E0EC0FFD1FE10F74
:10322000F11D17FDFA9580818A3010F097E301C0F7
:1032300090E3890F5ADFEDCF80E3A0960FB6F894A4
:10324000DEBF0FBECDBFDF91CF911F91FF90EF90FA
:10325000BF90AF909F908F9048CFA0960FB6F894F4
:10326000DEBF0FBECDBFDF91CF911F91FF90EF90DA
:10327000BF90AF909F908F900895CF92DF92EF9282
:10328000FF926B017C0197FF0AC08DE22EDFF09464
:10329000E094D094C094C11CD11CE11CF11C4AE004
:1032A000C701B601FF90EF90DF90CF9080CF41151E
:1032B000510511F4862F19CF4A30510509F4DDCF9D
:1032C00076CFAB01682F880F770B880B990BEFCF68
:1032D000AB01BC01990F880B990BE9CFAB01BC0185
:1032E000990F880B990BE3DF53CFE1DF51CF4115E5
:1032F000510511F4862FF9CE5ACFAB01BC0180E005
:1033000090E0F5CF8F929F92AF92BF92CF92DF92D3
:10331000EF92FF92CF936B017C01B42E20E030E05E
:10332000A9010E94B2AC87FF06C08DE2DEDEF7FA8B
:10333000F094F7F8F094C0E060E070E080E09FE384
:10334000CB1541F02DEC3CEC4CEC5DE30E94F0AE73
:10335000CF5FF6CF9B01AC01C701B6010E94D9AB8C
:103360006B017C010E9426AD4B015C014AE01FDF2E
:10337000CC2379F1C501B4010E9452AD9B01AC018F
:10338000C701B6010E94D8AB6B017C018EE2ADDEB5
:1033900020E030E040E251E4C701B6010E94F0AE07
:1033A0004B015C010E9421AD6B01770FEE08FF0815
:1033B000C701B60162DFC701B6010E9454AD9B018F
:1033C000AC01C501B4010E94D8AB6B017C01C150B6
:1033D000F9F6CF91FF90EF90DF90CF90BF90AF9034
:1033E0009F908F9008958ECFCF92DF92EF92FF92B1
:1033F0000F931F930E94681100915404109155047B
:1034000020915604309157046B017C01C01AD10AF7
:10341000E20AF30AF7FC52C08B019C010C53164FD1
:103420002F4F3F4F0093540410935504209356049C
:1034300030935704079B39C0069B37C0059B35C0A6
:103440002091B404211131C0049B2FC0009150047D
:10345000109151042091520430915304011511052B
:103460002105310571F0DC01CB01801B910BA20B12
:10347000B30B80569A4EA109B109B7FF02C068E7A5
:1034800001C060E060935804809102016111809551
:1034900088708093000170E086E01F910F91FF908B
:1034A000EF90DF90CF900C9434126093500470939F
:1034B00051048093520490935304C8CF1F910F91ED
:1034C000FF90EF90DF90CF90089581E080935904B2
:1034D0000895909115068917D1F00E94E15A8091C4
:1034E0001506882359F048E552E064E572E080E56E
:1034F00092E00E94A4591092150607C081E08093C3
:10350000150680E592E00E94125A0C94C14E08956F
:1035100080E0DFDF81EF95E00C9472A50F931F939D
:10352000CF93DF931F92CDB7DEB78C0181E493E098
:1035300069834BDBC80149DB6981662339F08AE086
:103540000F90DF91CF911F910F91CFCD0F90DF9111
:10355000CF911F910F91089561E088E393E0DECF52
:1035600061E081E393E0DACFEF92FF920F931F9334
:10357000CF93DF931F92CDB7DEB78C017B0180E242
:103580004983B3DD49814F3F11F084E501C082E4F6
:10359000ACDD8AE3AADDF8016081718182819381CB
:1035A00042E050E020DFF701408151816281738168
:1035B00083E593E055DB62E070E080E090E00F90FF
:1035C000DF91CF911F910F91FF90EF900C94991183
:1035D000FB01DC0112964D915D916D917C911597E7
:1035E000411551056105710599F080819181A28194
:1035F000B381841B950BA60BB70B80959095A09576
:10360000B0958827B7FD83959927AA27BB270895EA
:1036100080E00895811109C0CB016F3F710519F059
:1036200010F08FEF90E08093C704089597FF03C0D8
:103630008091B40409C027E1289FF001299FF00D73
:103640001124E853FB4F828590E008954F925F92DA
:103650006F927F928F929F92AF92BF92CF92DF92A2
:10366000EF92FF92CF93DF9300D01F92CDB7DEB7DA
:10367000E090D004F090D1048090CC049090CD04E0
:10368000A090CE04B090CF0420ED3CEC4CE45DE380
:103690006091DB047091DC048091DD049091DE0484
:1036A0000E94F0AE2B013C0120918C0430918D04DE
:1036B00040918E0450918F04C501B4010E94D8AB93
:1036C0009B01AC01C301B2010E94F0AE2B013C0191
:1036D00023E333E343E75FE3609188047091890457
:1036E00080918A0490918B040E94F0AE9B01AC0102
:1036F000C301B2010E94D9AB69837A838B839C8317
:10370000609388047093890480938A0490938B0457
:1037100080928C0490928D04A0928E04B0928F04BB
:10372000E114F104A1F0B701FF0C880B990B0E9482
:1037300054ADA50194010E94D8AB6B017C0120E03F
:1037400030E040E251EC0E94B2AC87FF07C081E05C
:1037500080937F04412C512C3201C1C020E030E025
:1037600040E251E4C701B6010E94B5AE181654F408
:1037700081E080937F04412C512C2FE7622E23E4BB
:10378000722EADC080917F04882351F010927B048B
:1037900010927C0410927D0410927E0410927F049B
:1037A00020917B0430917C0440917D0450917E04F3
:1037B000C701B6010E94D9AB4B015C0160937B0449
:1037C00070937C0480937D0490937E042091D304B5
:1037D0003091D4044091D5045091D604C701B6016C
:1037E0000E94F0AE2B013C01609380047093810431
:1037F00080938204909383042091D7043091D8045D
:103800004091D9045091DA04C501B4010E94F0AE90
:103810009B01AC01609384047093850480938604BB
:1038200090938704C301B2010E94D9AB29813A81E8
:103830004B815C810E94D8AB2B013C0120E030E041
:103840004FE753E40E94B5AE20E030E0A90118161E
:10385000DCF4C701B6010E94B5AE1816B4F5A70195
:103860009601C501B4010E94D8AB60937B047093AC
:103870007C0480937D0490937E04412C512C9FE71F
:10388000692E93E4792E2BC0C301B2010E94B2AC21
:1038900087FF25C020E030E0A901C701B6010E94E2
:1038A000B2AC87FF19C0A7019601C501B4010E94FF
:1038B000D8AB60937B0470937C0480937D049093D9
:1038C0007E04412C512C32010AC0412C512C8FE72F
:1038D000682E83E4782E03C0412C512C3201C301A1
:1038E000B2010F900F900F900F90DF91CF91FF904A
:1038F000EF90DF90CF90BF90AF909F908F907F9090
:103900006F905F904F9008954F925F926F927F9269
:103910008F929F92AF92BF92CF92DF92EF92FF92DF
:10392000CF93DF93CDB7DEB72C970FB6F894DEBFF9
:103930000FBECDBF8091AE049091AF04A091B004B2
:10394000B091B10489839A83AB83BC836091B20444
:103950007091B304072E000C880B990B0E9454AD94
:1039600029813A814B815C810E94D8AB6B017C013B
:1039700020917704309178044091790450917A0431
:103980000E94D9AB4B015C0160937704709378047B
:103990008093790490937A042091B5043091B60411
:1039A0004091B7045091B804C701B6010E94F0AE2F
:1039B0006D837E838F83988760936B0470936C0410
:1039C00080936D0490936E042091B9043091BA04F1
:1039D0004091BB045091BC04C501B4010E94F0AEFB
:1039E00069877A878B879C8760936F0470937004D4
:1039F000809371049093720420ED3CEC4CE45DE301
:103A00006091BD047091BE048091BF049091C00488
:103A10000E94F0AE2B013C012091670430916804B4
:103A20004091690450916A0469817A818B819C81FB
:103A30000E94D8AB9B01AC01C301B2010E94F0AE61
:103A40002B013C0123E333E343E75FE3609173041D
:103A50007091740480917504909176040E94F0AE88
:103A60009B01AC01C301B2010E94D9AB2B013C0107
:103A70006093730470937404809375049093760438
:103A800089819A81AB81BC8180936704909368049B
:103A9000A0936904B0936A0429853A854B855C85B7
:103AA0006D817E818F8198850E94D9ABA30192019F
:103AB0000E94D8AB2B013C0120E030E04FE753E4FB
:103AC0000E94B5AE20E030E0A9011816DCF4C70171
:103AD000B6010E94B5AE1816B4F5A7019601C5014E
:103AE000B4010E94D8AB60937704709378048093FC
:103AF000790490937A04412C512C9FE7692E93E42A
:103B0000792E2BC0C301B2010E94B2AC87FF25C041
:103B100020E030E0A901C701B6010E94B2AC87FFE6
:103B200019C0A7019601C501B4010E94D8AB6093EA
:103B30007704709378048093790490937A04412CED
:103B4000512C32010AC0412C512C8FE7682E83E49E
:103B5000782E03C0412C512C3201C301B2012C96A6
:103B60000FB6F894DEBF0FBECDBFDF91CF91FF90AF
:103B7000EF90DF90CF90BF90AF909F908F907F900D
:103B80006F905F904F9008954F925F926F927F92E7
:103B90008F929F92AF92BF92CF92DF92EF92FF925D
:103BA0000F931F93CF93DF933C01C62F662389F0B9
:103BB0001DD86AE070E08C2F90E08ADB86E893E005
:103BC00004D880E090E00E944CAA60E070E0CB0155
:103BD0007AC0B0E2A0E06A2F70E0AB014B0F511D3C
:103BE000559547954A1711F04B130BC0E8E4F7E0E1
:103BF00065917491072E000C880B990B0E9454ADAF
:103C000062C0CA010197880F991F880F991FFC0194
:103C1000E653F94F059114919A01220F331F220F99
:103C2000331FF901E653F94FC591D491601671061F
:103C300014F4B42FD2CFA42FC615D7050CF4CBCFD4
:103C40008453994FFC01E590F490F901E453F94F46
:103C5000C590D490B7010F2C000C880B990B0E94D3
:103C600054AD4B015C01B301601B710B072E000CBE
:103C7000880B990B0E9454AD2B013C01B6016E19C3
:103C80007F09072E000C880B990B0E9454AD9B01F5
:103C9000AC01C301B2010E94F0AE6B017C01C01BFC
:103CA000D10BBE01DD0F880B990B0E9454AD9B0117
:103CB000AC01C701B6010E94B9AC9B01AC01C501C2
:103CC000B4010E94D9ABDF91CF911F910F91FF906A
:103CD000EF90DF90CF90BF90AF909F908F907F90AC
:103CE0006F905F904F9008954F925F926F927F9286
:103CF0008F929F92AF92BF92CF92DF92EF92FF92FC
:103D00000F931F93CF93DF933C01BAE3A0E06A2F98
:103D100070E0AB014B0F511D559547954A1711F0B7
:103D20004B130BC0E8ECF6E065917491072E000C84
:103D3000880B990B0E9454AD62C0CA010197880F8D
:103D4000991F880F991FFC01EE51FA4F05911491AC
:103D50009A01220F331F220F331FF901EE51FA4F40
:103D6000C591D4916016710614F4B42FD2CFA42F4C
:103D7000C615D7050CF4CBCF8C519A4FFC01E590BA
:103D8000F490F901EC51FA4FC590D490B7010F2C83
:103D9000000C880B990B0E9454AD4B015C01B301E0
:103DA000601B710B072E000C880B990B0E9454AD01
:103DB0002B013C01B6016E197F09072E000C880B00
:103DC000990B0E9454AD9B01AC01C301B2010E944A
:103DD000F0AE6B017C01C01BD10BBE01DD0F880B67
:103DE000990B0E9454AD9B01AC01C701B6010E9422
:103DF000B9AC9B01AC01C501B4010E94D9ABDF9104
:103E0000CF911F910F91FF90EF90DF90CF90BF90D7
:103E1000AF909F908F907F906F905F904F9008959C
:103E2000CF93DF93C8ECD4E060E08A819B81ACDE65
:103E30006C837D838E839F83CAEAD4E08A819B81D1
:103E400053DF6C837D838E839F83A8951092A0049B
:103E5000DF91CF910895CF93DF93CDB7DEB7609711
:103E60000FB6F894DEBF0FBECDBF9C01E62F660FE4
:103E7000FF0BED51FE4FE4918E2F90E0FC01379740
:103E8000EC30F10508F0BFC08827EE55FF4F8F4F8B
:103E90000C941BB091E001C090E080E1FE013196EE
:103EA000DF01482F1D924A95E9F740EB50E05A8315
:103EB000498341EB50E05C834B8343EB50E05887F0
:103EC0004F8344EB50E05A87498742E04F87988BF5
:103ED000D90101900D928A95E1F7A2C081E001C05D
:103EE00080E08F5F01C080E040E950E0D901119689
:103EF0005C934E9341E950E013965C934E93129776
:103F000042E950E015965C934E93149748E950E0CF
:103F100017965C934E9316974AE950E019965C9376
:103F20004E9318974CE950E01B965C934E931A976A
:103F300046E950E01D965C934E931C9793E01E96C5
:103F40009C931E971F968C936BC081E001C080E00C
:103F50008F5F01C080E040EA50E0F9015183408367
:103F600041EA50E05383428342EA50E05583448360
:103F700048EA50E0578346834AEA50E05187408739
:103F80004CEA50E05387428746EA50E05587448721
:103F900094E09687878744C081E001C080E08F5F0E
:103FA00001C080E040E251E0D90111965C934E934C
:103FB00041E251E013965C934E93129742E251E036
:103FC00015965C934E93149748E251E017965C93D4
:103FD0004E9316974AE251E019965C934E931897C8
:103FE0004CE251E01B965C934E931A9746E251E0E7
:103FF0001D965C934E931C9795E01E969C931E977E
:104000001F968C930DC080E1FE013196DF01482F91
:104010001D924A95E9F7D90101900D928A95E1F731
:10402000C90160960FB6F894DEBF0FBECDBFDF9119
:10403000CF9108952F923F924F925F926F927F920D
:104040008F929F92AF92BF92CF92DF92EF92FF92A8
:104050000F931F93CF93DF93CDB7DEB7AE970FB615
:10406000F894DEBF0FBECDBF7CA36BA3682FCE013B
:104070004196F1DE2B893C893EA32DA33F8D3AA3C7
:10408000332309F429C1323021F0EE24EA94FE2CC6
:1040900003C0EE24EA94F12C4BA15CA1452B09F45A
:1040A000E0C09701322F2227330F330F330F40E048
:1040B00050E060E074E284EF90E00E94FFAF5901AD
:1040C0008FEFA81AB80A80E1E1E7F2E0DE0111966D
:1040D00001900D928A95E1F7FE013196F8A7EFA3C2
:1040E00001E011E019A288248A94912C412C94E2D9
:1040F000592E94EF692E712CFAA1F23059F1033048
:1041000009F4A4C0053009F4A1C0EFA1F8A582818B
:1041100093812BA13CA1289F6001299FD00C389F3F
:10412000D00C1124960140E050E0C301B2010E947E
:10413000FFAF190181E0281A31089601220F331FC1
:1041400040E050E0C301B2010E94FFAF21143104EE
:1041500031F40AC02FEF30E022242A94312CE214EB
:10416000F30428F4170103C022242394312C2115D1
:10417000310531F06901E216F30628F4670103C046
:10418000CC24C394D12CEFA1F8A50280F381E02DBB
:10419000FEA7EDA7C10101968E9F90018F9F300D64
:1041A0009E9F300D112440E050E0C301B2010E94F7
:1041B000FFAF29A73AA74BA75CA78DA59EA5880F9F
:1041C000991F8C9D90018D9D300D9C9D300D11246B
:1041D00040E050E0C301B2010E94FFAF69A57AA59B
:1041E0008BA19CA1681B790B77FF03C0719561952A
:1041F0007109D501EBA1FCA1AE1BBF0BB7FF03C03A
:10420000B195A195B109C901EBA1FCA18E1B9F0B32
:104210006A177B075CF4FC0197FF04C0EE27FF27B9
:10422000E81BF90BE617F7070CF049C097FF03C02E
:104230009195819591098A179B0744F4FAA1590138
:1042400009A34601F23009F045C011E00F5F2FA12C
:1042500038A52E5F3F4F38A72FA3083009F04CCF69
:1042600005C011E019A288248A94912CE989FA8961
:104270008081912F93708C7F892B8083EDA1FEA18B
:104280002081812F90E0959587959595879543E0BE
:10429000880F991F4A95E1F7122F177E812B808393
:1042A000808199A19770887FF92EF82AF082FAA16F
:1042B000F23091F0ED8DFE8D918280820DC02AA1A9
:1042C000A9A4BAA409A34101223011F01EE0BECF77
:1042D00013E0BCCF1AE0BACFAE960FB6F894DEBFAB
:1042E0000FBECDBFDF91CF911F910F91FF90EF9047
:1042F000DF90CF90BF90AF909F908F907F906F9006
:104300005F904F903F902F9008956D9A759880918F
:10431000010180618093010180910201807180938D
:104320000001809101018860809301018091020168
:104330008870809300019D9AA59880910101806208
:10434000809301016AE770E088E074DE80910101EA
:104350008860809301016AE770E086E06BDE87ED9C
:1043600080937A0010927E0010927D0080917E00F2
:10437000816080937E0080917E00846080937E00C7
:1043800080E888BD80916E00846080936E006AEF43
:1043900070E080E090E00E94991185E090E09093B9
:1043A0001A028093190260E0809115029091160222
:1043B000EBDB20E030E040EA50E40E94B2AC87FF43
:1043C0000AC08091150290911602409790931602B0
:1043D00080931502E8CF81E391E090931C028093D3
:1043E0001B0260E08091150290911602CDDB20E067
:1043F00030E848E953E40E94B5AE181654F48091B1
:104400001702909118024096909318028093170219
:10441000E8CF80911F029091200266DC20E030E01E
:1044200040EA50E40E94B2AC87FF0AC080911F02AC
:104430009091200240979093200280931F02E9CF31
:104440008091A8049091A9044FDC20E030E046E17F
:1044500053E40E94B5AE181654F480911F02909157
:10446000200240969093200280931F02E9CF089586
:104470004F925F926F927F92AF92BF92CF92DF92F4
:10448000EF92FF920F931F93CF93DF93CDB7DEB7D9
:1044900060970FB6F894DEBF0FBECDBF61157105F2
:1044A00011F4622F05C064177507C1F461E062273B
:1044B00060960FB6F894DEBF0FBECDBFDF91CF91EF
:1044C0001F910F91FF90EF90DF90CF90BF90AF9032
:1044D0007F906F905F904F900C948D13D22E8A0135
:1044E0007B01682FCE010196B6DC5F85E8895523F4
:1044F00009F44BC0A981BA814C91F0E083E090E0CF
:10450000BC016E1B7F0B660F771F2D2D30E02E5FD9
:104510003F4F062E01C0220F0A94EAF701C0880F10
:104520006A95EAF780958423282B2C93523029F042
:10453000AD85BE85CD90DC9003C0CC24CA94D12C2F
:104540003396EE0FFF1F81E090E08C0F9D1FE80F68
:10455000F91FA080B180B70180E090E00E9452ADC9
:104560002B013C01C601B8010E94C9AF80E090E078
:104570000E9452AD9B01AC01C301B2010E94F0AE9A
:104580000E9421ADF5017183608360960FB6F894A7
:10459000DEBF0FBECDBFDF91CF911F910F91FF9076
:1045A000EF90DF90CF90BF90AF907F906F905F9033
:1045B0004F900895CF92DF92EF92FF928091D004B6
:1045C0009091D1040097B9F0C090CC04D090CD0464
:1045D000E090CE04F090CF040D97BC01990F880BAA
:1045E000990B0E9454AD9B01AC01C701B6010E941A
:1045F000B2AC87FD09C01092C3041092C40410929B
:10460000C5041092C6041EC020E030E040E050E433
:10461000C701B6010E94D9AB0E9426AD7093C204B7
:104620006093C1040E946811DC01CB01805E914B54
:10463000AF4FBF4F8093C3049093C404A093C504AD
:10464000B093C604FF90EF90DF90CF900895CF9283
:10465000DF92EF92FF928091B2049091B3040097A1
:10466000B9F0C090AE04D090AF04E090B004F090E8
:10467000B1040897BC01990F880B990B0E9454ADA7
:104680009B01AC01C701B6010E94B2AC87FD09C015
:104690001092A4041092A5041092A6041092A704EC
:1046A0001EC020E030E040E050E4C701B6010E94A7
:1046B000D9AB0E9426AD7093A3046093A2040E941C
:1046C0006811DC01CB01805A9541AF4FBF4F8093F9
:1046D000A4049093A504A093A604B093A704FF900C
:1046E000EF90DF90CF90089580911B0290911C0273
:1046F0000F971816190614F480E090E09093D104F7
:104700008093D00480E056DF1092B3041092B2047C
:104710009EDF80911B0290911C020F9718161906BC
:1047200014F480E090E09093D1048093D00480E072
:1047300041DF1092D20475981092B3041092B20423
:104740001092B404A5980895EF92FF920F931F93CF
:10475000CF93C82F7B018A01809170028823D1F00A
:104760000E94F615C7010E94E51588E294E00E94B8
:10477000E515C7FD08C06AE070E08C2FCC0F990BDF
:104780000E94681904C084E294E00E94E5158AE062
:104790000E9475188091900481110DC010927002D2
:1047A00081E080939004C801CF911F910F91FF90F9
:1047B000EF900C944CAACF911F910F91FF90EF9026
:1047C00093CF8F3F19F040E154E002C040E254E043
:1047D0006EEF73E0B9CF8F3F19F04AEE53E002C09D
:1047E0004AEF53E068ED73E0AFCF2F923F924F92C4
:1047F0005F926F927F928F929F92BF92CF92DF9241
:10480000EF92FF920F931F93CF93DF936C014B01B5
:10481000B22E180127FD04C0C22F220FDD0B02C0EB
:10482000C1E0D0E0FA014080518062807380CC0FFB
:10483000DD1FCC0FDD1F8E01015A1B4FA30192011A
:10484000F80160817181828193810E94B2AC8823DA
:1048500091F0F801408251826282738211E020E07F
:1048600030E0A901C301B2010E94B5AE18160CF0E8
:1048700010E0F6011483F60184818230C9F08330A0
:1048800009F456C0813009F070C0FE01E15AFB4FB7
:104890002081318142815381F40160817181828163
:1048A00093810E94B2AC87FD60C082E0F6018483F0
:1048B000C15ADB4FB70180E090E00E9452AD9B01EE
:1048C000AC01688179818A819B810E94D8AB9B0170
:1048D000AC01F40160817181828193810E94B5AE47
:1048E00087FD15C00E9468112B013C019101A8EEC3
:1048F000B3E00E9423B0DC01CB01840D951DA61D01
:10490000B71DF60180839183A283B3832EC00E94DA
:104910006811F6010081118122813381DC01CB0114
:10492000801B910BA20BB30BB7FD1FC083E08483E8
:10493000FFEFBF1619F04FE653E002C042E853E024
:104940006FE573E08B2DDF91CF911F910F91FF9059
:10495000EF90DF90CF90BF909F908F907F906F905F
:104960005F904F903F902F90EFCEDF91CF911F91AE
:104970000F91FF90EF90DF90CF90BF909F908F901E
:104980007F906F905F904F903F902F900895CF92BF
:10499000DF92EF92FF920F931F93CF93DF93CDB7E8
:1049A000DEB728970FB6F894DEBF0FBECDBF80915B
:1049B0005A04811113C08091A004811114C028965B
:1049C0000FB6F894DEBF0FBECDBFDF91CF911F9120
:1049D0000F91FF90EF90DF90CF90089580E090E0EE
:1049E0000E944CAAE8CF1CDA0E9468116D837E8376
:1049F0008F839887809113029091140218161906DC
:104A00000CF0F3C00197909314028093130260910D
:104A1000D0047091D104072E000C880B990B0E94D2
:104A200054AD69837A838B839C833EE1E32EF12C22
:104A30000FE010E020E0AE014F5F5F4F6CEC74E0E0
:104A40008BE994E0D2DEC090CC04D090CD04E0900D
:104A5000CE04F090CF048091190290911A02BC010B
:104A6000990F880B990B0E9454AD9B01AC01C701B3
:104A7000B6010E94B5AE1816D4F460911B02709175
:104A80001C02072E000C880B990B0E9454AD9B0151
:104A9000AC01C701B6010E94B2AC87FF08C080E03C
:104AA0000E94261B0E9421AD7595679501C060E0AC
:104AB0006093D2048091C3049091C404A091C50472
:104AC000B091C6040097A105B10541F14D815E8109
:104AD0006F8178858A019B01081B190B2A0B3B0B00
:104AE00037FD1CC06091C1047091C20480E090E069
:104AF0000E9452AD9B01AC016091CC047091CD0439
:104B00008091CE049091CF040E94B2AC87FF8EC0FA
:104B100046EC53E067EB73E080E016DEBE016B5FAE
:104B20007F4F82EA94E00E94E81A8823D9F06091CE
:104B3000A2047091A30480E090E00E9452AD209105
:104B4000AE043091AF044091B0045091B1040E9482
:104B5000B5AE18160CF068C043EB53E064EA73E09E
:104B60008FEFF2DD6091B2047091B304072E000C58
:104B7000880B990B0E9454AD69837A838B839C8345
:104B80009AE0E92EF12C0FE010E02FEFAE014F5F1D
:104B90005F4F6EEA74E086E994E027DEC090AE04D1
:104BA000D090AF04E090B004F090B10420E030E089
:104BB00040EA50E4C701B6010E94B5AE87FD0AC0C5
:104BC00020E030E046E153E4C701B6010E94B2ACF8
:104BD000181624F460E06093B404F1CE0E94841CA3
:104BE0000E9421AD75956795F6CFC090CC04D0900A
:104BF000CD04E090CE04F090CF0420E030E848E906
:104C000053E4C701B6010E94B5AE181694F020E037
:104C100030E040EA50E4C701B6010E94B2AC87FF21
:104C2000F6CE80E0D8DDF3CE12DD9CCF80E0C2DC92
:104C300075CF80E0C6DDC090CC04D090CD04E0906C
:104C4000CE04F090CF04E3CFE8ECF4E080819181D2
:104C500093838283EAEAF4E0808191819383828363
:104C600081E08093A00408951F93CF93DF938091F8
:104C7000A004811101C0E8DF1092C9041092C80499
:104C80001092AB041092AA04C091CA04D091CB0434
:104C9000D195C195D1098091D0049091D10411E0B2
:104CA000181619062CF08091D204811101C010E071
:104CB00080911702909118029195819591098C1716
:104CC0009D0714F480E07DDD112361F080911502D1
:104CD00090911602919581959109C817D90714F4FE
:104CE00080E079DD8091B2049091B304C1E01816A0
:104CF00019062CF08091B404811101C0C0E020910C
:104D0000AC043091AD048091A8049091A90482175D
:104D1000930714F08FEF55DDCC2381F020911F0213
:104D2000309120028091AC049091AD0482179307DA
:104D30002CF08FEFDF91CF911F914DCDDF91CF916F
:104D40001F9108950F930FB70F9300916E000B7F83
:104D500000936E0078940F930BB70F930CB70F92DC
:104D60001F922F933F934F935F936F937F938F93F4
:104D70009F93AF93BF93EF93FF931124C7D0FF91FD
:104D8000EF91BF91AF919F918F917F916F915F91C3
:104D90004F913F912F911F900F900CBF0F910BBF20
:104DA0000F910460F89400936E000F910FBF0F9164
:104DB0001895CF93809112028F3790F08F57909172
:104DC000D20490935E04992311F0759A01C07598EE
:104DD0009091B40490935D04992359F0A59A0AC068
:104DE00090915E04891708F0759890915D04891779
:104DF00008F0A598805F8093120290915C0481E096
:104E0000892780935C048091110285301CF4C1E0F5
:104E1000C80F01C0C0E08230A1F184F4882329F1D9
:104E2000813009F062C010927B0080E480937C00A6
:104E300080917A00806480937A0057C0843009F4AE
:104E40003EC094F1853009F050C090915B049111FF
:104E500002C080935B0480915B04815080935B046B
:104E6000882309F442C0C5E040C0809110028F5FE2
:104E700080311CF48093100238C010921002F4DECE
:104E800034C080917A0086FD2DC080917800909189
:104E900079002091C8043091C904820F931F909328
:104EA000C9048093C80421C010927B0082E48093DF
:104EB0007C0080917A00806480937A0016C0809193
:104EC0007A0086FD11C08091780090917900209140
:104ED000AA043091AB04820F931F9093AB0480938C
:104EE000AA0403C0C2E001C0C4E0C09311020E9442
:104EF000C73180918F0690919006009729F0019715
:104F00009093900680938F06CF91089552CFFF9291
:104F10000F931F93CF93DF93CDB7DEB728970FB6CC
:104F2000F894DEBF0FBECDBFF82E08EC14E0F801F8
:104F300060857185072E000C880B990B0E9454AD7B
:104F400069837A838B839C83F80184819581A68110
:104F5000B7818D839E83AF83B8874DEFBE016F5FAE
:104F60007F4FCE0105960E94B41A0AEA14E0F801B8
:104F700060857185072E000C880B990B0E9454AD3B
:104F800069837A838B839C83F80184819581A681D0
:104F9000B7818D839E83AF83B8874FEFBE016F5F6C
:104FA0007F4FCE0105960E94B41A8BE593E00E94D4
:104FB000E5158F2D90E00E94161B6AE070E00E94BC
:104FC000681986E593E00E94E515F80182856AE09C
:104FD00070E090E00E94681928960FB6F894DEBF42
:104FE0000FBECDBFDF91CF911F910F91FF9008951C
:104FF0002F923F924F925F926F927F928F929F92E9
:10500000AF92BF92CF92DF92EF92FF920F931F93D6
:10501000CF93DF93CDB7DEB7CD54D1090FB6F89457
:10502000DEBF0FBECDBF2E969FAF8EAF2E97162F31
:10503000742E26962FAF26970E946811688B798B65
:105040008A8B9B8B17FD04C0A4E1EA2EF12C03C0D0
:10505000FCE3EF2EF12C2E96AEADBFAD2E972D9129
:105060003D914D915C912FA738AB49AB5AAB17FDE1
:1050700090C4C12E012E000CDD08F60183E0EE0F76
:10508000FF1F8A95E1F7EB5EFD4F668177816F50D8
:105090007109072E000C880B990B0E9454AD9B01DF
:1050A000AC016FA578A989A99AA90E94B5AE181676
:1050B000ECF487EB95E0C35BDF4F0FB6F894DEBFEF
:1050C0000FBECDBFDF91CF911F910F91FF90EF9059
:1050D000DF90CF90BF90AF909F908F907F906F9018
:1050E0005F904F903F902F900C94E51583EA95E0E8
:1050F0000E94E515F9DA27E12C9DC0012D9D900D48
:105100001124FC01E853FB4F2FE7228780E090E059
:10511000A0E5B1E423968CAF9DAFAEAFBFAF2397B0
:105120009701A8EEB3E00E9423B06BAF7CAF8DAFC8
:105130009EAF9B01AC0188899989AA89BB89280FF8
:10514000391F4A1F5B1F2BAB3CAB4DAB5EAB81E005
:1051500080936F0288889988AA88BB888EA29FA2B4
:10516000A8A6B9A6188E198E1A8E1B8E1C8A1D8AA7
:105170001E8A1F8A1A821B821C821D821A8690E454
:105180009C8FACE1AD8FB6E4BE8F1F8E18A219A222
:105190001AA21EA61FAA18AE19AE1AAE2FE730E04B
:1051A00040E050E02E833F8348875987EFE7CE2EBB
:1051B000D12CE12CF12C1AA61BA61CA61DA631E0B1
:1051C0003BA31F861E86212C312C00E0198247E16B
:1051D0001402C001112488539B4FDC011A962596B6
:1051E000BFAFAEAF2597FC013496FDA3ECA3272DEE
:1051F000770C330B28963FAF2EAF289780916F0224
:10520000882309F48FC20E9468112B013C01809110
:10521000A004882309F4FAC00E94101F17FF0AC0D7
:105220002090AE043090AF040091B0043091B104EE
:1052300039830CC0ACA1BDA12C9011963C90119764
:1052400012960C9112971396BC91B9839101402F3D
:1052500059816F8D78A189A19AA10E94B2AC87FF74
:1052600005C02F8E38A209A3E981EAA39101402F3E
:1052700059816A857C8D8D8D9E8D0E94B5AE1816E4
:105280002CF42A863C8E0D8FF981FE8F2BA12223D0
:1052900009F463C02E96AEADBFAD2E972D913D9112
:1052A0004D915C91B101802F99810E94B5AE181685
:1052B0000CF0ACC0A3019201281939094A095B0915
:1052C0002C962CAF3DAF4EAF5FAF2C97DA01C901E2
:1052D00088589341A109B109B7FD98C0D701C6010B
:1052E0002E813F8148855985821B930BA40BB50BFA
:1052F000B595A7959795879517FF03C08093B4043C
:1053000005C02596EEADFFAD259780832C962CAD7C
:105310003DAD4EAD5FAD2C972AA73BA74CA75DA72F
:105320002E96AEADBFAD2E97BC91BF8F2E96EEAD33
:10533000FFAD2E97F181F8A32E96AEADBFAD2E979F
:105340001296BC91B9A32E96EEADFFAD2E97F381C8
:10535000FAA34EA25FA268A679A62E96AEADBFAD07
:105360002E972D913D914D915C91B101802F9981A6
:105370000E94B2AC87FF0BC3D301C2012EA13FA193
:1053800048A559A5821B930BA40BB50BAC01BD011D
:10539000485853416109710977FDF9C24E855F850F
:1053A000452B09F0DAC18E819F81A885B9858C0DC6
:1053B0009D1DAE1DBF1DB595A7959795879517FFA8
:1053C000E0C28093B4042E853F852F5F3F4F3F8717
:1053D0002E872E96AEADBFAD2E97BC91BA872E9676
:1053E000EEADFFAD2E97F181FC8F2E96AEADBFAD29
:1053F0002E971296BC91BD8F2E96EEADFFAD2E97D7
:10540000F381FE8F5301420121E02BA320E030E025
:1054100040EA51E42E96AEADBFAD2E976D917D91D1
:105420008D919C910E94D9AB9B01AC01B101802F61
:1054300099810E94B5AE18162CF48FE295E00E9477
:10544000E51570C1D301C201288939894A895B8970
:10545000821B930BA40BB50BB7FD8BC0812F17FDDF
:1054600080E055DD8AE00E947518D301C2018053A7
:10547000984FAF4FBF4F888B998BAA8BBB8B9EA544
:10548000911155C02FA938AD49AD5AADB101802F4A
:1054900099810E94B5AE181694F520E030E040E006
:1054A00050E4B101802F99810E94D9AB6FAB78AFE6
:1054B00089AF9AAF2BAD3CAD4DAD5EAD240D351D22
:1054C000461D571D2BAB3CAB4DAB5EAB23962CADB5
:1054D0003DAD4EAD5FAD23976FA578A989A99AA977
:1054E0000E94D8AB9B01AC0181E08EA7B101802F57
:1054F00099810E94B5AE1816E4F11EA63AC0D301F8
:10550000C2012BA93CA94DA95EA9821B930BA40B38
:10551000B50BB7FD2EC01F3F19F049E155E002C0A1
:105520004BE255E06AE075E0812F0ED922C020E001
:1055300030E040EA51E42E96AEADBFAD2E976D91AE
:105540007D918D919C910E94D8AB9B01AC01B101E2
:10555000802F99810E94B2AC87FF0BC01F3F19F0CA
:1055600043EF54E002C046E055E063EE74E0812F63
:10557000EBD8D301C201880F991FAA1FBB1F2EA110
:105580003FA148A559A5821B930BA40BB50B881905
:105590009909AA09BB0981389F44A241B10528F0A5
:1055A00085EC94E00E94E515BDC04E855F85289688
:1055B0008EAD9FAD2897841795070CF01FCE433012
:1055C00051050CF41BCE88E694E00E94E51517FD0A
:1055D00005C023E6E22E24E0F22E04C094E6E92E74
:1055E00094E0F92E86E494E00E94E515C7010E943C
:1055F000E5154A815B816C817D818FE594E00E9495
:1056000030168AE00E94751886E494E00E94E51541
:10561000C7010E94E5154C895D896E897F898BE5FC
:1056200094E00E9430168AE00E94751886E494E0A7
:105630000E94E515C7010E94E515488D598D6A8DB8
:105640007B8D87E594E00E9430168AE00E947518F1
:1056500026969FAD2697992309F4BCC117FF31C048
:105660002A813B814C815D812093B5043093B6043F
:105670004093B7045093B8042CEA35EC47E25EE35C
:105680006C897D898E899F890E94F0AE6093B904F0
:105690007093BA048093BB049093BC042CEA35EC5D
:1056A00047E25EE3688D798D8A8D9B8D0E94B9AC4F
:1056B0006093BD047093BE048093BF049093C004B4
:1056C00089C147E1140290011124890108531B4F3D
:1056D0008A819B81AC81BD81F80183879487A587EE
:1056E000B6872CEA35EC47E25EE36C897D898E89CA
:1056F0009F890E94F0AED8011F966D937D938D9384
:105700009C9352972CEA35EC47E25EE3688D798DE5
:105710008A8D9B8D0E94B9ACF801638B748B858B4D
:10572000968B58C1C35BDF4F0FB6F894DEBF0FBE38
:10573000CDBFDF91CF911F910F91FF90EF90DF9040
:10574000CF90BF90AF909F908F907F906F905F9021
:105750004F903F902F900C9474238AA49BA4ACA4E8
:10576000BDA4880E991EAA1EBB1E2AA53BA54CA54A
:105770005DA5281B390B4A0B5B0BCA01B9012E81B1
:105780003F81488559850E94BAAFA50194010E94C6
:10579000FFAFD701C601820F931FA41FB51F84312D
:1057A0009105A105B105FCF06C017D018C3E9105D0
:1057B000A105B1052CF06BEEC62ED12CE12CF12CFD
:1057C00040E8C416D104E104F104DCF08EEF90E06F
:1057D000A0E0B0E08C199D09AE09BF098E839F83BC
:1057E000A887B98712C054E1C52ED12CE12CF12C29
:1057F00024E130E040E050E02E833F834887598722
:1058000004C0CE82DF82E886F986B701A6018BE963
:1058100095E00E9420164E815F816885798586E932
:1058200095E00E9420164A855C8D6D8D7E8D8FE8F7
:1058300095E00E9430164F8D58A169A17AA188E8A1
:1058400095E00E9430164E855F85433051050CF47B
:10585000AACD6E817F81888599850E9454AD20E014
:1058600030E040E850E40E94F0AE6A837B838C8392
:105870009D832A853C8D4D8D5E8D6F8D78A189A18C
:105880009AA10E94D8AB2BED3FE049E450E40E947E
:10589000F0AE20E030E040E05FE30E94F0AE9B011C
:1058A000AC016A817B818C819D810E94B9AC6A8741
:1058B0007B878C879D87C501B4010E9454AD2FE67C
:1058C00032E143E85AE30E94F0AE4B015C012AE961
:1058D00039E949E15FE36A857B858C859D850E9476
:1058E000F0AE6A837B838C839D839B01AC010E9415
:1058F000D9ABA50194010E94B9AC6C8B7D8B8E8BCA
:105900009F8BA50194016A817B818C819D810E947E
:10591000F0AE20E030E040E05EE30E94F0AE688F41
:10592000798F8A8F9B8F4A855B856C857D8582E820
:1059300095E00E943016B501A4018CE795E00E9425
:1059400030168CE695E00E94E5154A815B816C81FA
:105950007D8186E695E00E9430164C895D896E89CE
:105960007F8980E695E00E943016488D598D6A8DBA
:105970007B8D8AE595E00E9430168AE00E947518BA
:1059800012CD2596EEADFFAD259780831CCD1BA2D1
:105990003DCD20E030E047E053E46FA578A989A928
:1059A0009AA90E94B5AE18160CF483CB83EA95E051
:1059B0000E94E5150E9474238FE78093B40420E0D1
:1059C00030E040E051E423962CAF3DAF4EAF5FAFE7
:1059D0002397A6CBC35BDF4F0FB6F894DEBF0FBE95
:1059E000CDBFDF91CF911F910F91FF90EF90DF908E
:1059F000CF90BF90AF909F908F907F906F905F906F
:105A00004F903F902F900895CF92DF92EF92FF92A8
:105A1000809195048823A1F10E946811C09091049F
:105A2000D0909204E0909304F0909404DC01CB01B8
:105A30008C199D09AE09BF09B7FD22C00E946811EB
:105A40006B017C012091950430E0A8EEB3E00E9448
:105A500023B0DC01CB018C0D9D1DAE1DBF1D8093BD
:105A6000910490939204A0939304B093940480E0E3
:105A70004EDA8AE0FF90EF90DF90CF900C9475188B
:105A8000FF90EF90DF90CF9008952F923F924F922A
:105A90005F926F927F928F929F92AF92BF92CF92BE
:105AA000DF92EF92FF920F931F93CF93DF93CDB7C7
:105AB000DEB764970FB6F894DEBF0FBECDBF898BFB
:105AC0006A8B81E080936F021A821B821C821D8286
:105AD00019861A861B861C8621E0288719821D8656
:105AE0003CE33E874CE14F8756E4588BC12CD12CC8
:105AF00080E8E82E9FEBF92E812C912C54016091C7
:105B0000D0047091D104072E000C880B990B0E94D1
:105B100054AD6B8B7C8B182F092F9B01482F592F6D
:105B2000B601C7010E94B2AC882399F12091CC0440
:105B30003091CD044091CE045091CF046B897C8983
:105B4000812F902F0E94B2AC881F8827881F8983DD
:105B50008A89882311F199819923F9F080916F0244
:105B600064960FB6F894DEBF0FBECDBFDF91CF9124
:105B70001F910F91FF90EF90DF90CF90BF90AF906B
:105B80009F908F907F906F905F904F903F902F905D
:105B90000895CB8ADC8A1E2D0F2D0E9468116B019F
:105BA0007C01DC01CB0129853A854B855C85821B14
:105BB000930BA40BB50BB7FD34C0D701C6018851B8
:105BC0009C4FAF4FBF4F89879A87AB87BC87898926
:105BD0009ED98FE493E00E94E51581149104A104FD
:105BE000B104C9F0D501C40188519C4FAF4FBF4FDC
:105BF000BC01CD016C197D098E099F0928EE33E0A7
:105C000040E050E00E94DDAFCA01B9014AE050E037
:105C10000E94571903C08FE30E9475188AE00E9402
:105C200075180E9440AB0E9468116093FF0B70933F
:105C3000000C8093010C9093020C2090CC043090C7
:105C4000CD049091CE049E83A091CF04AF839101A7
:105C5000492F5A2F6B897C89812F902F0E94D8ABB6
:105C60002B013C0120E030E0A9010E94B5AE87FF86
:105C700004C0C301B201905802C0C301B20120E0C8
:105C800030E040E251E481149104A104B10481F4B4
:105C90000E94B2AC87FF12C0B88546015701BB23F2
:105CA00069F0E8EE8E0EE3E09E1EA11CB11C06C05A
:105CB0000E94B5AE181614F446015701F981FF236E
:105CC00091F12A813B814C815D812115310541058E
:105CD000510541F0D701C601821B930BA40BB50BF4
:105CE000B7FD21C091014E815F816D857E858F85D5
:105CF00098890E94D8AB20E030E040EC5FE30E943E
:105D0000B2AC87FD2BCFD701C601805A9541AF4F6A
:105D1000BF4F8A839B83AC83BD832D863E869E8145
:105D20009F87AF81A88B80916F02882309F416CFDB
:105D300081149104A104B10431F41886CB88DC8865
:105D4000E12EF02EDCCEB8EECB1AB3E0DB0AE10890
:105D5000F108C818D908EA08FB08F7FCEECFFECE18
:105D60002F923F924F925F926F927F928F929F926B
:105D7000AF92BF92CF92DF92EF92FF920F931F9359
:105D8000CF93DF93CDB7DEB763970FB6F894DEBF3E
:105D90000FBECDBF898B81E080936F021A821B8278
:105DA0001C821D8219861A861B861C8621E0288784
:105DB00019821D863CE33E874CE14F8756E4588BA1
:105DC000C12CD12C80E8E82E9FEBF92E812C912C50
:105DD00054016091B2047091B304072E000C880B3B
:105DE000990B0E9454AD6A8B7B8B182F092F9B0156
:105DF000482F592FB601C7010E94B2AC882399F1F0
:105E00002091AE043091AF044091B0045091B104A0
:105E10006A897B89812F902F0E94B2AC881F8827C6
:105E2000881F89838989882311F199819923F9F041
:105E300080916F0263960FB6F894DEBF0FBECDBFA0
:105E4000DF91CF911F910F91FF90EF90DF90CF9056
:105E5000BF90AF909F908F907F906F905F904F908A
:105E60003F902F900895CA8ADB8A1E2D0F2D0E9425
:105E700068116B017C01DC01CB0129853A854B85DA
:105E80005C85821B930BA40BB50BB7FD34C0D70107
:105E9000C60188519C4FAF4FBF4F89879A87AB8708
:105EA000BC8780E034D88BE493E00E94E515811430
:105EB0009104A104B104C9F0D501C40188519C4FDB
:105EC000AF4FBF4FBC01CD016C197D098E099F09F1
:105ED00028EE33E040E050E00E94DDAFCA01B90196
:105EE0004AE050E00E94571903C08FE30E947518E2
:105EF0008AE00E9475180E9440AB0E94681160936E
:105F0000FF0B7093000C8093010C9093020C909106
:105F1000AE049E83A091AF04AF832090B004309074
:105F2000B104292F3A2FA1016A897B89812F902FF3
:105F30000E94D8AB2B013C0120E030E0A9010E9477
:105F4000B5AE87FF04C0C301B201905802C0C301BF
:105F5000B20120E030E040EA50E481149104A10451
:105F6000B10481F40E94B2AC87FF12C0B88546012B
:105F70005701BB2369F0E8EE8E0EE3E09E1EA11CE4
:105F8000B11C06C00E94B5AE181614F446015701A4
:105F9000F981FF2391F12A813B814C815D8121159B
:105FA00031054105510541F0D701C601821B930B14
:105FB000A40BB50BB7FD21C02E813F81A1016D85DA
:105FC0007E858F8598890E94D8AB20E030E040EC38
:105FD0005FE30E94B2AC87FD2BCFD701C601805A88
:105FE0009541AF4FBF4F8A839B83AC83BD839E8116
:105FF0009D87AF81AE872F86388A80916F02882374
:1060000009F416CF81149104A104B10431F4188667
:10601000CA88DB88E12EF02EDCCEB8EECB1AB3E0D6
:10602000DB0AE108F108C818D908EA08FB08F7FC00
:10603000EECFFECEEBE9F4E01082118212821382E1
:1060400014820895CF93C82F6115710519F0CB0103
:106050000E94E51589E597E00E94E515C11103C08E
:106060008AE497E002C08FE497E00E94E5158AE099
:10607000CF910C9475188091E7048093E8040895FB
:106080008091E604882319F01092E604089585EBC8
:1060900097E00C944CAA8091E804811105C080918E
:1060A000E204811101C0089562E070E080E090E0B8
:1060B0000E94A3158091E304882339F061E070E029
:1060C00080E090E00E94A315F5CF08958093E80446
:1060D0008093E704E0CF26982E9A25982D9A24984D
:1060E0002C9A3F98479A0A98129A0998119A81E037
:1060F000EDCF8093E804CFCF8093E204CCCF8091A2
:10610000E604882339F19091E6048091E104981720
:1061100009F10E94F31586EA97E00E94E515809147
:10612000E60480FD1CC08091E60484FD18C08091C7
:10613000E60481FD1EC08091E60485FD1AC08091B1
:10614000E60482FD20C08091E60486FD1CC08AE042
:106150000E9475188091E6048093E104089580E020
:106160000E94A85AAB01BC0182EA97E00E94301657
:10617000DECF81E00E94A85AAB01BC018EE997E016
:106180000E943016DCCF82E00E94A85AAB01BC010D
:106190008AE997E00E943016DACFCF9380E897E043
:1061A0000E94E51583B1C1E086FB882780F96AE784
:1061B00077E08C2747DF86B164E777E0881F882780
:1061C000881F40DF83B185FB882780F96EE677E082
:1061D0008C2738DF80B182FB882780F968E677E07A
:1061E0008C2730DF83B18295817062E677E08C275F
:1061F00029DF80B1869581706CE577E08C27CF919F
:1062000021CF8091E5041E9904C081608093E5044C
:1062100003C08E7F8093E5048091E504379B4DC0D9
:1062200080618093E5048091E5041D9904C082603B
:106230008093E50403C08D7F8093E5048091E5049D
:10624000029904C080628093E50403C08F7D80932F
:10625000E5048091E5041C9904C084608093E50402
:1062600003C08B7F8093E5048091E504019904C00D
:1062700080648093E50403C08F7B8093E504909154
:10628000E0048091E504981731F092E09093E304E4
:106290008093E00409C08091E304882329F08150B1
:1062A0008093E304882369F08091E80481110CC095
:1062B0008091E204811108C008958F7E8093E504E7
:1062C000B2CF9093E404F0CF8091570580FF1BC0BC
:1062D000909158058091E40490FF0BC080FF13C09B
:1062E0008091E60481608093E60480E00E94A65AD3
:1062F0000AC084FF08C08091E60480618093E604B0
:1063000080E00E94A65A8091570581FF1BC09091A2
:1063100058058091E40491FF0BC081FF13C0809168
:10632000E60482608093E60481E00E94A65A0AC0D7
:1063300085FF08C08091E60480628093E60481E0D6
:106340000E94A65A8091570582FF20C0809158056F
:1063500082FF10C08091E2048823C1F08091E404A0
:1063600082FF14C08091E60484608093E60482E09A
:106370000C94A65A8091E40486FF08C08091E6043C
:1063800080648093E60482E00C94A65A089539CF85
:10639000CF938823A1F0C82F0E94F31584E50E94B3
:1063A00075186AE070E08C2F90E00E94681980E216
:1063B0000E94751883EC97E0CF910C94E515CF916E
:1063C000089508958091940690919106891B8F708D
:1063D00019F480E090E0089590918E06992351F091
:1063E000833030F48FEF890F19F080938E06F1CF50
:1063F00010928E06E091910686E5E89FF001112447
:10640000EB56F94F808180FDE4CF809191068F5F3C
:106410008F708093930690919106809192069813C5
:1064200006C08091930680939206CF010895CF0114
:106430000895EFE6F0E08081826080830895809186
:10644000580580FF09C080910B018270809309017B
:106450008FEF8093E90409C080910B0180958270D1
:106460008093090181E08093E9048091580581FFC0
:106470000AC080910B0180958170809309018FEF94
:106480008093EA0408C080910B0181708093090118
:1064900081E08093EA048091580582FF09C08091D1
:1064A0000B018470809309018FEF8093EB0409C086
:1064B00080910B01809584708093090181E0809325
:1064C000EB0400000000000008950F930FB70F9336
:1064D00000916E000F930B7F00936E0000916F0090
:1064E0000D7F00936F000F930BB70F930CB70F92B4
:1064F0001F922F933F934F935F936F937F938F934D
:106500009F93AF93BF93EF93FF9311240E94453B5A
:10651000FF91EF91BF91AF919F918F917F916F917B
:106520005F914F913F912F911F900F900CBF0F9152
:106530000BBF0F910260F89400936F000F910093CE
:106540006E000F910FBF0F911895CF92DF92EF92CF
:10655000FF920F931F93809156058823D1F01092DC
:1065600056058091590590915A05892B91F010920A
:10657000570510925A0510925905909194068091F2
:106580009106981731F0809191068F5F8F708093FC
:1065900091068091590590915A05892B09F4AAC159
:1065A0004091250550912605609127057091280599
:1065B00090914D050091190510911A0520911B0528
:1065C00030911C05041B150B260B370B892F90E00F
:1065D000A0E0B0E0081719072A073B0710F4D9011B
:1065E000C801E82F840F951FA61FB71F80932505AC
:1065F00090932605A0932705B09328052091840049
:1066000030918500225E3F4F40913D0550913E05FF
:1066100060913F057091400580912D0590912E0568
:10662000A0912F05B0913005840F951FA61FB71FAD
:1066300080933D0590933E05A0933F05B0934005A0
:10664000B7FD1CC0409A4091ED045091EE0460915A
:10665000EF047091F0048091E904082E000C990B6E
:10666000AA0BBB0B840F951FA61FB71F8093ED04C9
:106670009093EE04A093EF04B093F0044091410591
:106680005091420560914305709144058091310518
:1066900090913205A0913305B0913405840F951F78
:1066A000A61FB71F8093410590934205A093430511
:1066B000B0934405B7FD1CC0419A4091F10450913C
:1066C000F2046091F3047091F4048091EA04082EBE
:1066D000000C990BAA0BBB0B840F951FA61FB71FAD
:1066E0008093F1049093F204A093F304B093F40424
:1066F00040914505509146056091470570914805C8
:106700008091350590913605A0913705B0913805F7
:10671000840F951FA61FB71F8093450590934605CC
:10672000A0934705B0934805B7FD1CC0429A40911D
:10673000F5045091F6046091F7047091F80480918B
:10674000EB04082E000C990BAA0BBB0B840F951FB2
:10675000A61FB71F8093F5049093F604A093F70447
:10676000B093F8044091490550914A0560914B055A
:1067700070914C058091390590913A05A0913B05A7
:10678000B0913C05840F951FA61FB71F8093490544
:1067900090934A05A0934B05B0934C05B7FD3CC0C0
:1067A000C090F904D090FA04E090FB04F090FC044F
:1067B0004091EC04042E000C550B660B770B4C0D2E
:1067C0005D1D6E1D7F1D4093F9045093FA04609384
:1067D000FB047093FC044091290550912A056091B7
:1067E0002B0570912C05841B950BA60BB70B809382
:1067F000490590934A05A0934B05B0934C059091A1
:10680000580580910E0593FF04C0815080930E05BA
:1068100003C08F5F80930E05809184009091850066
:1068200082179307C8F380913D0590913E05A09192
:106830003F05B0914005B7FD15C040912905509125
:106840002A0560912B0570912C05841B950BA60BD6
:10685000B70B80933D0590933E05A0933F05B09301
:10686000400540988091410590914205A0914305D3
:10687000B0914405B7FD15C04091290550912A05F6
:1068800060912B0570912C05841B950BA60BB70B03
:106890008093410590934205A0934305B09344052E
:1068A00041988091450590914605A0914705B0918A
:1068B0004805B7FD15C04091290550912A05609102
:1068C0002B0570912C05841B950BA60BB70B8093A1
:1068D000450590934605A0934705B0934805429817
:1068E000E15041F0809184009091850082179307D8
:1068F000C8F388CE1F910F91FF90EF90DF90CF905B
:106900000895CF92DF92EF92FF9280910D05882338
:1069100009F465C0C0902505D0902605E0902705B4
:10692000F090280540911D0550911E0560911F05AE
:106930007091200580910E054C155D056E057F0553
:10694000E8F42091130530911405E0911105F091C0
:106950001205E217F30790F4815080930E05215041
:10696000310930931405209313054091250250916D
:106970002602609127027091280234C0C416D50601
:10698000E606F706E8F420911305309114054091CE
:106990000F05509110052417350790F48F5F8093F1
:1069A0000E052F5F3F4F3093140520931305409140
:1069B000250250912602609127027091280212C090
:1069C0008FEF9FEFDC018093250290932602A09326
:1069D0002702B09328024FEF5FEFBA0103C04FEFD9
:1069E0005FEFBA0180910E0587FD06C080910B0113
:1069F00080748093090106C080910B01809580749A
:106A0000809309012091840030918500225E3F4FE0
:106A100080910E05882311F1439A80918400909112
:106A2000850082179307C8F380910E0587FF04C085
:106A30008F5F80930E0503C0815080930E054398AD
:106A400080910E05882321F3809184009091850028
:106A500082179307C8F3225E3F4FDACFCB01BA010A
:106A6000FF90EF90DF90CF900895BC0120915905E1
:106A700030915A054091590550915A052417350710
:106A800011F09A01F7CF81E06217730709F080E0F7
:106A90000895CF93DF93EC0188819981AA81BB810E
:106AA000EDEEF4E080839183A283B383EB018881D0
:106AB0009981AA81BB8184839583A683B783EA01E8
:106AC00088819981AA81BB8180879187A287B387BA
:106AD000E90188819981AA81BB8184879587A687EE
:106AE000B787DF91CF9108953F924F925F926F9257
:106AF0007F928F929F92AF92BF92CF92DF92EF924E
:106B0000FF920F931F93CF93DF93CDB7DEB72897F4
:106B10000FB6F894DEBF0FBECDBFA0915905B0915E
:106B20005A05109739F18090250590902605A09080
:106B30002705B09028054091190550911A056091DC
:106B40001B0570911C0584169506A606B706C8F0AD
:106B50001092570510925A0510925905909194067B
:106B600080919106981731F0809191068F5F8F7018
:106B70008093910670EDC72E77E0D72EE12CF12C93
:106B800097C1409121055091220560912305709194
:106B90002405481559056A057B0508F46EC0009167
:106BA0005205109153052091540530915505D19609
:106BB0004D915D916D917C91D497EE27059FF12DBC
:106BC000169FC001269F900D259F800D911D069F49
:106BD000F00D811D9E1F159FF00D811D9E1F249F8E
:106BE000F00D811D9E1F149FF10D8E1F9E1FF695A7
:106BF0008E1F9E1F709F800D911D719F900D1124FF
:106C0000FD01EB5BFF4F4081518162817381480F31
:106C1000591F611D711D4093090550930A0560932A
:106C20000B0570930C053497C080D180E280F3800F
:106C3000C416D506E606F70640F4C0920905D092C0
:106C40000A05E0920B05F0920C0540910905509160
:106C50000A0560910B0570910C0581E298E0BB2458
:106C6000B394FC01C590D590E590F490C416D50678
:106C7000E606F70608F475C27FC240901D055090E5
:106C80001E0560901F0570902005481459046A0481
:106C90007B0408F080C020914E0530914F05409153
:106CA0005005509151052D833E834F835887D196CF
:106CB0000D911D912D913C91D4974D815E816F81F5
:106CC0007885EE27419FF12D529FC001629F900D64
:106CD000619F800D911D429FF00D811D9E1F519F50
:106CE000F00D811D9E1F609FF00D811D9E1F509F06
:106CF000F10D8E1F9E1FF6958E1F9E1F349F800DD7
:106D0000911D359F900D11248C0120E030E0C09042
:106D10000905D0900A05E0900B05F0900C05CD0117
:106D2000875B9F4FFC010C151D052E053F05C0F428
:106D3000408151816281738149835A836B837C8353
:106D4000C01AD10AE20AF30AC416D506E606F70607
:106D500010F46A017B0181E298E03324339410C07F
:106D6000C080D180E280F380F6CFF694E794D79488
:106D7000C794330C049628E08D33920709F480C23F
:106D8000FC0105911591259134910C151D052E05D9
:106D90003F0558F375C280910E058823D9F0D79628
:106DA0004D915C91D89760E070E0009125021091C0
:106DB0002602209127023091280204171507260782
:106DC000370741F01092290210922A0210922B02EA
:106DD00010922C02409121025091220260912302D4
:106DE0007091240277FF5CC0AF5BBF4F8D919D9186
:106DF0000D90BC91A02D21E238E041E0F901C59051
:106E0000D590E590F490C816D906EA06FB0658F42A
:106E1000B695A79597958795440F2C5F3F4F58E0FF
:106E20002D33350759F740934D0580329105A10563
:106E3000B10520F480E290E0A0E0B0E08097A109E5
:106E4000B109811578E09707A105B10508F4CEC214
:106E500024E0929FF00111249F012F5B334FF90131
:106E6000329665917491EE27879FA001869F410D10
:106E70005E1F06944E1F5E1F112460E070E0F90152
:106E800085919491A0E0B0E0841B950BA60BB70B05
:106E90008093210290932202A0932302B0932402B4
:106EA000C0902102D0902202E0902302F0902402B0
:106EB0008091590590915A05892B09F01DC382DAFA
:106EC00090935A0580935905892B09F415C3E091D5
:106ED0005905F0915A05808183FF19C09F012F5DEC
:106EE0003F4FAF01435E5F4FBF01675E7F4FCF01F2
:106EF0004596CFDD90919406809191069817F9F20E
:106F0000809191068F5F8F7080939106D8CFC5884E
:106F1000D688E788F08C81E0C114D104E104F10443
:106F200009F480E0018D128D238D348D011511053A
:106F30002105310509F08260458D568D678D70A160
:106F4000411551056105710509F08460809357056D
:106F500010924E0510924F05109250051092510557
:106F60001092520510925305109254051092550537
:106F700085A196A1A7A1B0A58093190590931A05A4
:106F8000A0931B05B0931C05882499245401881AEA
:106F9000990AAA0ABB0A8092490590924A05A092D2
:106FA0004B05B0924C058092450590924605A09203
:106FB0004705B09248058092410590924205A09203
:106FC0004305B092440580923D0590923E05A09203
:106FD0003F05B0924005CC0CDD1CEE1CFF1CC0929E
:106FE0002D05D0922E05E0922F05F0923005000F6E
:106FF000111F221F331F0093310510933205209378
:10700000330530933405440F551F661F771F409397
:10701000350550933605609337057093380541A1C7
:1070200052A163A174A1440F551F661F771F40939F
:10703000390550933A0560933B0570933C05880FE2
:10704000991FAA1FBB1F8093290590932A05A0931F
:107050002B05B0932C051092250510922605109251
:1070600027051092280581A592A5A3A5B4A5809314
:10707000210590932205A0932305B093240585A5AF
:1070800096A5A7A5B0A980931D0590931E05A09372
:107090001F05B093200586A980930D05882309F16B
:1070A00083AD94AD909312058093110581AD92AD9F
:1070B0009093100580930F051092290210922A02D6
:1070C00010922B0210922C0287A990ADA0E0B0E0A4
:1070D0008093250290932602A0932702B093280262
:1070E0000BC08FEF9FEFDC01809325029093260267
:1070F000A0932702B093280285A99091580589177B
:1071000019F0809358059BD97CD88FEF9FEFDC0155
:107110008093210290932202A0932302B093240231
:10712000E0915905F0915A05EB5BFF4F8081918109
:10713000A281B3818093090590930A05A0930B0562
:10714000B0930C0521E238E041E0F901C590D590FB
:10715000E590F490C816D906EA06FB0608F46BC160
:1071600076C17695679557954795BB0C0496E8E0F0
:107170008D339E0709F075CDB0924D054032510513
:107180006105710520F440E250E060E070E040529B
:10719000510961097109411588E0580761057105B8
:1071A00000F194E0599FF0011124CF018F5B934FC0
:1071B000FC013296E590F490F701DD244F9F5001D9
:1071C0004E9FA10CBD1C0694AD1CBD1C1124FC01DE
:1071D000C590D490E12CF12CCA18DB08E108F10825
:1071E00024C06A017B01F694E794D794C794F60112
:1071F000EC7FCF018F5B974F7C01FC0185919491CF
:10720000F7013296E590F49047704E9DB0014F9D86
:10721000700D1124AB0163E0569547956A95E1F72F
:107220006C01C41AD50AE12CF12C0C0D1D1D2E1D6C
:107230003F1D00935205109353052093540530933E
:10724000550590910D0580910E05992309F465C0AF
:10725000882309F42DCED7968D919C91D897A0E0E4
:10726000B0E0409125025091260260912702709172
:107270002802481759076A077B0709F051C018CE42
:1072800030924D05F0E2CF16D104E104F10428F468
:1072900030E2C32ED12CE12CF12CF0E2CF1AD10830
:1072A000E108F108C11428E0D206E104F10408F471
:1072B00040C034E0D39EC00111248F5B934FFC018A
:1072C0003296059114916C2D3327619FA001609F28
:1072D000410D531F0694431F531F1124FC01C590F9
:1072E000D490E12CF12CC41AD50AE108F1084D81A3
:1072F0005E816F8178854C0D5D1D6E1D7F1D4093F5
:107300004E0550934F056093500570935105809141
:107310000D05811132C080910E05882309F4C8CD76
:107320001092290210922A0210922B0210922C0223
:10733000BFCD970186013695279517950795F801DA
:10734000EC7FCF018F5B974FFC0105911491FC01FD
:107350003296459154913C2D3770349FC001359F32
:10736000900D112423E0969587952A95E1F7680101
:10737000C81AD90AE12CF12CBACF430C511C611C5C
:10738000711C481459046A047B04C8F480910E05EA
:10739000882309F48DCDD7964D915C91D89760E004
:1073A00070E0009125021091260220912702309171
:1073B0002802041715072607370709F479CD10921C
:1073C000290210922A0210922B0210922C02D796B8
:1073D0008D919C91D897A0E0B0E080932502909386
:1073E0002602A0932702B093280262CDAC01BD0112
:1073F0007695679557954795FA01EC7FAF014F5BFE
:10740000574FFA0125913491FA01329665917491A2
:107410008770869FA001879F500D1124CA01F3E059
:1074200096958795FA95E1F7A901481B590BCA0172
:10743000A0E0B0E02DCDB695A79597958795440F20
:107440002C5F3F4F68E02D33360709F07ECE409326
:107450004D0580329105A105B10520F480E290E050
:10746000A0E0B0E08097A109B109811558E0950727
:10747000A105B105F8F064E0969FF00111249F0189
:107480002F5B334FF901329665917491EE27879FF8
:10749000A001869F410D5E1F06944E1F5E1F1124A2
:1074A000F901C590D490E12CF12CC41AD50AE10859
:1074B000F10822C0AC01BD017695679557954795B7
:1074C000FA01EC7FAF014F5B574FFA01C590D490A2
:1074D000FA013296459154918770849F9001859F5F
:1074E000300D1124C901A3E096958795AA95E1F77F
:1074F000C81AD90AE12CF12CC701B60128960FB69B
:10750000F894DEBF0FBECDBFDF91CF911F910F91D9
:10751000FF90EF90DF90CF90BF90AF909F908F90B3
:107520007F906F905F904F903F900895CF92DF9241
:10753000EF92FF921F93CF93DF938FEF9FEF909384
:107540008900809388001AE0C0E0D0E078948091B0
:10755000150590911605A0911705B0911805892B76
:107560008A2B8B2B11F40E94A532809129029091D5
:107570002A02A0912B02B0912C02892B8A2B8B2BF3
:1075800049F4BFD96093290270932A0280932B0299
:1075900090932C028091150590911605A0911705E6
:1075A000B0911805892B8A2B8B2B49F49DDA6093B7
:1075B0001505709316058093170590931805C090D4
:1075C0001505D0901605E0901705F090180540912C
:1075D000290250912A0260912B0270912C02FC2DFD
:1075E000ED2D3E2D2F2D4C155D056E057F0520F4EC
:1075F000F42FE52F362F272F8F2F9E2FA32FB22F5B
:10760000009721E0A207B10520F08FEF9FEFA0E0E7
:10761000B0E0C81AD90AEA0AFB0AC0921505D0924E
:107620001605E0921705F09218054F3F2FEF52070D
:107630006207720761F0481B590B6A0B7B0B409382
:10764000290250932A0260932B0270932C02F89423
:107650002091840030918500205F3F4F115039F018
:10766000C80FD91FC217D30708F470CF01C0E901B2
:10767000D0938900C09388007894DF91CF911F91B7
:10768000FF90EF90DF90CF90089550CF90916F00D2
:1076900091FB222720F991FF05C090916F009D7FFB
:1076A00090936F0094E0899FF0011124E351FB4F08
:1076B0006081718182819381222329F020916F0062
:1076C000226020936F00089590916F0091FB222714
:1076D00020F991FF05C090916F009D7F90936F00FE
:1076E00034E0839FC0011124FC01E351FB4F408132
:1076F000518162817381FC01E350FB4F40835183D0
:107700006283738381E080935605222329F0809160
:107710006F00826080936F00089590916F0091FBDD
:10772000222720F991FF05C090916F009D7F9093D3
:107730006F0094E0899FF0011124E350FB4F6081BA
:10774000718182819381222329F020916F00226030
:1077500020936F0008954F925F926F927F928F9265
:107760009F92AF92BF92CF92DF92EF92FF92809161
:107770006F0081FB992790F981FF05C080916F0010
:107780008D7F80936F004090ED045090EE046090E8
:10779000EF047090F0048090F1049090F204A090B7
:1077A000F304B090F404C090F504D090F604E09097
:1077B000F704F090F804992329F080916F0082601B
:1077C00080936F0087E198E00E94E5154AE050E061
:1077D000C301B2010E94571983E198E00E94E515A8
:1077E0004AE050E0C501B4010E9457198FE098E0CB
:1077F0000E94E5154AE050E0C701B6010E94571902
:107800008AE0FF90EF90DF90CF90BF90AF909F9075
:107810008F907F906F905F904F900C947518DB0164
:1078200090916705992309F440C0833070F494E087
:10783000899FF0011124E55AFA4FAB01770F660BCF
:10784000770B4083518362837383813091F018F00A
:107850008230E9F008952FEF30E00E9432B020ED41
:1078600037E040E050E00E94FFAFB9018EE20C9497
:1078700034122FEF30E00E9432B020ED37E040E0CC
:1078800050E00E94FFAFB9018DE20C9434122FEF4B
:1078900030E00E9432B020ED37E040E050E00E943E
:1078A000FFAFB9018CE20C94341208958091670502
:1078B000882391F060915B0570915C0580E0AFDFFB
:1078C00060915F057091600581E0A9DF60916305BB
:1078D0007091640582E0A3CF0895EAE0F1E0808131
:1078E00088608083808180618083808180628083E2
:1078F000DDDFE1E2F1E08081887F816080830895AF
:1079000067FD2CC0813061F028F0823099F083301F
:10791000D9F024C0662311F0A19A2AC0A19828C0EA
:10792000809108016111809580788093060147FF5E
:1079300027C008958091080161118095807480931B
:10794000060147FF23C008958091080161118095C9
:1079500088708093060147FF21C0089547FD26C027
:10796000813071F038F0823089F08330B9F00895B9
:1079700047FD1CC0442311F0A09A0895A0980895D3
:10798000442311F0A29A0895A298089580910801C5
:1079900041118095807280930601089580910801BD
:1079A0004111809580718093060108950895643097
:1079B00091F040F4613059F06230A9F420E040E0E9
:1079C00061E09ECF683059F0603149F00CC020E092
:1079D00040E060E095CF20E041E060E091CF20E022
:1079E00041E061E08DCF0E94F61587EF97E00C949F
:1079F000E5150F931F93CF93999A989A8091070159
:107A00008068809307019A9A80910701806480932F
:107A1000070180910701806280930701809107012F
:107A2000886080930701809107018061809307013E
:107A300001E313E0C0E0F80161918F018C2FB7DF03
:107A4000CF5FC630C1F7CF911F910F910895D1DF5D
:107A5000EAE0F1E0808182608083808181608083C0
:107A60008081846080838081806480830F9A179AEC
:107A70000E9A169A0D9A159A0C9A149A389A40985A
:107A8000179A809191058E7F80939105399A41983C
:107A9000169A809191058D7F809391053A9A42982C
:107AA000159A809191058B7F809391053B9A43981D
:107AB000149AA0E8B0E08C918C7F8C93E1E8F0E020
:107AC0008081877E886080838C918F738C93808186
:107AD000887F8260808380E090E490938900809327
:107AE00088001092850010928400EFE6F0E080811B
:107AF00082608083789482E0809358050E941F32D0
:107B000081E080936705E9CE82EE97E00E94E5155B
:107B1000919902C080E301C081E30E947518909999
:107B200002C080E301C081E30E9475188EED97E0EA
:107B30000E94E51580910601881F8827881F805DB7
:107B40000E947518929902C080E301C081E30E94EF
:107B500075188AED97E00E94E5158091060186FD73
:107B600002C080E301C081E30E9475188091060184
:107B700085FD02C080E301C081E30E94751885ED98
:107B800097E00E94E5158091060183FD02C080E325
:107B900001C081E30E9475188091060184FD02C036
:107BA00080E301C081E30C947518CF93DF93CDB7C8
:107BB000DEB760970FB6F894DEBF0FBECDBF8091E1
:107BC000500290915102A0915202B09153028983C8
:107BD0009A83AB83BC838091540290915502A0910B
:107BE0005602B09157028D839E83AF83B8878091F0
:107BF000580290915902A0915A02B0915B02898774
:107C00009A87AB87BC8780915C0290915D02A091BE
:107C10005E02B0915F028D879E87AF87B88B0E940E
:107C20005C6B6091640270916502072E000C880BFA
:107C3000990B0E9454AD2AE037ED43E25CE30E94C9
:107C4000F0AE609360027093610280936202909341
:107C5000630280E00E94D15081E00E94D15082E016
:107C60000E94D15023DE0E94A36B40E150E060E50A
:107C700072E0CE0101960E946AB4892B51F06096A1
:107C80000FB6F894DEBF0FBECDBFDF91CF910C943D
:107C9000994E60960FB6F894DEBF0FBECDBFDF9150
:107CA000CF9108958734924041F00E94F61586E8FE
:107CB00093E10E94E51581E0089580E00895EF9238
:107CC000FF920F931F93CF93DF93CDB7DEB7C458C6
:107CD000D1090FB6F894DEBF0FBECDBFED961CAE36
:107CE0001DAE1EAE1FAEED9785E492E5A2E5B0E0B5
:107CF000E9968CAF9DAFAEAFBFAFE997CF57DF4FDF
:107D000019821882C158D04084E690E0C158DF4FF4
:107D100099838883CF57D0400E94921610926905AC
:107D20009E012F573F4F44E050E0BE016B587F4FFC
:107D3000CE0181589F4F0E949616C158DF4F88810F
:107D40009981CF57D0400296C158DF4F99838883DD
:107D5000CF57D040CF57DF4F19821882C158D0403B
:107D600081E0CC57DF4F8883C458D0409E012F5705
:107D70003F4F41E050E0BE016C577F4FCE0181582C
:107D80009F4F0E9496169E012F573F4F48E450E0A8
:107D900066E476E0CE0181589F4F0E9496169E01C0
:107DA0002F573F4F40E150E066E176E0CE01815829
:107DB0009F4F0E9496168AE097EDA3EABCE3ED96EA
:107DC0008CAF9DAFAEAFBFAFED979E012F573F4F2A
:107DD00044E050E0BE0167587F4FCE0181589F4F6D
:107DE0000E9496168E010F5F1F4F8CE0F8011192D2
:107DF0008A95E9F79E012F573F4F4CE050E0B801BC
:107E0000CE0181589F4F0E94961680E090E0A0E23C
:107E1000B1E489839A83AB83BC839E012F573F4F84
:107E200044E050E0B801CE0181589F4F0E94961661
:107E3000ED961CAE1DAE1EAE1FAEED9783E0AE9666
:107E40008FAFAE9789839E012F573F4F44E050E09C
:107E5000BE0167587F4FCE0181589F4F0E949616F2
:107E60009E012F573F4F41E050E0BE0163597F4FC5
:107E7000CE0181589F4F0E9496169E012F573F4F6B
:107E800041E050E0B801CE0181589F4F0E94961604
:107E90002AE0F22EFA949E012F573F4F44E050E023
:107EA000FF2049F0BE0167587F4FCE0181589F4F98
:107EB0000E949616EFCF6AE675E0CE0181589F4F7B
:107EC0000E9496169E012F573F4F44E250E061EF0B
:107ED00075E0CE0181589F4F0E94961683E0CD57E2
:107EE000DF4F8883C358D040EE968FAFEE97E19670
:107EF0001CAE1DAE1EAE1FAEE19719821A821B8208
:107F00001C82ED961CAE1DAE1EAE1FAEED979E01FF
:107F10002F573F4F41E050E0BE016D577F4FCE01DC
:107F200081589F4F0E9496169E012F573F4F41E068
:107F300050E0BE0163587F4FCE0181589F4F0E9491
:107F400096169E012F573F4F44E050E0B801CE01F6
:107F500081589F4F0E9496169E012F573F4F44E035
:107F600050E0BE0163597F4FCE0181589F4F0E9460
:107F700096169AE0E92EF12CF1E0EF1AF10871F073
:107F80009E012F573F4F44E050E0BE0167587F4F9E
:107F9000CE0181589F4F0E949616EECFAE961FAE2F
:107FA000AE978FEF89839E012F573F4F41E050E0FE
:107FB000BE0163597F4FCE0181589F4F0E94961694
:107FC0009E012F573F4F41E050E0B801CE0181584C
:107FD0009F4F0E94961680E1F82EF8018F2D119286
:107FE0008A95E9F79E012F573F4F40E150E0B801D5
:107FF000CE0181589F4F0E94961688EC90E0AF9674
:108000009FAF8EAFAF9780EF90E0E1969FAF8EAFBE
:10801000E19786E490E09A8389838EE690E09C83E2
:108020008B83EE961FAEEE97EF961FAEEF979E01F5
:108030002F573F4F44E050E0BE0163597F4FCE01C0
:1080400081589F4F0E9496169E012F573F4F44E044
:1080500050E0B801CE0181589F4F0E9496169E01B4
:108060002F573F4F42E050E0BE0163587F4FCE0193
:1080700081589F4F0E949616F8011192FA94E9F7E1
:1080800080E090E0A0E8BFE38D879E87AF87B88B44
:108090008091D3049091D404A091D504B091D604DA
:1080A00089839A83AB83BC838091D7049091D80451
:1080B000A091D904B091DA048D839E83AF83B887F1
:1080C0008091DB049091DC04A091DD04B091DE048A
:1080D00089879A87AB87BC879E012F573F4F40E126
:1080E00050E0B801CE0181589F4F0E94961684E15E
:1080F00090E09A8389839E012F573F4F42E050E0E2
:10810000B801CE0181589F4F0E9496169E012F57AD
:108110003F4F4CE050E065EB74E0CE0181589F4F3B
:108120000E94961680E290E09A8389839E012F57E1
:108130003F4F42E050E0B801CE0181589F4F0E946E
:10814000961681E089839E012F573F4F41E050E012
:10815000B801CE0181589F4F0E94961680E2E1E857
:10816000F2E0D80101900D928A95E1F79E012F5718
:108170003F4F40E250E0B801CE0181589F4F0E942E
:108180009616AE961FAEAE979E012F573F4F41E019
:1081900050E0BE0163597F4FCE0181589F4F0E942E
:1081A0009616198280E090E0A0E4B0E4ED968CAFE2
:1081B0009DAFAEAFBFAFED979E012F573F4F41E050
:1081C00050E0B801CE0181589F4F0E9496169E0143
:1081D0002F573F4F44E050E0BE0167587F4FCE011C
:1081E00081589F4F0E9496168AE1F80111928A9554
:1081F000E9F79E012F573F4F4AE150E0B801CE0109
:1082000081589F4F0E94961684E3E1EAF2E0D8017C
:1082100001900D928A95E1F79E012F573F4F44E35D
:1082200050E0B801CE0181589F4F0E9496161A82E5
:1082300019821C821B821E821D829E012F573F4F76
:1082400046E050E0B801CE0181589F4F0E9496163B
:108250008DE0F80111928A95E9F79E012F573F4F63
:108260004DE050E0B801CE0181589F4F0E94961614
:108270009E012F573F4F44E050E068EB75E0CE0180
:1082800081589F4F0E9496169E012F573F4F4CE0FA
:1082900050E06BE575E0CE0181589F4F0E94961625
:1082A0008CE6F80111928A95E9F79E012F573F4F0E
:1082B0004CE650E0B801CE0181589F4F0E949616BF
:1082C0009E012F573F4F4CE050E065EE75E0CE0128
:1082D00081589F4F0E949616E1961CAE1DAE1EAEB1
:1082E0001FAEE197E5961CAE1DAE1EAE1FAEE59724
:1082F0009E012F573F4F48E050E0BE0163597F4F2A
:10830000CE0181589F4F0E94961680916905811178
:108310004FC0C158DF4F08811981CF57D040045654
:108320001109CF57DF4F88819981C158D040AF964E
:108330009FAF8EAFAF9784E690E0C158DF4F99832F
:108340008883CF57D0409E012F573F4F44E050E0E5
:1083500067E373E0CE0181589F4F0E9496169E01FD
:108360002F573F4F42E050E0BE0163597F4FCE018F
:1083700081589F4F0E9496160E94F315B80184E71A
:1083800093E10E945016AF964EAD5FADAF9760E09F
:1083900070E087E693E10E945A1684E693E10E941A
:1083A000E515C8017FDC90916905892B80936905EB
:1083B0000E9494169091690581E08927CC57DF4F80
:1083C0000FB6F894DEBF0FBECDBFDF91CF911F91E6
:1083D0000F91FF90EF9008951F93CF93DF93CDB748
:1083E000DEB72C970FB6F894DEBF0FBECDBFA6E464
:1083F000B6E020E030E0C9012430310510F083E020
:1084000090E0880F991F880F991FFC01ED54FD4ED5
:10841000459155916591749154964D935D936D93EB
:108420007C935797FC01ED55FD4E45915591659113
:10843000749194964D935D936D937C939797FC0103
:10844000ED56FD4E45915591659174914D935D9317
:108450006D937D932F5F3F4F2430310509F0CBCFD3
:1084600080E29EE4A0E0B0E0809356069093570629
:10847000A0935806B093590680E090E0AAEFB4E4C8
:1084800080937A0690937B06A0937C06B0937D063A
:1084900040E050E86BE375E440937E0650937F061E
:1084A0006093800670938106809382069093830682
:1084B000A0938406B09385061092860610928706D4
:1084C000109288061092890610928A0610928B06E6
:1084D00010928C0610928D0680E090E0A0E4B1E44A
:1084E0008093160690931706A0931806B09319066A
:1084F00080931A0690931B06A0931C06B0931D064A
:108500008DEC9CECACECBEE380931E0690931F06B2
:10851000A0932006B093210680E090E0A0E2B1E4B1
:108520008093220690932306A0932406B0932506F9
:108530000E94881A80E090E0A0EBBFEB80936A0570
:1085400090936B05A0936C05B0936D0583E393E363
:10855000A6E1B2E48093D3049093D404A093D5040D
:10856000B093D6048EEA92E1A2E6BFE38093D704EB
:108570009093D804A093D904B093DA0480E896E7E6
:10858000A7ECB3E48093DB049093DC04A093DD04B8
:10859000B093DE0480E090E0A3E9B3E48093B504F7
:1085A0009093B604A093B704B093B80483EC94E618
:1085B000AAE2B1E48093B9049093BA04A093BB04F7
:1085C000B093BC0480EB98EBA1E1B5E48093BD04CB
:1085D0009093BE04A093BF04B093C00481E00E94B6
:1085E00066300E94E1311092B8051092B9051092E0
:1085F000BA051092BB058CE0E5EDF2E0DE011196C4
:1086000001900D928A95E1F713E01150C0F084E0DB
:10861000189F90011124E1E0F0E0EC0FFD1FE20F44
:10862000F31F6081718182819381F901E55AFA4FCC
:108630006083718382839383812FF1D8E6CFB5DA8B
:108640000E94F31580E792E12C960FB6F894DEBFF6
:108650000FBECDBFDF91CF911F910C94E515CF9345
:10866000C82F811102C00E94F31589E592E10E9492
:10867000E51584E490E10E94E5158AE00E947518F2
:108680008AE00E947518C11106C00E94F31588E4A3
:1086900092E10E94E5156FEF81E08C270E94F29332
:1086A000C11108C00E94F3158AE292E10E94E5150B
:1086B0000E94F31540916A0650916B0660916C061A
:1086C00070916D0681E292E10E94301640916E0633
:1086D00050916F0660917006709171068EE192E183
:1086E0000E94301640917206509173066091740694
:1086F000709175068BE192E10E94301640917606EA
:1087000050917706609178067091790688E192E140
:108710000E9430168AE00E947518C11108C00E949C
:10872000F31586EF91E10E94E5150E94F315609123
:1087300046067091470680914806909149060E942E
:1087400052ADAB01BC018DEE91E10E9430166091FB
:108750004A0670914B0680914C0690914D060E94FE
:1087600052ADAB01BC018AEE91E10E9430166091DE
:108770004E0670914F0680915006909151060E94CE
:1087800052ADAB01BC0187EE91E10E9430166091C1
:1087900052067091530680915406909155060E949E
:1087A00052ADAB01BC0184EE91E10E9430168AE02B
:1087B0000E947518C11108C00E94F3158AE991E161
:1087C0000E94E5150E94F31540917A0650917B06B0
:1087D00060917C0670917D0681E991E10E943016DE
:1087E00040917E0650917F066091800670918106CF
:1087F0008EE891E10E9430164091820650918306E6
:1088000060918406709185068BE891E10E94301694
:108810008AE00E947518C11113C00E94F31583E409
:1088200091E10E94E51588E191E10E94E51589E05A
:1088300091E10E94E5158AE00E9475180E94F315E7
:10884000609156067091570680915806909159068E
:108850000E9452ADAB01BC0180E091E10E94301654
:10886000409186065091870660918806709189062E
:108870008DEF90E10E94301640918A0650918B0650
:1088800060918C0670918D068AEF90E10E943016FF
:1088900040911606509117066091180670911906BE
:1088A00087EF90E10E94301640911A0650911B0606
:1088B00060911C0670911D0684EF90E10E943016B5
:1088C00040911E0650911F0660912006709121066E
:1088D00081EF90E10E9430164091220650912306CC
:1088E00060912406709125068EEE90E10E9430166C
:1088F0008AE00E947518C11108C00E94F3158AED24
:1089000090E10E94E5150E94F3156091150670E054
:1089100081ED90E10E9416168AE00E947518C1113F
:1089200008C00E94F31582EC90E10E94E5150E94B8
:10893000F3154091D3045091D4046091D504709103
:10894000D60489EB90E10E9430162CEA35EC47E220
:108950005EE36091D7047091D8048091D90490911E
:10896000DA040E94B9ACAB01BC0186EB90E10E9435
:1089700040162CEA35EC47E25EE36091DB0470912F
:10898000DC048091DD049091DE040E94F0AEAB0126
:10899000BC0183EB90E10E9440168AE00E947518AA
:1089A000C11102C00E94F3154091B5045091B60464
:1089B0006091B7047091B8048AEA90E10E94301681
:1089C0002CEA35EC47E25EE36091B9047091BA0499
:1089D0008091BB049091BC040E94B9ACAB01BC0176
:1089E00087EA90E10E9440162CEA35EC47E25EE30C
:1089F0006091BD047091BE048091BF049091C00449
:108A00000E94F0AEAB01BC0184EA90E10E944016E6
:108A10008AE00E947518C11110C00E94F31585E903
:108A200090E10E94E51584E490E10E94E51581E45F
:108A300090E10E94E5150E94F31540916A0550915E
:108A40006B0560916C0570916D058CE890E10E945A
:108A500030168AE00E947518C11108C00E94F315F3
:108A60008BE790E10E94E5150E94F3154091B8054F
:108A70005091B9056091BA057091BB0582E790E10C
:108A80000E9430168AE00E947518C11108C00E9429
:108A9000F31589E590E10E94E5150E94F3154091D8
:108AA0005B0550915C0560915D0570915E0580E508
:108AB00090E10E945A1640915F05509160056091C7
:108AC0006105709162058DE490E10E945A16409113
:108AD00063055091640560916505709166058AE4AF
:108AE00090E10E945A168AE0CF910C9475182F924B
:108AF0003F924F925F926F927F928F929F92AF922E
:108B0000BF92CF92DF92EF92FF920F931F93CF937A
:108B1000DF93CDB7DEB7C45AD1090FB6F894DEBFE4
:108B20000FBECDBF2DB73EB7CD55DF4F398328835C
:108B3000C35AD040C756DF4F19821882C959D04056
:108B400084E690E0C956DF4F99838883C759D040A7
:108B50000E94921601E09E0127563F4F44E050E0EC
:108B6000BE016F567F4FCE0189569F4F0E94EB1674
:108B70009E0127563F4F42E050E0BE016B567F4FAB
:108B8000CE0189569F4F0E94EB1643E050E0BE0194
:108B90006F567F4F87E393E00E9489B4892B19F1C8
:108BA000CC56DF4F8881C459D040882359F08FE3D9
:108BB000CF56DF4F8883C159D040CE56DF4F188241
:108BC000C259D0400E94F315BE016F567F4F83E417
:108BD00093E10E94F91585E393E10E94E51581E098
:108BE0008093690524C5C357DF4F188219821A8202
:108BF0001B82CD58D040C756DF4F19821882C95901
:108C0000D04001E09E0127563F4F41E050E0BE01B9
:108C100064567F4FCE0189569F4F0E94EB168DB749
:108C20009EB7C156DF4F99838883CF59D0406E01DC
:108C30009DE7C90ED11C80E1E1EEF2E0D601019082
:108C40000D928A95E1F77E01EDE6EE0EF11C80E1D2
:108C5000E1EFF2E0D70101900D928A95E1F780E112
:108C6000E1E0F3E09E012F5F3F4F5901D9010190F0
:108C70000D928A95E1F7C456DF4F4881CC59D04018
:108C800050E04D5F5F4F440F551F440F551F8DB788
:108C90009EB7841B950B0FB6F8949EBF0FBE8DBF79
:108CA000EDB7FEB731961F010091680511E001276D
:108CB00028563F4FBF01CE0189569F4F0E94EB16A9
:108CC0000091680501279E0127563F4F44E050E080
:108CD00066E576E0CE0189569F4F0E94EB16C4569A
:108CE000DF4F8880CC59D040912CF3E08F0E911C3F
:108CF000880C991C880C991C2DB73EB72819390986
:108D00000FB6F8943EBF0FBE2DBF8DB79EB701962C
:108D10002C01EDB7FEB7E819F9090FB6F894FEBFBC
:108D20000FBEEDBF2DB73EB72F5F3F4F390100910A
:108D3000680501279E0127563F4FA401BC01CE01C3
:108D400089569F4F0E94EB160091680501279E01EE
:108D500027563F4FA401B301CE0189569F4F0E9471
:108D6000EB1630916805C256DF4F3883CE59D0409C
:108D7000332309F4CBC011E0C256DF4F0881CE592E
:108D8000D04001279E0127563F4F44E050E06AE75C
:108D900076E0CE0189569F4F0E94EB160091680540
:108DA00001279E0127563F4F44E050E06EE776E0F2
:108DB000CE0189569F4F0E94EB160091680501274E
:108DC0009E0127563F4F44E050E062E876E0CE0136
:108DD00089569F4F0E94EB160091680501279E015E
:108DE00027563F4F44E050E066E876E0CE018956D2
:108DF0009F4F0E94EB160091680501279E012756A0
:108E00003F4F44E050E06AE876E0CE0189569F4F3C
:108E10000E94EB160091680501279E0127563F4FDF
:108E200040E150E066E176E0CE0189569F4F0E9416
:108E3000EB160091680501279E0127563F4F44E03D
:108E400050E0BE0163577F4FCE0189569F4F0E946D
:108E5000EB16C156DF4F88819981CF59D0400FB6AC
:108E6000F8949EBF0FBE8DBF0091680501279E013B
:108E700027563F4F4CE050E0BE016F5F7F4FCE0161
:108E800089569F4F0E94EB160091680501279E01AD
:108E900027563F4F44E050E0BE0163577F4FCE015D
:108EA00089569F4F0E94EB160091680501279E018D
:108EB00027563F4F44E050E0BE0163577F4FCE013D
:108EC00089569F4F0E94EB1601E09E0127563F4FA7
:108ED00041E050E0B701CE0189569F4F0E94EB164A
:108EE0009E0127563F4F41E050E0BE016F5F7F4F2C
:108EF000CE0189569F4F0E94EB16F701A080898111
:108F0000A89E50011124812C912C9DC0C456DF4F86
:108F10008881CC59D04090E09C012E5F3F4FCF55C7
:108F2000DF4F39832883C15AD040A6E4B6E040E041
:108F300050E080E090E04601B70131E0C356DF4FDA
:108F40003883CD59D040CF55DF4FE881F981C15AE0
:108F5000D040E817F90764F4C356DF4F1882CD59A3
:108F6000D0409C018430910558F023E030E008C0E7
:108F7000F101E40FF51F00811181228133810BC0C3
:108F8000220F331F220F331FF401E20FF31F008162
:108F90001181228133810D931D932D933D93C356EF
:108FA000DF4FF881CD59D040FF2341F0F201E40FAB
:108FB000F51F008111812281338111C09C01843011
:108FC000910510F023E030E0220F331F220F331FF2
:108FD000FB01E20FF31F0081118122813381509642
:108FE0000D931D932D933C935397C356DF4F2881C8
:108FF000CD59D040222341F0F301E40FF51F008149
:1090000011812281338111C09C018430910510F0BF
:1090100023E030E0220F331F220F331FF501E20F50
:10902000F31F008111812281338190960D931D934E
:109030002D933C93939701964C5F5F4F843091053D
:1090400009F07BCF98CE009168058A149B0491F0BB
:1090500001279E0127563F4F44E050E0BE01635771
:109060007F4FCE0189569F4F0E94EB163FEF831A28
:10907000930AE9CF11E001279E0127563F4F44E0B4
:1090800050E06AE675E0CE0189569F4F0E94EB16CC
:109090000091680501279E0127563F4F44E250E0AA
:1090A00061EF75E0CE0189569F4F0E94EB1601E0FB
:1090B0009E0127563F4F41E050E0BE0165567F4F6D
:1090C000CE0189569F4F0E94EB169E0127563F4FB7
:1090D00041E050E0B601CE0189569F4F0E94EB1649
:1090E0000091680501279E0127563F4F44E050E05C
:1090F000B701CE0189569F4F0E94EB16009168057B
:1091000001279E0127563F4F44E050E0BE016F5FAC
:109110007F4FCE0189569F4F0E94EB16C556DF4FF9
:10912000A880CB59D040F6018081A89E500111241F
:10913000812C912C009168058A149B0491F00127E1
:109140009E0127563F4F44E050E0BE0163577F4FDA
:10915000CE0189569F4F0E94EB16FFEF8F1A9F0A90
:10916000E9CF11E001279E0127563F4F41E050E033
:10917000B701CE0189569F4F0E94EB1600916805FA
:1091800001279E0127563F4F41E050E0BE016F5F2F
:109190007F4FCE0189569F4F0E94EB1600916805C4
:1091A00001279E0127563F4F40E150E0BE016F5F0F
:1091B0007F4FCE0189569F4F0E94EB1600916805A4
:1091C00001279E0127563F4F44E050E0B701CE01F2
:1091D00089569F4F0E94EB160091680501279E015A
:1091E00027563F4F44E050E0BE016F5F7F4FCE01F6
:1091F00089569F4F0E94EB160091680501279E013A
:1092000027563F4F42E050E0B601CE0189569F4FAE
:109210000E94EB160091680501279E0127563F4FDB
:1092200040E150E0BE016F5F7F4FCE0189569F4FF6
:109230000E94EB160091680501112EC089809A806A
:10924000AB80BC8020E030E84BE355E4C501B401BD
:109250000E94B2AC882301F18092D3049092D4048E
:10926000A092D504B092D6048D819E81AF81B8853D
:109270008093D7049093D804A093D904B093DA04D0
:1092800089859A85AB85BC858093DB049093DC044B
:10929000A093DD04B093DE0411E001279E01275660
:1092A0003F4F42E050E0BE016F5F7F4FCE018956D5
:1092B0009F4F0E94EB160091680501279E012756DB
:1092C0003F4F4CE050E0BE016F5F7F4FCE018956AB
:1092D0009F4F0E94EB1600916805011115C020E018
:1092E00030E84BE355E469817A818B819C810E944F
:1092F000B2AC882349F08CE0FE013196A5EBB4E0D6
:1093000001900D928A95E1F711E001279E01275601
:109310003F4F42E050E0BE016F5F7F4FCE01895664
:109320009F4F0E94EB160091680501279E0127566A
:109330003F4F41E050E0BE016F5F7F4FCE01895645
:109340009F4F0E94EB160091680501279E0127564A
:109350003F4F40E250E0BE016F5F7F4FCE01895624
:109360009F4F0E94EB160091680501279E0127562A
:109370003F4F41E050E0B701CE0189569F4F0E9418
:10938000EB160091680501279E0127563F4F45E0E7
:1093900050E0BE016F5F7F4FCE0189569F4F0E9404
:1093A000EB1680916805811102C00E94E1310091A5
:1093B000680511E001279E0127563F4F4AE150E022
:1093C000BE016F5F7F4FCE0189569F4F0E94EB1603
:1093D0000091680501279E0127563F4F44E350E066
:1093E000BE016F5F7F4FCE0189569F4F0E94EB16E3
:1093F0000091680501279E0127563F4F46E050E047
:10940000BE016F5F7F4FCE0189569F4F0E94EB16C2
:109410000091680501279E0127563F4F4DE050E01F
:10942000BE016F5F7F4FCE0189569F4F0E94EB16A2
:109430000091680501279E0127563F4F44E050E008
:10944000BE016F5F7F4FCE0189569F4F0E94EB1682
:109450000091680501110CC089819A81AB81BC81A2
:109460008093B8059093B905A093BA05B093BB0556
:1094700081E008279E0127563F4F4CE050E0BE0197
:109480006F5F7F4FCE0189569F4F0E94EB16009170
:109490006805011109C08CE0FE013196ABE5B5E02D
:1094A00001900D928A95E1F711E001279E01275660
:1094B0003F4F4CE650E0BE016F5F7F4FCE018956B3
:1094C0009F4F0E94EB1619821A821B821C821D82FA
:1094D0001E821F82188619861A861B861C8600919A
:1094E000680501279E0127563F4F4CE050E0BE0122
:1094F0006F5F7F4FCE0189569F4F0E94EB16009100
:10950000680501279E0127563F4F48E050E0BE0105
:109510006F5F7F4FCE0189569F4F0E94EB16C95651
:10952000DF4F88819981C759D040845691090E94A4
:10953000523E809369058823C1F00E94F315C956F5
:10954000DF4F68817981C759D040645671098DE237
:1095500093E10E94161667E472E085E293E10E94AF
:1095600050168AE00E94751858C0C756DF4F2881F0
:109570003981C959D040CB56DF4F88819981C5596F
:10958000D04028173907E9F0109369050E94F615B5
:10959000CB56DF4F68817981C559D04085E093E192
:1095A0000E945016C756DF4F68817981C959D04053
:1095B00080E093E10E94501680EF92E10E94E51551
:1095C0002CC080916805811128C00E94F31507E323
:1095D00013E0F80181918F01882319F00E9475181A
:1095E000F8CFC956DF4F68817981C759D04064569A
:1095F000710983ED92E10E941616C756DF4F48812C
:109600005981C959D04060E070E086EC92E10E9437
:109610005A1683EC92E10E94E5158091680581114C
:1096200006C080916905811102C00E94D53D8091DC
:109630006805811101C013D80E94941690916905A4
:1096400081E08927CD55DF4F28813981C35AD04029
:109650000FB6F8943EBF0FBE2DBFCC55DF4F0FB6EF
:10966000F894DEBF0FBECDBFDF91CF911F910F9158
:10967000FF90EF90DF90CF90BF90AF909F908F9032
:109680007F906F905F904F903F902F90089581E072
:10969000809368052CDA109268050895F8DF81112F
:1096A00026CA0E94EC4181E00895BF92CF92DF92DA
:1096B000EF92FF920F931F93CF93DF93CDB7DEB757
:1096C00028970FB6F894DEBF0FBECDBF9091E2048D
:1096D000981709F47AC0B82E882309F453C080E0A3
:1096E00090E0A0EAB0E48D839E83AF83B887C090FA
:1096F0006A05D0906B05E0906C05F0906D0520E058
:1097000030E0A901C701B6010E94B2AC87FF0CC0CE
:10971000A701960160E070E080EA90E40E94D8AB77
:109720006D837E838F83988720E030E04FE153E4A0
:109730006D817E818F8198850E94B5AE181644F4A4
:1097400080E090E0AFE1B3E48D839E83AF83B88780
:10975000209158023091590240915A0250915B0277
:109760006D817E818F8198850E94B5AE181654F464
:1097700019821A821B821C82BE016F5F7F4FCE014D
:10978000059698D4609150027091510280915202D6
:10979000909153022091540230915502409156020B
:1097A0005091570219821A821B821C82E090580243
:1097B000F090590200915A0210915B02FE0131961D
:1097C0006F01C4D38B2D0E947C3080E028960FB6A9
:1097D000F894DEBF0FBECDBFDF91CF911F910F91E7
:1097E000FF90EF90DF90CF90BF9008952F923F921F
:1097F0004F925F926F927F928F929F92AF92BF92A1
:10980000CF92DF92EF92FF920F931F93CF93DF934C
:10981000CDB7DEB7A0970FB6F894DEBF0FBECDBFB1
:109820001C017F8F6E8F498F28A3DC018D909D9046
:10983000AD90BC90FB01408051806280738022ED2E
:1098400030E040EE50ECC301B201002309F43BC00C
:109850000E94B5AE87FD35C227E030E04EE353E409
:10986000C301B2010E94B2AC18160CF42AC223EA5A
:1098700031E040E450ECC501B4010E94B5AE87FD73
:1098800020C227E030E042E253E4C501B4010E9467
:10989000B2AC18160CF415C227E030E041E253E4F4
:1098A000C501B4010E94B2AC18160CF40AC227E03C
:1098B00030E041E253E4C301B2010E94B2AC181699
:1098C0000CF4FFC124C00E94B5AE87FDFAC127E0A9
:1098D00030E04EE353E4C301B2010E94B2AC18166B
:1098E0000CF4EFC123EA31E040E450ECC501B401CF
:1098F0000E94B5AE87FDE5C127E030E042E253E4C7
:10990000C501B4010E94B2AC18160CF4DAC1E090A3
:109910005802F090590200915A0210915B02809116
:109920004C0290914D02A0914E02B0914F028A8F4D
:109930009B8FAC8FBD8F8091460290914702A09182
:109940004802B091490280934C0290934D02A0933B
:109950004E02B0934F0219821A821B821C82DE01D2
:1099600011966D01A3019201C501B401EFD281E00E
:109970009CDE81113EC18091910582FF11C0209132
:109980006A0530916B0540916C0550916D0560E062
:1099900070E080E890EC0E94D8AB6B017C0106C0BF
:1099A000C12CD12C40E2E42E41ECF42ECD8ADE8A8B
:1099B000EF8AF88E812C912CA12C31E4B32E898A68
:1099C0009A8AAB8ABC8ABE016F5E7F4FCE014596F4
:1099D00071D31091E6041092E60482E0FCD1D1D15B
:1099E00012FD05C060E070E080EC9FE7BDC04090D4
:1099F00058025090590260905A0270905B0289821E
:109A00009A82AB82BC8220E030E040EA50E4C3019D
:109A1000B2010E94D9AB6D837E838F8398878E01BC
:109A20000B5F1F4FBE016F5F7F4FC80143D3CD86D1
:109A3000DE86EF86F88A80E090E0A0E8BFE38987C1
:109A40009A87AB87BC87BE01675F7F4FCE010D96BB
:109A500031D3F090E6041092E60482E0BCD191D1BB
:109A6000F2FEC0CF80912D0C8F3F09F45BC0C090F7
:109A70005802D0905902E0905A02F0905B02809018
:109A8000580290905902A0905A02B0905B0220E0D8
:109A900030E040E05FE3C701B6010E94D9AB9B0113
:109AA000AC01C501B4010E94B2AC87FF1CC01C9977
:109AB0001AC080E090E0A0E8BFE389839A83AB837B
:109AC000BC832AE037ED43EA5BE3C501B4010E94A1
:109AD000D9AB6D837E838F839887BE016F5F7F4F85
:109AE000C801E8D2CCCFA7019601C501B4010E94FC
:109AF000D8AB9B01AC016091360C7091370C809112
:109B0000380C9091390C0E94D9AB6093360C70934D
:109B1000370C8093380C9093390C80912D0C8F5F0B
:109B200080932D0C20E030E040E450E46091580236
:109B30007091590280915A0290915B020E94F0AE9E
:109B40006B017C01A3019201C301B2010E94D9AB58
:109B50009B01AC01C701B6010E94D9AB2DEC3CECD6
:109B60004CE45EE30E94F0AE20916A0530916B05F3
:109B700040916C0550916D050E94D9AB7B018C0121
:109B8000898D8250823048F580E090E0A0E0B1E419
:109B900089839A83AB83BC83609158027091590288
:109BA00080915A0290915B02A98DA33029F020E0A8
:109BB00030E040EA50E404C020E030E048EC51E4FA
:109BC0000E94D9AB6D837E838F839887BE016F5FC0
:109BD0007F4FCE0105966ED207C0B98DB13021F40A
:109BE00080E063DD811105C0E8A1E33008F449C0DD
:109BF00008C098A1933008F46DC0E12CF12C00EC62
:109C00001FE72BE3C22E23E0D22ED6018D916D01EA
:109C1000882319F00E947518F8CFF10160817181D5
:109C20008281938143E050E00E94F31993E4C92EAE
:109C300093E0D92ED6018D916D01882319F00E94F1
:109C40007518F8CFEE8DFF8D6081718182819381CF
:109C500043E050E00E94F31988E4C82E83E0D82E38
:109C6000D6018D916D01882319F00E947518F8CFE7
:109C700043E050E0B701C8010E94F3198AE00E9456
:109C800075188A8D9B8DAC8DBD8D80934C02909301
:109C90004D02A0934E02B0934F029701A801B70165
:109CA000C8010E949EAF882389F080E0FEDC0E94FC
:109CB000F6158EE993E10E94E5152E2D7F2DC80142
:109CC0001AC020E070E080EC9FE715C02E2D7F2D9C
:109CD000C80111C08A8D9B8DAC8DBD8D80934C02C7
:109CE00090934D02A0934E02B0934F02E12CF12CC1
:109CF00000EC1FE7DACFC22ED72E7C01C701B601D8
:109D0000A0960FB6F894DEBF0FBECDBFDF91CF9106
:109D10001F910F91FF90EF90DF90CF90BF90AF9089
:109D20009F908F907F906F905F904F903F902F907B
:109D30000895CF93DF93C0E5D2E0488159816A81CD
:109D40007B8187E294E10E9430164C815D816E81B7
:109D50007F8183E294E10E943016488559856A85A7
:109D60007B858FE194E10E9430164C855D856E8580
:109D70007F858BE194E10E943016DF91CF910C94A6
:109D8000AB3B2CE532E048E552E064E572E080E56B
:109D900092E00C94B36A8CE592E00C94006BCF9344
:109DA000DF9380E00E94CD5AC4E7D5E068837983D1
:109DB0008A839B8381E00E94CD5A6C837D838E834E
:109DC0009F8382E00E94CD5A688779878A879B8724
:109DD000DF91CF9108951F93CF93DF93CDB7DEB777
:109DE00060970FB6F894DEBF0FBECDBF182FD7DF38
:109DF0008091740590917505A0917605B0917705D5
:109E000089839A83AB83BC8380917805909179058F
:109E1000A0917A05B0917B058D839E83AF83B8872F
:109E200080917C0590917D05A0917E05B0917F0584
:109E300089879A87AB87BC8780915C0290915D028D
:109E4000A0915E02B0915F028D879E87AF87B88B2D
:109E5000CE0101960E94125A1E3F51F480E1FE018C
:109E60003196A0E5B2E001900D928A95E1F716C017
:109E700024E0129FC0011124FC01E05BFD4FA1E032
:109E8000B0E0AC0FBD1FA80FB91F8D919D910D9033
:109E9000BC91A02D80839183A283B38360960FB67B
:109EA000F894DEBF0FBECDBFDF91CF911F91089513
:109EB000AF92BF92CF92DF92EF920F931F93A12C9C
:109EC000B12C6501E12C8C012CE532E048E552E033
:109ED00064E572E080E592E00E9477691F910F913E
:109EE000EF90DF90CF90BF90AF900895AF92BF9268
:109EF000CF92DF92EF920F931F93CF93DF9300D017
:109F00001F92CDB7DEB769837A838B839C83A12CA4
:109F1000B12C6501E12C8E010F5F1F4F2CE835E05D
:109F200048E855E064E875E080E895E00E947769CC
:109F30000F900F900F900F90DF91CF911F910F9185
:109F4000EF90DF90CF90BF90AF9008954F925F92C7
:109F50006F927F928F929F92AF92BF92CF92DF9239
:109F6000EF92FF920F931F93CF93DF93CDB7DEB79E
:109F70002C970FB6F894DEBF0FBECDBF2B013C016E
:109F800029873A874B875C8747015801F601E080B3
:109F9000F1800281138120E030E0A901B701C801FE
:109FA0000E94B2AC811107C0E2E3F4E18591959182
:109FB000A591B49102C0C701D8018D839E83AF8360
:109FC000B88720E030E0A901B701C8010E94B2AC17
:109FD000811108C0E0904602F090470200914802CB
:109FE00010914902C701D80189839A83AB83BC834E
:109FF000A5019401609158027091590280915A0212
:10A0000090915B020E94B2AC87FF0BC08092580215
:10A0100090925902A0925A02B0925B02CE0105962C
:10A0200047DF409250025092510260925202709269
:10A03000530289859A85AB85BC85809354029093A1
:10A040005502A0935602B0935702CE01019630DF1D
:10A05000A5019401609158027091590280915A02B1
:10A0600090915B020E94B5AE18165CF48092580283
:10A0700090925902A0925A02B0925B02CE010596CC
:10A0800017DF0E94E15A2C960FB6F894DEBF0FBE80
:10A09000CDBFDF91CF911F910F91FF90EF90DF9097
:10A0A000CF90BF90AF909F908F907F906F905F9078
:10A0B0004F900895CF92DF92EF92FF920F931F93EC
:10A0C0006B01FC01E080F18002811381E0E5F2E0A8
:10A0D000248135814681578160817181828193819C
:10A0E00035DF1F910F91FF90EF90DF90CF90089593
:10A0F000CF92DF92EF92FF920F931F936A01E0904D
:10A100005802F090590200915A0210915B02FB0133
:10A110002081318142815381FC0160817181828182
:10A12000938114DF1F910F91FF90EF90DF90CF90FC
:10A13000089580914C0290914D02A0914E02B091F1
:10A140004F028093700590937105A0937205B093B0
:10A15000730580914A0290914B0290936F05809312
:10A160006E0584E690E090934B0280934A02089536
:10A170008091700590917105A0917205B091730561
:10A1800080934C0290934D02A0934E02B0934F02E5
:10A1900080916E0590916F0590934B0280934A02D7
:10A1A000089524E0829FC0011124FC01E759FB4E71
:10A1B0004591559165917491FC01E75CFD4F408399
:10A1C000518362837383FC01E35AFB4E45915591A1
:10A1D00065917491FC01E35DFD4F4083518362837F
:10A1E00073830895CF92DF92EF92FF92CF93DF9324
:10A1F00020914502222309F485C0EC01C090390268
:10A20000D0903A02E0903B02F0903C02A701960108
:10A21000688179818A819B810E94B2AC87FF04C0EA
:10A22000C882D982EA82FB82C0902D02D0902E0291
:10A23000E0902F02F0903002A701960168817981A9
:10A240008A819B810E94B5AE181624F4C882D982F7
:10A25000EA82FB82C0903D02D0903E02E0903F0235
:10A26000F0904002A70196016C817D818E819F81D3
:10A270000E94B2AC87FF04C0CC82DD82EE82FF82F6
:10A28000C0903102D0903202E0903302F09034025C
:10A29000A70196016C817D818E819F810E94B5AE60
:10A2A000181624F4CC82DD82EE82FF82C090410237
:10A2B000D0904202E0904302F0904402A701960140
:10A2C000688579858A859B850E94B2AC87FF04C02A
:10A2D000C886D986EA86FB86C0903502D0903602C1
:10A2E000E0903702F0903802A701960168857985E1
:10A2F0008A859B850E94B5AE181624F4C886D98637
:10A30000EA86FB86DF91CF91FF90EF90DF90CF90B0
:10A3100008958F929F92AF92BF92CF92DF92EF9269
:10A32000FF9280E895E05EDF8091A90383FD7DC008
:10A33000C0908C05D0908D05E0908E05F0908F0533
:10A3400020915C0230915D0240915E0250915F026B
:10A35000C701B6010E94B2AC882309F466C06091BF
:10A36000CC047091CD048091CE049091CF042091C3
:10A37000A104211117C00E9421AD20911D0230912E
:10A380001E026217730774F4C0925C02D0925D02E1
:10A39000E0925E02F0925F020E94F31580E094E189
:10A3A0000E94E51580908C0590908D05A0908E05FB
:10A3B000B0908F0520915C0230915D0240915E0269
:10A3C00050915F02C501B4010E94D8AB6B017C01C2
:10A3D00020E030E0A9010E94B5AE87FF04C0C701AC
:10A3E000B601905802C0C701B601209160023091B9
:10A3F000610240916202509163020E94F0AE20E03F
:10A4000030E048E453E40E94B5AE181674F480922C
:10A410005C0290925D02A0925E02B0925F020E9486
:10A42000F31581EE93E10E94E51560914A02709167
:10A430004B02072E000C880B990B0E9454AD209103
:10A440004C0230914D0240914E0250914F020E94B9
:10A45000F0AE2AE037ED43E25CE30E94F0AE46DD69
:10A4600080E1E0E8F5E0A0E5B2E001900D928A9588
:10A47000E1F7FF90EF90DF90CF90BF90AF909F906B
:10A480008F9008951F93CF93DF93882329F0D09165
:10A490009205D095D17001C0D0E0662339F01091BB
:10A4A00092051695117081E0182701C010E0442331
:10A4B00041F0C0919205C2FBCC27C0F981E0C827CA
:10A4C00001C0C0E0D11104C0111102C0CC23D1F0F1
:10A4D0000E94F3158BED93E10E94E515DD2319F041
:10A4E00088E50E947518112319F089E50E947518F6
:10A4F000CC2319F08AE50E94751883ED93E10E9440
:10A50000E515C1E08C2FDF91CF911F910895CF9277
:10A51000DF92EF92FF92CF93DF93C82FD0E0FE013E
:10A52000E053FC4E8491811107C00E94F3158EEA1E
:10A5300093E10E94E5158AE0FE01EE0FFF1FEE0F8A
:10A54000FF1FE65DFB4EC590D590E590F490682F17
:10A5500070E080E090E00E9454AD9B01AC01C70127
:10A56000B6010E94B9ACDF91CF91FF90EF90DF90E0
:10A57000CF9008954F925F926F927F928F929F92A9
:10A58000AF92BF92CF92DF92EF92FF920F931F9301
:10A59000CF93DF93CDB7DEB768970FB6F894DEBFE1
:10A5A0000FBECDBF2A013B016901E82EF12CF70156
:10A5B000EA5CFB4EE491AA24A3941E160CF4A12C91
:10A5C000BB24B39420E030E0A901C301B2010E9492
:10A5D000B5AE18160CF0B12C80E0DFD769837A8312
:10A5E0008B839C8381E0D9D76D837E838F8398870B
:10A5F00082E0D3D769877A878B879C8783E0CDD722
:10A600006D877E878F87988BEE0CFF1CEE0CFF1CEE
:10A6100088248394912C8C0E9D1E8E0C9F1CF4011B
:10A6200010821182128213829E01235F3F4FAE017E
:10A63000475F5F4FBE016B5F7F4FCE0101960E9467
:10A64000D869F4014082518262827382198A1A8A1F
:10A650001B8A1C8A20E030E0A901B801C6010E94D3
:10A66000B2AC811108C0F701E65DFB4E8591959172
:10A67000A591B49102C0C801D6018D8B9E8BAF8B82
:10A68000B88FCE0141966C01E12C8E010B5E1F4FFD
:10A690009E01235F3F4FAE01475F5F4FBE016B5F7F
:10A6A0007F4F40970E9494688CD7AB100E94403037
:10A6B00068960FB6F894DEBF0FBECDBFDF91CF9185
:10A6C0001F910F91FF90EF90DF90CF90BF90AF90D0
:10A6D0009F908F907F906F905F904F90089521E0B2
:10A6E00030E0082E01C0220F0A94EAF790919105FC
:10A6F000922B9093910590919205292B209392058E
:10A7000024E0829FC0011124FC01EF5AFB4E4591C9
:10A71000559165917491FC01E05BFD4F408351833D
:10A720006283738308954F925F926F927F928F92AC
:10A730009F92AF92BF92FF920F931F93CF93DF939D
:10A74000833008F06AC0F82EC82FD0E0FE01EA5C22
:10A75000FB4E8491CC0FDD1FCC0FDD1FFE01EB5BA8
:10A76000FB4E4590559065907490682F880F770B3D
:10A77000880B990B0E9454AD4B015C0120E030E046
:10A7800040EC5FE3C301B2010E94F0AEA501940169
:10A790000E94F0AEAB01BC0100E010E098018F2DEB
:10A7A000E9DEFE01E75CFB4E259135914591549120
:10A7B000C501B4010E94F0AE4B015C0120E030E025
:10A7C000A9010E94B2AC8823C1F0B501A401705860
:10A7D00000E010E098018F2DCDDE8F2D98DE2B014B
:10A7E0003C01A5019401C501B4010E94D9ABAB01A4
:10A7F000BC01930182018F2DBDDE8F2D70DFC1DA88
:10A80000FE01E058FA4FC05BDD4F88819981AA8133
:10A81000BB8180839183A283B383DF91CF911F910A
:10A820000F91FF90BF90AF909F908F907F906F900F
:10A830005F904F90089580E1E5EDF5E0DF01982FFE
:10A840001D929A95E9F7E8EAF5E0DF01982F1D924D
:10A850009A95E9F7E1ECF5E0DF011D928A95E9F7B9
:10A860001092BD051092BE051092BF051092C00552
:10A8700081EF95E00E9472A51092910610929406C5
:10A88000109292061092930610928E0608954F929F
:10A890005F926F927F928F929F92AF92BF92CF9270
:10A8A000DF92EF92FF920F931F93CF93DF93CDB779
:10A8B000DEB768970FB6F894DEBF0FBECDBF8C0130
:10A8C0005B014A01FC01EF5BFF4F60817181828176
:10A8D00093810E9452AD6B017C01D5012D913D9178
:10A8E0004D915C910E94F0AE0E949FAC0E9426ADFB
:10A8F00069877A878B879C87F40120813181428127
:10A900005381C701B6010E94F0AE0E949FAC0E9425
:10A9100026AD6D877E878F87988B29853A854B85F5
:10A920005C85283731054105510540F488E790E002
:10A93000A0E0B0E089879A87AB87BC872D853E85EC
:10A940004F855889283731054105510540F488E77E
:10A9500090E0A0E0B0E08D879E87AF87B88B98012C
:10A96000235B3F4FD9018D919D910D90BC91A02DFE
:10A9700089839A83AB83BC83BC01CD010E9454AD13
:10A980002B013C0169857A858B859C850E9452AD9F
:10A99000698B7A8B8B8B9C8B20E030E0A901C30103
:10A9A000B2010E94B2AC882329F1A7019601C70128
:10A9B000B6010E94F0AE4B015C0129893A894B89AE
:10A9C0005C89CA01B9010E94F0AE9B01AC01C501CE
:10A9D000B4010E94D8AB4B015C01A3019201C301F9
:10A9E000B2010E94D9AB9B01AC01C501B4010E9428
:10A9F000B9AC03C060E070E0CB010E949FAC0E9444
:10AA000026AD6D837E838F83988769817A818B8160
:10AA10009C8190958095709561957F4F8F4F9F4F4A
:10AA20000E9454AD4B015C016D857E858F859889B0
:10AA30000E9452AD69837A838B839C8320E030E04F
:10AA4000A901C501B4010E94B2AC882349F1298152
:10AA50003A814B815C81CA01B9010E94F0AE6D8BD5
:10AA60007E8B8F8B988FA7019601C701B6010E943C
:10AA7000F0AE9B01AC016D897E898F89988D0E9413
:10AA8000D8AB6B017C01A5019401C501B4010E9402
:10AA9000D9AB9B01AC01C701B6010E94B9AC03C0A0
:10AAA00060E070E0CB010E948FADF80185A096A018
:10AAB000A7A0B0A4750164012D813E814F81588506
:10AAC000C21AD30AE40AF50A0E9426ADC61AD70AAA
:10AAD000E80AF90AF7FE73C020E030E0A901C301DB
:10AAE000B2010E94B2AC882309F443C0A3019201D1
:10AAF000C301B2010E94D9AB6B017C01C501B40155
:10AB00000E9452AD9B01AC01C701B6010E94F0AE9C
:10AB10006B017C0129893A894B895C89CA01B90199
:10AB20000E94F0AE9B01AC01C701B6010E94D8ABF8
:10AB30006B017C0129813A814B815C81CA01B90199
:10AB40000E94F0AE9B01AC01C701B6010E94D9ABD7
:10AB50006B017C0120E030E040E850E4C301B20129
:10AB60000E94F0AE9B01AC01C701B6010E94B9ACD6
:10AB700003C060E070E0CB010E949FAC7B016C01E0
:10AB800020E030E0A9010E94B5AE181624F0E12CB7
:10AB9000F12CC12CD12CB701C6010E9426AD6D83CA
:10ABA0007E838F83988786169706A806B90620F4B9
:10ABB0008D829E82AF82B886C12CD12C76018D8188
:10ABC0009E81AF81B885F80181A792A7A3A7B4A7FA
:10ABD000C80ED91EEA1EFB1EC5A6D6A6E7A6F0AA79
:10ABE000EB5BFF4F29853A854B855C85208331835C
:10ABF0004283538334968D859E85AF85B889808343
:10AC00009183A283B38368960FB6F894DEBF0FBE1C
:10AC1000CDBFDF91CF911F910F91FF90EF90DF900B
:10AC2000CF90BF90AF909F908F907F906F905F90EC
:10AC30004F9008952F923F924F925F926F927F9222
:10AC40008F929F92AF92BF92CF92DF92EF92FF923C
:10AC50000F931F93CF93DF93009709F471C08B017B
:10AC6000EC01D984CA847B846C848D809E80AF8003
:10AC7000B8842D2D3C2D472D562DC501B4010E94C1
:10AC8000B2AC811108C00115110509F459C0F801D1
:10AC9000808180FF55C0888181FD34C00115110578
:10ACA00031F0F801258036804780508408C08BE061
:10ACB000282E87ED382E83E2482E8BE3582E898983
:10ACC0009A89AB89BC89BC01CD0190589B01AC012C
:10ACD0000E94D9AB2D853E854F8558890E94F0AEE4
:10ACE0009B01AC01C201B1010E94D8AB7B018C0178
:10ACF0009B01AC016D2D7C2D872D962D0E94B2AC51
:10AD000087FF04C0ED2CFC2C072D162D9701A80100
:10AD1000C501B4010E94B2AC882391F088818160A2
:10AD20008883CE010E943535882321F088818E7F6B
:10AD3000888306C0A701B8014D835E836F8378873F
:10AD4000DF91CF911F910F91FF90EF90DF90CF9007
:10AD5000BF90AF909F908F907F906F905F904F903B
:10AD60003F902F900895FF920F931F93CF93DF93FF
:10AD7000C0919406C150CF70D091920680919406F4
:10AD8000D817E9F060E070E086E5F82ECD17B9F04D
:10AD9000FC9E800111240B56194FF801808183FD20
:10ADA00003C0C80147DFB801C150CF70809192063F
:10ADB000D81761F3CD1719F0DF5FDF70F7CFDF91A0
:10ADC000CF911F910F91FF9008954F925F926F92D4
:10ADD0007F928F929F92AF92BF92FF920F931F9399
:10ADE000CF93DF93009709F459C0F42EEB018C0147
:10ADF000FC01808181FD3CC0458056806780708465
:10AE00008D809E80AF80B884A5019401C301B201FA
:10AE10000E94B2AC87FF2CC0F80181899289A38976
:10AE2000B489BC01CD0190589B01AC010E94D9AB03
:10AE3000F80125853685478550890E94F0AE9B0133
:10AE4000AC01C301B2010E94D8AB2B013C01A501AA
:10AE500094010E94B2AC87FF0BC088818160888317
:10AE6000CE010E943535882391F088818E7F8883BA
:10AE700029853A854B855C856D817E818F8198859A
:10AE80000E94B2AC81110AC0F092920607C04D82B6
:10AE90005E826F827886F0929206EACFDF91CF9140
:10AEA0001F910F91FF90BF90AF909F908F907F90D8
:10AEB0006F905F904F900895CF92DF92EF92FF9244
:10AEC0000F931F93CF93DF9310919206C0E0D0E0D1
:10AED00086E5C82E80919406181709F1C19EB0012D
:10AEE0001124CB018B56994F7C01FC01808183FD9D
:10AEF0000AC00E2DDF2C209769F0CE010E94353557
:10AF0000882341F002C00C2FDD2E1F5F1F70C02F61
:10AF1000DD2DE0CF412FB701CE0157DFF6CFDF9116
:10AF2000CF911F910F91FF90EF90DF90CF900895F8
:10AF30002F923F924F925F926F927F928F929F9249
:10AF4000AF92BF92CF92DF92EF92FF920F931F9337
:10AF5000CF93DF93CDB7DEB72E970FB6F894DEBF51
:10AF60000FBECDBF209191062987309194063B8773
:10AF700096E58B85E9858E1759F08B8581508F700A
:10AF8000989FF0011124EB56F94F208123FD0DC04D
:10AF9000812C912CA12CB12C1A861C861D861E8614
:10AFA000212C312C00E010E01AC08B87E2CFF6E5AF
:10AFB0002985F29FC0011124FC01EB56F94F1F01B6
:10AFC000808183FF11C0FA84EC84DD84CE8489857E
:10AFD0008F5F8F708987FA86EC86DD86CE86F9854D
:10AFE0002B85F213E4CF93C06581768187819085AC
:10AFF0000E945DAFF62EE72ED82EC92E0115110541
:10B0000009F47FC0F801808180FD04C0F1018081D6
:10B0100080FF77C0F801808181608083C8010E9431
:10B02000353581116AC0F801618172818381948113
:10B030000E945DAF2B013C019B01AC0160E070E020
:10B0400080E89FE30E94B9AC4B015C019B01AC011D
:10B050006F2D7E2D8D2D9C2D0E94F0AE69837A83FD
:10B060008B839C83A50194016A857C858D859E8553
:10B070000E94F0AE6D837E838F839887AE014F5F11
:10B080005F4FBE016B5F7F4FC80101DCF80186A9ED
:10B09000882399F12091B8053091B9054091BA05FE
:10B0A0005091BB05FD9660817181828193810E94E0
:10B0B000F0AE209166063091670640916806509187
:10B0C00069060E94F0AE4B015C019B01AC01C3011B
:10B0D000B2010E94F0AE0E9426ADF80172AF61AFDE
:10B0E000A50194016F2D7E2D8D2D9C2D0E94F0AE1B
:10B0F0000E9426ADF80174AF63AFF80180818E7FA6
:10B1000080838F2C9E2CAD2CBC2C810160CF211410
:10B11000310409F473C0F101808181608083C8012A
:10B120000E943535811166C0F10161817281838190
:10B1300094810E945DAF6B017C019B01AC0160E0DA
:10B1400070E080E89FE30E94B9AC2B013C012DEC3C
:10B150003CEC4CE45DE30E94F0AE69837A838B8320
:10B160009C83A3019201B401C5010E94F0AE6D83DE
:10B170007E838F839887AE014F5F5F4FBE016B5F09
:10B180007F4FC10184DBF10186A9882399F12091C9
:10B19000B8053091B9054091BA055091BB05FD96AF
:10B1A00060817181828193810E94F0AE2091660658
:10B1B0003091670640916806509169060E94F0AE92
:10B1C0004B015C019B01AC01C701B6010E94F0AECE
:10B1D0000E9426ADF10172AF61AF2DEC3CEC4CE466
:10B1E0005DE3C501B4010E94F0AE0E9426ADF101FD
:10B1F00074AF63AFF10180818E7F80832E960FB68E
:10B20000F894DEBF0FBECDBFDF91CF911F910F919C
:10B21000FF90EF90DF90CF90BF90AF909F908F9076
:10B220007F906F905F904F903F902F900895809106
:10B2300094069091920681508F70891711F093DDDA
:10B240003BDE76CEAF92BF92CF92DF92EF92FF922B
:10B250000F931F93CF939091940680919106981726
:10B2600091F0E091910686E5E89FF0011124EA5102
:10B27000F94FC0818091910690919406891729F029
:10B280008F5F8F70F9CFC091C704CC2339F10E9432
:10B2900068110091A4051091A5052091A605309193
:10B2A000A705DC01CB01011511052105310571F45C
:10B2B0008C599F4FAF4FBF4F8093A4059093A50526
:10B2C000A093A605B093A705CFEF21C0801B910BDB
:10B2D000A20BB30BB7FF1BC0CFEF19C01092A40590
:10B2E0001092A5051092A6051092A70560E070E0E7
:10B2F00020E04FEF50E088E0CF911F910F91FF9039
:10B30000EF90DF90CF90BF90AF900C9438226C2FCD
:10B3100070E080E090E01F921F921F922FEF2F931A
:10B3200026E4A22EB12CC12CD12CE12CF12C8701CA
:10B33000EA9421E030E040E050E00E943E150F909A
:10B340000F900F900F90D4CFCF92DF92EF92FF9299
:10B350000F931F93CF93DF93CDB7DEB728970FB628
:10B36000F894DEBF0FBECDBF20911506222309F44D
:10B370004AC06A018B017C0120E030E040E450E4E7
:10B38000FC0160817181828193810E94D9AB6D83C0
:10B390007E838F83988720E030E04EE353E4F8010A
:10B3A00060817181828193810E94D8AB69837A83A5
:10B3B0008B839C839601AE014F5F5F4FBE016B5F35
:10B3C0007F4F81EF95E00E94AAA420E030E040E4A6
:10B3D00050E46D817E818F8198850E94D8ABF70102
:10B3E000608371838283938320E030E04EE353E4F3
:10B3F00069817A818B819C810E94D9ABF80160833D
:10B4000071838283938328960FB6F894DEBF0FBEB4
:10B41000CDBFDF91CF911F910F91FF90EF90DF9003
:10B42000CF9008950F931F93CF93DF93CDB7DEB7DF
:10B43000AC970FB6F894DEBF0FBECDBF20911506B6
:10B44000222309F450C08C0161EF75E0CE01019612
:10B450000E942DA620E030E040E450E4F801608135
:10B460007181828193810E94D9AB69A77AA78BA74A
:10B470009CA720E030E04EE353E4F801648175813D
:10B48000868197810E94D8AB6DA37EA38FA398A7D6
:10B490009801285F3F4FAE014B5D5F4FBE01675D76
:10B4A0007F4FCE0101960E94AAA420E030E040E444
:10B4B00050E469A57AA58BA59CA50E94D8ABF8019C
:10B4C000608371838283938320E030E04EE353E412
:10B4D0006DA17EA18FA198A50E94D9ABF8016483CC
:10B4E000758386839783AC960FB6F894DEBF0FBE44
:10B4F000CDBFDF91CF911F910F91089580916F0083
:10B5000081FB992790F981FF05C080916F008D7FA5
:10B5100080936F00809191068093940680939206A9
:10B520008093930684E680938E0628EE33E0309372
:10B53000900620938F06992329F080916F008260F6
:10B5400080936F0081E08093560508950C94643BCE
:10B55000CF93C82F0E948D3B0E9454AD24E0C29F20
:10B56000F0011124EA5DF94F20813181428153813C
:10B570000E94F0AECF91089590919406809191062B
:10B58000981719F00E9440ABF7CF80918F069091E9
:10B590009006892BB9F70C9417AACF93C82F0E9455
:10B5A000463B0E9454AD24E0C29FF0011124EA5DA5
:10B5B000F94F20813181428153810E94F0AECF91B9
:10B5C00008959091940680919106981719F00E9421
:10B5D00040ABF7CF80918F0690919006892BB9F7F9
:10B5E00008952F923F924F925F926F927F928F9227
:10B5F0009F92AF92BF92CF92DF92EF92FF920F9302
:10B600001F93CF93DF93CDB7DEB766970FB6F8944D
:10B61000DEBF0FBECDBFB88AAF86E091A305DC2C9C
:10B62000DE26672B682B692B19F48D2D8E7FD82E83
:10B63000232B242B252B19F49D2D9D7FD92EEF280C
:10B64000E02AE12A19F4AD2DAB7FDA2E8D2D8E275D
:10B650008093A30580913A0C90913B0CA0913C0CF7
:10B66000B0913D0C8D839E83AF83B88720E030E09E
:10B67000A901BC01CD010E94B2AC882309F424C108
:10B680008091670290916802A0916902B0916A026C
:10B6900089879A87AB87BC87AEE3BCE0BE87AD875E
:10B6A000EF85F889FA83E98387E995E09E8B8D8B96
:10B6B000A6E4B6E0BC83AB83212C312C812C912CE9
:10B6C0005401EC2DF0E0FA8BE98B8D2D90E09C8BF2
:10B6D0008B8BAD85BE85CD90DD90ED90FD90BE87C6
:10B6E000AD8720E030E0A901C701B6010E94B2ACED
:10B6F000882309F4D2C009891A89022C02C0159541
:10B7000007950A94E2F7017011278B899C89022C16
:10B7100002C0959587950A94E2F780FF38C0ED89BD
:10B72000FE8960817181828193810E9454AD2B01D9
:10B730003C010115110529F420E030E040E85FE309
:10B7400004C020E030E040E85FEB6D817E818F81B6
:10B7500098850E94F0AEA70196010E94F0AEAB81E1
:10B76000BC8154962D913D914D915C9157970E94CB
:10B77000F0AE9B01AC01C301B2010E94D9AB0E94A3
:10B7800021ADED89FE896083718382839383AD89C6
:10B79000BE89CD90DD90ED90FC90C114D104E10400
:10B7A000F10409F47AC020E030E0A90169857A85C6
:10B7B0008B859C850E94B2AC882309F445C0D701D3
:10B7C000C6018827B7FD83959927AA27BB270817A5
:10B7D000190709F062C020E030E0A901C501B401F9
:10B7E0000E94B2AC81111CC029853A854B855C85CD
:10B7F000EF85F88965857685878590890E94B9AC43
:10B800004B015C0120E030E040E85FE30E94B5AE10
:10B81000181634F4812C912C80E8A82E8FE3B82ED2
:10B82000C701B6010E9454AD9B01AC01C501B40132
:10B830000E94F0AE0E949FAC0E9421AD611571057F
:10B840008105910519F429C0C701B6018B019C013E
:10B8500097FF07C0002711279801061B170B280B1D
:10B86000390BA981BA8155964D905D906D907C9071
:10B870005897040D151D261D371DFD01058B168BD0
:10B88000278B308FC61AD70AE80AF90AAD89BE8914
:10B89000CD92DD92ED92FC921397BFEF2B1A3B0AEB
:10B8A000E981FA813496FA83E9838D899E89049629
:10B8B0009E8B8D8BAB81BC811496BC83AB83B3E034
:10B8C0002B16310409F005CF66960FB6F894DEBF4B
:10B8D0000FBECDBFDF91CF911F910F91FF90EF90E1
:10B8E000DF90CF90BF90AF909F908F907F906F90A0
:10B8F0005F904F903F902F9008952F923F924F92DC
:10B900005F926F927F928F929F92AF92BF92CF92EF
:10B91000DF92EF92FF920F931F93CF93DF93CDB7F8
:10B92000DEB7C756D1090FB6F894DEBF0FBECDBF44
:10B930001C01A4966FAFA4976F965FAF4EAF6F9741
:10B9400069963FAF2EAF69972896EFAE2897FFAE66
:10B9500060960FAF609764961FAF6497CFAAA196C9
:10B96000BFAEAEAEA197DA014D915D916D917C9124
:10B970008091D5059091D605A091D705B091D805B5
:10B980008A019B01081B190B2A0B3B0B0BA31CA361
:10B990002DA33EA36F96AEADBFAD6F9714964D919C
:10B9A0005D916D917C9117978091D9059091DA0501
:10B9B000A091DB05B091DC058A019B01081B190BE6
:10B9C0002A0B3B0B0FA318A729A73AA76F96AEAD7A
:10B9D000BFAD6F9718964D915D916D917C911B97BE
:10B9E0008091DD059091DE05A091DF05B091E00525
:10B9F0008A019B01081B190B2A0B3B0B0FA718ABE5
:10BA000029AB3AAB6F96AEADBFAD6F971C96CD909C
:10BA1000DD90ED90FC901F978091E1059091E205FB
:10BA2000A091E305B091E40526013701481A590AAF
:10BA30006A0A7B0A09F497C06091CC047091CD0426
:10BA40008091CE049091CF042091A10421112AC0AD
:10BA50000E9421AD20911D0230911E0262177307D2
:10BA60000CF5C092E105D092E205E092E305F09278
:10BA7000E4056996EEADFFAD699784859585A68549
:10BA8000B7858093B4059093B505A093B605B093A0
:10BA9000B7050E94F31584E994E10E94E515412C55
:10BAA000512C3201C301B2010E9454AD1FA904E020
:10BAB000109FF0011124E05AFD4F20813181428115
:10BAC00053810E94F0AE6B017C0120E030E0A901BF
:10BAD0000E94B5AE87FF04C0F7FAF094F7F8F0942F
:10BAE000609166067091670680916806909169067C
:10BAF0000E9421AD9B01AC01A8ECB0E00E9438B0DF
:10BB00000E9454AD9B01AC01C701B6010E94B5AEC5
:10BB100018164CF56F96EEADFFAD6F978485958541
:10BB2000A685B7858093E1059093E205A093E30590
:10BB3000B093E4056996EEADFFAD69978485958570
:10BB4000A685B7858093B4059093B505A093B605F7
:10BB5000B093B7050E94F31585E794E10E94E515BF
:10BB6000412C512C32018BA19CA1ADA1BEA18827F3
:10BB7000B7FD83959927AA27BB27182F2FA138A592
:10BB800049A55AA557FD12608FA598A9A9A9BAA9D8
:10BB9000B7FD146077FC1860C301B2010E9454AD78
:10BBA000BFA9A4E0BA9FF0011124E05AFD4F208103
:10BBB0003181428153810E94F0AE4B015C0120E053
:10BBC00030E0A9010E94B5AE87FF04C0C501B401F1
:10BBD000905802C0C501B40120E030E040E05FE3CE
:10BBE0000E94D9AB0E9426AD6BAF7CAF8DAF9EAFEC
:10BBF000F101108215AB2BA13CA14DA15EA12BA799
:10BC00003CA74DA75EA757FF0BC0509540953095B8
:10BC100021953F4F4F4F5F4F2BA73CA74DA75EA7E6
:10BC20008BA59CA5ADA5BEA5F101858B968BA78B99
:10BC3000B08F2FA138A549A55AA52BAB3CAB4DAB76
:10BC40005EAB57FF0BC050954095309521953F4F07
:10BC50004F4F5F4F2BAB3CAB4DAB5EAB8BA99CA961
:10BC6000ADA9BEA9F101818F928FA38FB48F2FA5AB
:10BC700038A949A95AA92F962CAF3DAF4EAF5FAF57
:10BC80002F9757FF0DC050954095309521953F4F08
:10BC90004F4F5F4F2F962CAF3DAF4EAF5FAF2F97FB
:10BCA0002F968CAD9DADAEADBFAD2F97F101858FB9
:10BCB000968FA78FB0A36BA17CA18DA19EA10E949E
:10BCC00054AD2091260630912706409128065091C8
:10BCD00029060E94F0AE27966CAF7DAF8EAF9FAF66
:10BCE0002797698B7A8B8B8B9C8B6FA178A589A505
:10BCF0009AA50E9454AD20912A0630912B064091BE
:10BD00002C0650912D060E94F0AE6B017C016D8BCC
:10BD10007E8B8F8B988F6FA578A989A99AA90E948D
:10BD200054AD20912E0630912F064091300650914F
:10BD300031060E94F0AE6D966CAF7DAF8EAF9FAFB7
:10BD40006D97698F7A8F8B8F9C8F209132063091FF
:10BD500033064091340650913506C501B4010E9466
:10BD6000F0AE4B015C016D8F7E8F8F8F98A32BA55A
:10BD70003CA54DA55EA5263031054105510544F58C
:10BD80008BA99CA9ADA9BEA90697A105B10504F58B
:10BD90002F962CAD3DAD4EAD5FAD2F9726303105C2
:10BDA00041055105ACF420E030E0A901C501B40122
:10BDB0000E94B5AE87FF04C0B7FAB094B7F8B0944C
:10BDC000D1011D968D929D92AD92BC92509759C013
:10BDD000A196EEADFFADA19780809180A280B38047
:10BDE00020E030E0A901C501B4010E94B2AC882373
:10BDF00041F0D1011D968D929D92AD92BC925097CB
:10BE000031C027962CAD3DAD4EAD5FAD2797CA0131
:10BE1000B9010E94F0AE4B015C01A7019601C70178
:10BE2000B6010E94F0AE9B01AC01C501B4010E94B5
:10BE3000D9AB4B015C016D962CAD3DAD4EAD5FAD08
:10BE40006D97CA01B9010E94F0AE9B01AC01C5011A
:10BE5000B4010E94D9AB0E945DAFF101658776877E
:10BE60008787908B5101C12EEFA4F8A809A91AA9C0
:10BE70002FA138A549A55AA56BA17CA18DA19EA192
:10BE8000B0DB0BAD1CAD2DAD3EADD10191960D9348
:10BE90001D932D933C93949755964D915D916D9183
:10BEA0007C9158975D960D911D912D913C919097A5
:10BEB00059968D919D910D90BC91A02D8017910761
:10BEC000A207B30710F4D901C80184179507A60784
:10BED000B70710F4DB01CA010BAD1CAD2DAD3EADB3
:10BEE00080179107A207B30710F4D901C801F10127
:10BEF00085A396A3A7A3B0A70697A105B105A8F1AE
:10BF00008091C704EF5AFF4F8083452B462B472B68
:10BF100009F01798F101818D928DA38DB48D892B35
:10BF20008A2B8B2B09F01698F101858D968DA78DA4
:10BF3000B0A1892B8A2B8B2B09F015980BAD1CAD6A
:10BF40002DAD3EAD012B022B032BD1F08091BC0512
:10BF5000882319F081508093BC051FA9111107C0D7
:10BF6000149880E28093BC0502C080E0FEC7E09098
:10BF70008606F0908706009188061091890608C011
:10BF8000E0908A06F0908B0600918C0610918D0649
:10BF90009701A80128966FAD28977FAD60968FAD69
:10BFA000609764969FAD64970E94B2AC87FFD2C73A
:10BFB000D1011D962D913D914D915C9150976D96BB
:10BFC0002CAF3DAF4EAF5FAF6D9760E070E080E8A3
:10BFD0009FE30E94B9AC2B966CAF7DAF8EAF9FAF45
:10BFE0002B979B01AC01B701C8010E94F0AE4B0139
:10BFF0005C018091940690919306891B8F70249622
:10C000008FAF2497A501940160E074E284E799E47E
:10C010000E94B9AC0E94C0AE6B017C0124968FAD2A
:10C02000249782508630C0F580915606909157062D
:10C03000A0915806B0915906C816D906EA06FB0623
:10C0400058F58C199D09AE09BF09BC01CD01660FD9
:10C05000771F881F991F2496BFAD24970B2F10E0E0
:10C0600020E030E0A90198010E94DDAFCA01B901CA
:10C070000E9452AD0E94C0AE6C0D7D1D8E1D9F1D95
:10C080000E9452AD9B01AC0160E074E284E799E448
:10C090000E94B9AC4B015C01A50194016D966CAD99
:10C0A0007DAD8EAD9FAD6D970E94F0AE9B01AC0152
:10C0B0000E94F0AE23966CAF7DAF8EAF9FAF2397FB
:10C0C000F101618372838383948305A116A127A163
:10C0D00030A50FA718AB29AB3AABC901B8010E9434
:10C0E00052AD6FAB78AF89AF9AAFA50194010E94B2
:10C0F000F0AE0E949FAC0E9426AD63966CAF7DAF00
:10C100008EAF9FAF6397F101EF5BFF4F6083718349
:10C11000828393838E010F5E1F4F1CA70BA70051D4
:10C1200011092D961FAF0EAF2D970AE616E0A196C6
:10C130001FAF0EAFA1978E010F5D1F4F1AA309A36A
:10C140002D960EAD1FAD2D971CAB0BAB1BA21FA2E6
:10C1500000E81FE3ABA5BCA56D917D918D919D91EC
:10C16000BCA7ABA7A50194010E94F0AE6B017C01B6
:10C17000EBA9FCA96193719381939193FCABEBAB19
:10C1800020E030E0A9010E94B5AE87FF04C0F7FAB5
:10C19000F094F7F8F094A196AEADBFADA1972D91B4
:10C1A0003D914D915D91A196BFAFAEAFA1976796BE
:10C1B0002CAF3DAF4EAF5FAF6797C701B6010E948E
:10C1C000B5AE1816C4F4A701960167966CAD7DADA7
:10C1D0008EAD9FAD67970E94B9AC6B017C019B014E
:10C1E000AC016BA17FA1C8010E94B5AE18161CF46A
:10C1F000CBA2DFA28701EBA5FCA529A13AA1E217FA
:10C20000F30709F0A7CF20E030E040E85FE36BA13F
:10C210007FA1C8010E94B2AC87FF4BC06E0131E123
:10C22000C30ED11C2D96EEACFFAC2D972BA13FA1D8
:10C23000A801D7016D917D918D919C910E94F0AEE6
:10C24000F70161937193819391937F01EC15FD0543
:10C2500069F77101F1E4EF0EF11C63966CAD7DADF1
:10C260008EAD9FAD63970E9452AD2BA13FA1A80157
:10C270000E94F0AE0E9426ADD7016D937D938D9301
:10C280009C9313972BA13FA1A8016BA17FA1C8018B
:10C290000E94F0AE9B01AC0123966CAD7DAD8EADDE
:10C2A0009FAD23970E94F0AEF10161837283838377
:10C2B00094832B962CAD3DAD4EAD5FAD2B976FA902
:10C2C00078AD89AD9AAD0E94F0AE6BAB7CAB8DAB17
:10C2D0009EABD10155960D911D912D913C91589792
:10C2E0000BA31CA32DA33EA35D960D911D912D9133
:10C2F0003C9190970FA318A729A73AA759960D919B
:10C300001D912D913C915C970BA71CA72DA73EA7D3
:10C310000BA11CA12DA13EA1012B022B032B41F54A
:10C320002BA53CA54DA55EA5232B242B252B01F584
:10C330008FA198A5A9A5BAA5892B8A2B8B2BC1F40F
:10C3400020917E0630917F064091800650918106B3
:10C350006BA97CA98DA99EA90E94F0AE0E949FACFA
:10C360000E9426AD4B015C01D101D6961C92F0C211
:10C370000BAD1CAD2DAD3EAD012B022B032B49F0B7
:10C3800060917A0670917B0680917C0690917D0683
:10C3900008C0609182067091830680918406909116
:10C3A00085062BA93CA94DA95EA90E94F0AE0E946A
:10C3B0009FAC0E9426AD4B015C012BAD3CAD4DAD59
:10C3C0005EAD232B242B252BA9F020E030E0A90122
:10C3D0006091B8057091B9058091BA059091BB053F
:10C3E0000E94B2AC882331F081E0141415041604C5
:10C3F00017040CF080E0D101D6968C93882309F4C1
:10C40000BAC02091A8053091A9054091AA05509184
:10C41000AB056996EEADFFAD699760817181828150
:10C4200093810E94D8AB2B013C012091AC05309147
:10C43000AD054091AE055091AF056996AEADBFAD6B
:10C44000699714966D917D918D919C9117970E949B
:10C45000D8AB6BAF7CAF8DAF9EAF2091B005309164
:10C46000B1054091B2055091B3056996EEADFFADAF
:10C47000699760857185828593850E94D8AB6B0131
:10C480007C01A3019201C301B2010E94F0AE2B0115
:10C490003C012BAD3CAD4DAD5EADCA01B9010E9472
:10C4A000F0AE9B01AC01C301B2010E94D9AB2B01DC
:10C4B0003C01A7019601C701B6010E94F0AE9B01A5
:10C4C000AC01C301B2010E94D9AB0E945DAF6B0108
:10C4D0007C012091B4053091B5054091B60550918D
:10C4E000B7056996AEADBFAD69971C966D917D910C
:10C4F0008D919C911F970E94D8ABA70196010E9435
:10C50000B9AC6B017C01F101FD966083718382837C
:10C51000938320E030E040E450E40E94B5AE18166A
:10C520001CF4F10116AA27C02091B8053091B90575
:10C530004091BA055091BB05C701B6010E94F0AE0B
:10C540009B01AC0160912206709123068091240624
:10C55000909125060E94B9AC2BA93CA94DA95EA9D2
:10C560000E94F0AE0E9426AD681579058A059B05EC
:10C5700010F44B015C018091D1059091D205A091FE
:10C58000D305B091D405F10141A052A063A074A0DD
:10C590000FA518A929A93AA980179107A207B307DF
:10C5A00008F4CDC02BA13CA14DA15EA1232B242BCF
:10C5B000252B61F1209136063091370640913806DF
:10C5C00050913906281539054A055B05F8F46FA521
:10C5D00078A989A99AA90E94BAAF6B017C01A5012B
:10C5E00094016BA17CA18DA19EA10E94BAAFC61639
:10C5F000D706E806F90650F4C701B6012BA13CA105
:10C600004DA15EA10E94DDAF49015A018BA59CA5F9
:10C61000ADA5BEA5892B8A2B8B2B61F120913A0603
:10C6200030913B0640913C0650913D062815390556
:10C630004A055B05F8F46FA578A989A99AA90E9413
:10C64000BAAF6B017C01A50194016BA57CA58DA5FA
:10C650009EA50E94BAAFC616D706E806F90650F4A2
:10C66000C701B6012BA53CA54DA55EA50E94DDAF77
:10C6700049015A010FA118A529A53AA5012B022BA2
:10C68000032B61F120913E0630913F064091400618
:10C6900050914106281539054A055B05F8F46FA548
:10C6A00078A989A99AA90E94BAAF6B017C01A5015A
:10C6B00094016FA178A589A59AA50E94BAAFC61664
:10C6C000D706E806F90650F4C701B6012FA138A530
:10C6D00049A55AA50E94DDAF49015A0141145104F0
:10C6E0006104710409F434C120914206309143067B
:10C6F0004091440650914506281539054A055B05C9
:10C7000008F026C16FA578A989A99AA90E94BAAF95
:10C710006B017C01A5019401C301B2010E94BAAF73
:10C72000C616D706E806F90608F012C1C701B60119
:10C73000A30192010E94DDAF49015A0109C12BA159
:10C740003CA14DA15EA1232B242B252BE9F1609167
:10C750003606709137068091380690913906681533
:10C7600079058A059B0580F50E9452AD2FA938AD49
:10C7700049AD5AAD0E94F0AE6B017C016BA17CA16A
:10C780008DA19EA10E9452AD6BA37CA38DA39EA3FD
:10C79000C501B4010E9452AD2BA13CA14DA15EA1E7
:10C7A0000E94F0AEA70196010E94B5AE181664F47F
:10C7B0002BA13CA14DA15EA1C701B6010E94B9AC5D
:10C7C0000E9426AD4B015C018BA59CA5ADA5BEA525
:10C7D000892B8A2B8B2BE9F160913A0670913B06ED
:10C7E00080913C0690913D06681579058A059B0568
:10C7F00080F50E9452AD2FA938AD49AD5AAD0E94C7
:10C80000F0AE6B017C016BA57CA58DA59EA50E9459
:10C8100052AD6BA37CA38DA39EA3C501B4010E945E
:10C8200052AD2BA13CA14DA15EA10E94F0AEA7018B
:10C8300096010E94B5AE181664F42BA13CA14DA13F
:10C840005EA1C701B6010E94B9AC0E9426AD4B01A2
:10C850005C010FA118A529A53AA5012B022B032BDA
:10C86000E9F160913E0670913F06809140069091FB
:10C870004106681579058A059B0580F50E9452AD31
:10C880002FA938AD49AD5AAD0E94F0AE6B017C01C5
:10C890006FA178A589A59AA50E9452AD6BA37CA330
:10C8A0008DA39EA3C501B4010E9452AD2BA13CA152
:10C8B0004DA15EA10E94F0AEA70196010E94B5AE07
:10C8C000181664F42BA13CA14DA15EA1C701B601CD
:10C8D0000E94B9AC0E9426AD4B015C014114510489
:10C8E00061047104A9F16091420670914306809140
:10C8F000440690914506681579058A059B0540F523
:10C900000E9452AD2FA938AD49AD5AAD0E94F0AE8C
:10C910006B017C01C301B2010E9452AD2B013C01AD
:10C92000C501B4010E9452ADA30192010E94F0AE74
:10C93000A70196010E94B5AE181654F4A301920106
:10C94000C701B6010E94B9AC0E9426AD4B015C0143
:10C95000F101E35BFF4F80829182A282B382C50125
:10C96000B4010E9452AD6B017C012BA93CA94DA9D9
:10C970005EA90E94B9AC2B966CAF7DAF8EAF9FAF16
:10C980002B97D10151966D937D938D939C935497E2
:10C990002DEB37E346E051E4C701B6010E94F0AE4B
:10C9A0000E9426ADF10161AB72AB83AB94AB86A95B
:10C9B000882381F1FD9620813181428153816091EC
:10C9C000B8057091B9058091BA059091BB050E9498
:10C9D000F0AE2B962CAD3DAD4EAD5FAD2B970E94CA
:10C9E000F0AE20916606309167064091680650913E
:10C9F00069060E94F0AE9B01AC0160E074E284EF36
:10CA000099E40E94B9AC0E9426ADD101D8967C93DE
:10CA10006E93D797D10111960D911D912D913C9157
:10CA2000149763960CAF1DAF2EAF3FAF6397C9014C
:10CA3000B8010E945DAF6FA77BAF8FAB9BA706E1EC
:10CA400016E065961FAF0EAF65973E0111E1610ECE
:10CA5000711C06E116E021961FAF0EAF21972D96AF
:10CA60004EAC5FAC2D976BA37FA3182F092F1BAA89
:10CA7000D201CD90DD90ED90FD902D0120E030E0D1
:10CA8000A901C701B6010E94B5AE87FF04C0F7FA3D
:10CA9000F094F7F8F0942196EEADFFAD21978190D8
:10CAA0009190A190B1902196FFAFEEAF2197A50193
:10CAB0009401C701B6010E94B5AE18160CF03FC034
:10CAC000FBA9FF2329F1A50194016FA57BAD8FA9D7
:10CAD0009BA50E94F0AE4B015C012BA13FA1412F11
:10CAE000502FC701B6010E94F0AEA50194010E942B
:10CAF000B5AE181614F5A7019601C501B4010E9440
:10CB0000B9AC6BA37FA3182F092F21E02BAB17C063
:10CB1000A7019601C501B4010E94B9AC9B01AC010B
:10CB20006BA17FA1812F902F0E94F0AE6BA37FA3FA
:10CB3000182F092F31E03BAB02C041E04BAB46144C
:10CB4000570409F095CF5BA1A5965FAFA5978FA17C
:10CB5000A6968FAFA697A7961FAFA797A8960FAFD9
:10CB6000A89724969FAD2497992309F44CC1C090AF
:10CB7000BD05D090BE05E090BF05F090C0052DEB3F
:10CB800037E346E855E3C701B6010E94B2AC87FD22
:10CB90003AC1C701B6010E945DAF6B017C019B01E8
:10CBA000AC016FA57BAD8FA99BA50E94B2AC87FDA0
:10CBB00004C0CFA6DBAEEFAAFBA69601A7016FA526
:10CBC0007BAD8FA99BA50E94B9ACA3966CAF7DAF3E
:10CBD0008EAF9FAFA397A1ECB5E02196BFAFAEAFEC
:10CBE000219720E030E040E85FE32BAB3CAB4DAB5E
:10CBF0005EAB24961FAE24972196AEADBFAD2197B4
:10CC00006D917D918D919D912196BFAFAEAF219792
:10CC1000A3962CAD3DAD4EAD5FADA3970E94F0AE97
:10CC20006B017C012D96EEADFFAD2D97819091901B
:10CC3000A190B1902D96FFAFEEAF2D972496FFAD4A
:10CC40002497FF2391F02BA93CA94DA95EA90E942E
:10CC5000F0AE6B017C012BA93CA94DA95EA9C501D1
:10CC6000B4010E94F0AE4B015C01A5019401C70123
:10CC7000B6010E94B5AE20E030E0A90118164CF5CF
:10CC8000C501B4010E94B5AE18164CF020E030E0AA
:10CC9000A901C701B6010E94B2AC87FF09C0A50176
:10CCA0009401C701B6010E94D8AB2B013C0139C0E9
:10CCB0002401350177FA709477F87094A3019201FA
:10CCC000C701B6010E94B5AE18165CF52601370102
:10CCD00028C0C501B4010E94B2AC87FD09C020E0A4
:10CCE00030E0A901C701B6010E94B5AE18164CF498
:10CCF000A7019601C501B4010E94D8AB2B013C01EC
:10CD000010C02601370177FA709477F87094A50166
:10CD10009401C301B2010E94B5AE181614F02401AB
:10CD200035016596AEADBFAD6597CD90DD90ED90C8
:10CD3000FD906596BFAFAEAF6597A7019601C301A1
:10CD4000B2010E94B5AE1816CCF4A3019201C7013E
:10CD5000B6010E94B9AC9B01AC016BA97CA98DA95D
:10CD60009EA90E94F0AE6BAB7CAB8DAB9EAB2496C4
:10CD7000BFAD2497BF5F2496BFAF24972196EEAD39
:10CD8000FFAD2197E15DF54009F036CF24963FAD28
:10CD90002497332371F02BA93CA94DA95EA96FA557
:10CDA0007BAD8FA99BA50E94F0AE6FA77BAF8FAB29
:10CDB0009BA724EA30E74DE75FE36FA57BAD8FA922
:10CDC0009BA50E94F0AE6B017C019B01AC016091C0
:10CDD00093057091940580919505909196050E9418
:10CDE000B5AE181654F4A70196016BA17FA1812F4F
:10CDF000902F0E94B5AE181634F00FA50BA31BADF3
:10CE00001FA31FA90BA5A5968FADA597A6969FADAD
:10CE1000A697A796AFADA797A896BFADA897809302
:10CE2000930590939405A0939505B09396052BA137
:10CE30003FA1412F502F6BA17FA1812F902F0E94E6
:10CE4000F0AE7B018C01CB01D801F1018187928783
:10CE5000A387B4872B966CAD7DAD8EAD9FAD2B9720
:10CE600090589B01AC010E94D9AB6D962CAD3DADA5
:10CE70004EAD5FAD6D970E94F0AE9B01AC016BE0D3
:10CE800077ED83E29BE30E94D8AB5B016C01A49633
:10CE9000FFADA497FF2361F09B01AC01B701C8016E
:10CEA0000E94B2AC87FD09C09A2D8B2D860107C068
:10CEB0009BE087ED03E21BE302C09E2D8F2D492FDF
:10CEC000582FB801D10115964D935D936D937C93C6
:10CED00018971C919501A60163966CAD7DAD8EAD42
:10CEE0009FAD63970E94B2AC181614F481E001C0A4
:10CEF00083E0182BF101108380E1FE013196A1EC53
:10CF0000B5E001900D928A95E1F7F101818192815E
:10CF1000A381B4818093BD059093BE05A093BF0506
:10CF2000B093C00580E16F96EEADFFAD6F97A5EDB4
:10CF3000B5E001900D928A95E1F780E16996EEAD3A
:10CF4000FFAD6997A8EAB5E001900D928A95E1F7E7
:10CF500081E00BC02896EFAC2897FFAC60960FAD30
:10CF6000609764961FAD649723C8C959DF4F0FB609
:10CF7000F894DEBF0FBECDBFDF91CF911F910F910F
:10CF8000FF90EF90DF90CF90BF90AF909F908F90E9
:10CF90007F906F905F904F903F902F9008956F9289
:10CFA0007F928F929F92AF92BF92CF92DF92EF9239
:10CFB000FF920F931F93CF93DF9300D01F92CDB7B3
:10CFC000DEB74C013B0180918F0690919006892B32
:10CFD000D9F59091940680919106981B9F709F308F
:10CFE00059F429833A834B835C830E9440AB5C8174
:10CFF0004B813A812981EDCFD0909406809194069F
:10D0000066E5869FC00111245701C02E79018A016F
:10D010009301A40160E08B56994F0E947D5C8823A8
:10D02000A9F02091940690919106291303C094E6EB
:10D0300090938E0691E09D0D9F7090939406898346
:10D040000E941759898103C080E001C081E00F90E0
:10D050000F900F900F90DF91CF911F910F91FF9044
:10D06000EF90DF90CF90BF90AF909F908F907F9088
:10D070006F9008958091940690919106891B8F700E
:10D080008F3019F40E9440ABF5CF809194068F5FEA
:10D090008F70E091940696E59E9FF0011124EB5667
:10D0A000F94FDF011D929A95E9F798E0908340913E
:10D0B000D5055091D6056091D7057091D805458B5F
:10D0C000568B678B708F4091D9055091DA0560912E
:10D0D000DB057091DC05418F528F638F748F409117
:10D0E000DD055091DE056091DF057091E005458F0B
:10D0F000568F678F70A34091E1055091E2056091D2
:10D10000E3057091E40541A352A363A374A32091A6
:10D11000940690919106291303C094E690938E068D
:10D12000809394060C9419322F923F924F925F9203
:10D130006F927F928F929F92AF92BF92CF92DF9227
:10D14000EF92FF920F931F93CF93DF93CDB7DEB78C
:10D15000A9970FB6F894DEBF0FBECDBFF801A0911E
:10D160008F06B0919006AB2B09F0A7C016010E2DCB
:10D17000F8A7EFA33EA32DA36A017B01FC01408029
:10D1800051806280738020915A0630915B064091F5
:10D190005C0650915D06C301B2010E94F0AE0E9490
:10D1A000C0AE698B7A8B8B8B9C8BD7018D909D90B9
:10D1B000AD90BC9020915E0630915F064091600674
:10D1C00050916106C501B4010E94F0AE0E94C0AE4C
:10D1D0006D8B7E8B8F8B988FD6012D913D914D91CC
:10D1E0005C9129A33AA34BA35CA3209162063091E2
:10D1F0006306409164065091650669A17AA18BA1EE
:10D200009CA10E94F0AE0E94C0AE698F7A8F8B8F76
:10D210009C8FEDA1FEA1C080D180E280F38020919F
:10D220006606309167064091680650916906C7010D
:10D23000B6010E94F0AE0E94C0AE6D8F7E8F8F8FC0
:10D2400098A349825A826B827C828D829E82AF82B1
:10D25000B88629A13AA14BA15CA129873A874B87BF
:10D260005C87CD86DE86EF86F88A2091A90323FFAE
:10D2700010C06093E1057093E2058093E3059093FD
:10D28000E405C092B405D092B505E092B605F092DF
:10D29000B705AFA1B8A52D913D914D915C9171015C
:10D2A000BE016F5F7F4FCE01419679DE882331F05A
:10D2B00089A70E94193289A501C080E0A9960FB6FE
:10D2C000F894DEBF0FBECDBFDF91CF911F910F91BC
:10D2D000FF90EF90DF90CF90BF90AF909F908F9096
:10D2E0007F906F905F904F903F902F900895AF92F6
:10D2F000BF92CF92DF92EF920F931F93CF93DF9362
:10D30000CDB7DEB764970FB6F894DEBF0FBECDBFC2
:10D31000A98ABA8ACB8ADC8AFC0180819181A281A8
:10D32000B38189839A83AB83BC83FB018081918124
:10D33000A281B3818D839E83AF83B887FA018081F8
:10D340009181A281B38189879A87AB87BC87F901D4
:10D3500080819181A281B3818D879E87AF87B88BB1
:10D36000AE01475F5F4FBE016B5F7F4FCE010196FD
:10D370000E94A459CE0141966C019E01235F3F4F4C
:10D38000AE01475F5F4FBE016B5F7F4F4097CCDEC2
:10D3900064960FB6F894DEBF0FBECDBFDF91CF917C
:10D3A0001F910F91EF90DF90CF90BF90AF900895B5
:10D3B0008F929F92AF92BF92EF92FF920F931F9323
:10D3C000CF93DF937B018A01E901FC01808091808A
:10D3D000A280B38020915A0630915B0640915C0692
:10D3E00050915D06C501B4010E94F0AE0E94C0AE2E
:10D3F0006093D5057093D6058093D7059093D80593
:10D4000020915E0630915F06409160065091610662
:10D41000F70160817181828193810E94F0AE0E9448
:10D42000C0AE6093D9057093DA058093DB059093C5
:10D43000DC052091620630916306409164065091AC
:10D440006506F80160817181828193810E94F0AE4E
:10D450000E94C0AE6093DD057093DE058093DF050A
:10D460009093E0052091660630916706409168062A
:10D4700050916906688179818A819B810E94F0AE12
:10D480000E94C0AE6093E1057093E2058093E305CE
:10D490009093E4058092A8059092A905A092AA0510
:10D4A000B092AB05F70180819181A281B381809315
:10D4B000AC059093AD05A093AE05B093AF05F80110
:10D4C00080819181A281B3818093B0059093B10551
:10D4D000A093B205B093B30588819981AA81BB81DD
:10D4E0008093B4059093B505A093B605B093B705A6
:10D4F0009091940680919106981759F0DF91CF9101
:10D500001F910F91FF90EF90BF90AF909F908F90E1
:10D51000B1CD0E94E15A80916F0081FBCC27C0F908
:10D5200081FF05C080916F008D7F80936F0021EE99
:10D5300035E04DED55E069ED75E085ED95E00E9433
:10D540004935CC2329F080916F00826080936F0071
:10D55000DF91CF911F910F91FF90EF90BF90AF900F
:10D560009F908F900895CF93DF93CDB7DEB76097EC
:10D570000FB6F894DEBF0FBECDBFFC018081918154
:10D58000A281B38189839A83AB83BC83FB018081B1
:10D590009181A281B3818D839E83AF83B887FA0185
:10D5A00080819181A281B38189879A87AB87BC876B
:10D5B000F90180819181A281B3818D879E87AF8798
:10D5C000B88BAE01475F5F4FBE016B5F7F4FCE01EF
:10D5D00001960E94A4599E01235F3F4FAE01475F11
:10D5E0005F4FBE016B5F7F4FCE010196E1DE60961B
:10D5F0000FB6F894DEBF0FBECDBFDF91CF91089577
:10D60000CF92DF92EF92FF92FC01C080D180E28046
:10D61000F38020916606309167064091680650912C
:10D620006906C701B6010E94F0AE0E94C0AE6093C9
:10D63000E1057093E2058093E3059093E405C092C1
:10D64000B405D092B505E092B605F092B705909179
:10D65000940680919106981729F0FF90EF90DF9043
:10D66000CF9008CD0E94E15A80916F0081FB9927ED
:10D6700090F981FF05C080916F008D7F80936F00CE
:10D680004091E1055091E2056091E3057091E40558
:10D690004093F9045093FA046093FB047093FC04E4
:10D6A000992329F080916F00826080936F00FF9032
:10D6B000EF90DF90CF900895CF92DF92EF92FF929C
:10D6C0000F931F93CF93DF93C6E4D6E006E316E0F3
:10D6D000C12CD12C7601C39469917991899199914A
:10D6E0000E9452AD288939894A895B890E94F0AE2F
:10D6F0000E9426ADF80161937193819391938F01FC
:10D70000C616D706E806F90610F46B017C01F6E0B0
:10D71000C635DF0709F76FEF7FEFCB01A701960151
:10D720000E94DDAF2093D1053093D2054093D305FD
:10D730005093D405DF91CF911F910F91FF90EF90FF
:10D74000DF90CF9008950F931F93CF93DF930AE557
:10D7500016E0C6E2D6E0F801219131914191519154
:10D760008F0160E070E080E89FE30E94B9AC6993AC
:10D77000799389939993F6E0C633DF0761F72CE537
:10D7800032E048E552E064E572E080E592E0EBDEED
:10D79000DF91CF911F910F918FCF85EF9BE00C947C
:10D7A0001B5481548A3108F041C0A82FB0E0409149
:10D7B0001E0C50911F0C6091200C7091210C04C024
:10D7C00076956795579547958A95D2F740FF2EC075
:10D7D000E091290CF0912A0CAC5FB34F8C91882317
:10D7E000E9F0E80FF11D808190ED980F9A3098F0E4
:10D7F0008E3211F481810CC08D3211F08B3271F4B4
:10D80000818190ED980F9A3030F08E3239F4828118
:10D8100080538A3018F49E2F8F2F02C090E080E052
:10D820009093250C8093260C81E0089580E0089564
:10D83000B8DF882341F081E02091250C3091260C3F
:10D84000232B09F480E008950F931F93CF938091C9
:10D85000250C9091260C009711F1FC018F01C191CC
:10D860002C2F2F7DA9F0C53411F0C536B9F7F8017A
:10D87000108260E070E08091250C9091260C0E944F
:10D8800042B0F801C083562F472F382F292F0BC0E5
:10D8900060E070E0CF911F910F910C9442B050E086
:10D8A00040E030E020E0652F742F832F922FCF913E
:10D8B0001F910F9108958091250C9091260C00974F
:10D8C00031F04AE050E060E070E00C94A8B160E014
:10D8D00070E0CB010895CF9384E5AADF882359F146
:10D8E000EADF97FD24C0E7DF6F3F710581059105F1
:10D8F00009F0FCF4E0DFC62F1616FCF40E94F315C5
:10D900008DE40E9475186AE070E08091220C90917D
:10D91000230C0E9468196C2FCC0F770B87E095E1E0
:10D920000E9416168AE00E9475188FEF07C0C0E0AB
:10D9300004C0CFEF02C080E001C08C2FCF910895CA
:10D94000BF92CF92DF92EF92FF920F931F93CF93EC
:10D95000DF9380E8E82E85E0F82E00E512E09BEFEB
:10D96000C92E9BE0D92ECDE4D3E0BC2E84E0B80EC6
:10D9700089915EDF8823B1F067DFF60120812111F4
:10D9800004C020919005222339F0F80120813181D3
:10D99000428153810E94D9ABF701608371838283F6
:10D9A00093830AC0F80180819181A281B381F7013C
:10D9B00080839183A283B383F4E0EF0EF11C0C5FAC
:10D9C0001F4F8FEFC81AD80ABC12D2CF86E430DFBF
:10D9D0008823B9F039DF20E030E0A9010E94B5AE1C
:10D9E00018167CF431DF20E030E040E752E40E947A
:10D9F000B9AC60934C0270934D0280934E029093A9
:10DA00004F02DF91CF911F910F91FF90EF90DF9028
:10DA1000CF90BF900895CF92DF92EF92FF926B016B
:10DA20007C010E946811C60ED71EE81EF91E0E94D6
:10DA30006811DC01CB018C199D09AE09BF09B7FF44
:10DA400003C00E9440ABF3CFFF90EF90DF90CF90E8
:10DA500008956F927F928F929F92AF92BF92CF92D2
:10DA6000DF92EF92FF920F931F93CF93DF93CDB787
:10DA7000DEB73C01A090290CB0902A0CCDB6DEB6E2
:10DA80006AE070E0C3010E9415B47C01009721F0A8
:10DA90008C010619170904C0C3010E9420B48C012F
:10DAA000C80101962DB73EB7281B390B0FB6F89465
:10DAB0003EBF0FBE2DBF8DB79EB701964C01A8018A
:10DAC000B3010E9441B4F401E00FF11F1082C401C0
:10DAD00048D581E034D0E114F10451F037019FEFD3
:10DAE000691A790A0FB6F894DEBE0FBECDBEC6CF56
:10DAF0000FB6F894DEBE0FBECDBEC501DF91CF914B
:10DB00001F910F91FF90EF90DF90CF90BF90AF905B
:10DB10009F908F907F906F9024C5CF93C3E00E9419
:10DB2000DB87882341F0C15019F00E942AAAF7CF61
:10DB3000CF910C9457AA80EF94E1CF918ACFCF93E5
:10DB4000C82F41E04093FA0B9091240C9D3409F4C6
:10DB50005EC0943509F4F7C1973409F0F8C12091FB
:10DB6000220C3091230C2B31310509F43EC0CCF44A
:10DB70002430310544F42230310564F537FDE7C126
:10DB80000E948697E7C12C30310561F125313105BE
:10DB900009F4E0C12430310509F0D9C10E948F9702
:10DBA000D9C12A35310551F154F42D31310521F116
:10DBB000FCF02E31310509F0CAC151D2CBC12C3550
:10DBC000310511F1F4F0293A314009F0C0C10E9449
:10DBD0009185C0C181E02230310509F080E00E94CA
:10DBE000B79BB8C10E949A92B5C10E949E92B2C1E1
:10DBF00080E00E948F7BAEC190DFACC11092900597
:10DC0000A9C140939005A6C10E94BB79A3C12091F0
:10DC1000220C3091230C2937310509F45DC10CF039
:10DC200083C02836310509F42AC10CF044C02C34D5
:10DC3000310509F421C104F52231310509F43EC151
:10DC400064F437FD84C1223031050CF40DC121315B
:10DC5000310509F07CC19ED77DC12A32310509F416
:10DC600005C12B34310509F404C12F31310509F008
:10DC70006EC10E9498786EC12335310509F41BC12D
:10DC80006CF42135310509F411C10CF011C12D34AA
:10DC9000310509F05CC10E94D6775CC1253531059C
:10DCA00009F40EC10CF40AC12C35310509F04FC13D
:10DCB0000E942D944FC12037310509F44BC1CCF49B
:10DCC0002C36310509F446C15CF42A36310509F4D5
:10DCD000E7C00CF0E8C00E94F7A11092FA0B41C116
:10DCE0002E36310509F4CEC00CF0CFC00E9484A1BD
:10DCF00031C12537310509F4E8C06CF4223731050C
:10DD000009F4E0C00CF4C3C02337310509F01FC18A
:10DD10000E9451791FC12737310509F4D8C00CF092
:10DD2000D9C00E94057916C12E3581E0380709F463
:10DD300008C10CF04BC0233D310509F4D8C01CF5D7
:10DD4000293C310509F4CAC07CF42B39310509F4AA
:10DD5000A4C02E3B310509F49DC02C38310509F0D3
:10DD6000F6C00E94DBA0F6C02C3C310509F4B9C016
:10DD70002D3C310509F4B8C02B3C310509F0E7C052
:10DD80000E94C795E7C02D3281E0380709F4B6C07C
:10DD90007CF42D3D310509F4ACC0223E310509F477
:10DDA000ABC02C3D310509F0D2C00E94DC93D2C03B
:10DDB0002F3281E0380709F4A7C00CF4A2C0203349
:10DDC000314009F0C4C00E946A93C4C0243F81E07E
:10DDD000380709F4A8C014F5223981E0380709F49E
:10DDE0009AC06CF4203981E0380709F490C00CF037
:10DDF00090C02F35314009F0AAC0ABD5ABC0243A52
:10DE000081E0380709F489C0293A81E0380709F42C
:10DE100087C02A39314009F09AC09CC0283F81E070
:10DE2000380709F486C04CF4263F81E0380709F42E
:10DE30007CC00CF07CC010D58DC0243883E038073E
:10DE400009F479C034F42335334009F080C040D25E
:10DE500081C02B3883E0380709F470C0273E334077
:10DE600009F075C093D776C0ACD274C00E947377A6
:10DE700071C00E94D2776EC00E94D4776BC00E949E
:10DE800061A168C00E94A17965C00AD763C00E94E1
:10DE9000C37860C00E94F4A05DC00E941AA15AC05D
:10DEA0000E94DAA157C00E94F0A154C05ED752C0B0
:10DEB0000E947F974FC00E9482974CC06DD64AC087
:10DEC00018D648C00E94017945C07AD243C00E944A
:10DED000F97840C081D73EC082D73CC00E94989557
:10DEE00039C00E94EC9536C00E94629633C07CD740
:10DEF00031C00E940F932EC0C0D52CC00E94E8965E
:10DF000029C00E94019526C00E9426A023C06AD77E
:10DF100021C09BD01FC09ED01DC00E94C1861AC0C8
:10DF20000E944A7A17C096D415C098D413C098D4CA
:10DF300011C0BBD40FC00E9419920CC00E94EA927B
:10DF400009C0D2D407C08091220C1ED603C083E042
:10DF50009CE072D41092FA0BC11103C0CF910C94C3
:10DF6000419ECF910895CF93DF93C091C50E80E677
:10DF7000C89FE0011124CC51D34F8091A90380FFA9
:10DF800005C00E94F315CE010E94CC18CE01E9D243
:10DF900080E0DF91CF91D3CDCF92DF92EF92FF92CD
:10DFA0000F931F930E9468116B017C018091E50E15
:10DFB00081112FC080916602882359F18091FA0B5C
:10DFC000882339F14091F60B5091F70B6091F80BD3
:10DFD0007091F90B97018601041B150B260B370B6B
:10DFE00037FD2CC0833079F03CF4813094F00E94EE
:10DFF000F3158EED94E10BC0843059F40E94F315B3
:10E000008FEA94E104C00E94F31587EC94E10E942A
:10E01000E5152091660230E0A8EEB3E00E9423B03F
:10E02000DC01CB018C0D9D1DAE1DBF1D8093F60B39
:10E030009093F70BA093F80BB093F90B1F910F91EE
:10E04000FF90EF90DF90CF90089581E00E94554BB4
:10E050000C94994E80E00E94554B0C94994E8F92EF
:10E060009F92AF92BF92CF92DF92EF92FF920F9367
:10E070001F93CF93DF93CDB7DEB728970FB6F894F1
:10E08000DEBF0FBECDBFC0905002D0905102E090D5
:10E090005202F090530288E5CBDB811108C020E0EA
:10E0A00030E0A901C701B6010E94D9AB01C0CCDBA9
:10E0B0006D837E838F839887C0905402D0905502E1
:10E0C000E0905602F090570289E5B2DB811108C05A
:10E0D00020E030E0A901C701B6010E94D9AB01C020
:10E0E000B3DB6B017C0169837A838B839C838D8096
:10E0F0009E80AF80B88422ED30E040EE50EC0E946C
:10E10000B5AE87FDD2C027E030E04EE353E4C7014F
:10E11000B6010E94B2AC18160CF4C7C023EA31E075
:10E1200040E450ECC501B4010E94B5AE87FDBDC00E
:10E1300027E030E042E253E4C501B4010E94B2ACF2
:10E1400018160CF4B2C027E030E041E253E4C501F8
:10E15000B4010E94B2AC18160CF4A7C027E030E05E
:10E1600041E253E4C701B6010E94B2AC18160CF4A8
:10E170009CC080E00E94691A0E94995085E458DB97
:10E18000182F8823B1F08091250C9091260C892BB3
:10E1900009F489C090DB97FD0FC08DDB6F3F7105DF
:10E1A0008105910509F04CF486DB61117CC040E0EB
:10E1B00005C085E4F6DA77C010E0412F01E021E0E8
:10E1C000BE016F5F7F4FCE0105960E94F64B6B013B
:10E1D0007C019B01AC010E949EAF81115FC08D80CC
:10E1E0009E80AF80B88420E030E0A901C501B40171
:10E1F0000E94B2AC87FD05C027E137EB41E558E34B
:10E2000004C027E137EB41E558EBC501B4010E949A
:10E21000D9ABAB01BC0184E295E10E943016898044
:10E220009A80AB80BC8020E030E0A901C501B40138
:10E230000E94B2AC87FD05C027E137EB41E558E30A
:10E2400004C027E137EB41E558EBC501B4010E945A
:10E25000D9ABAB01BC018FE195E10E94301620E003
:10E2600030E0A901C701B6010E94B2AC87FD05C02C
:10E2700027E137EB41E558E304C027E137EB41E5FF
:10E2800058EBC701B6010E94D9ABAB01BC018AE1D2
:10E2900095E10E9430168AE00E9475180E94B850DD
:10E2A0000E94994E02C041E089CF28960FB6F8949B
:10E2B000DEBF0FBECDBFDF91CF911F910F91FF90B9
:10E2C000EF90DF90CF90BF90AF909F908F90089588
:10E2D000EF92FF920F931F93CF93DF938AE561DA5A
:10E2E000882309F456C08091250C9091260C009744
:10E2F00009F44FC0FC017F01C1912C2F2F7D89F0C3
:10E30000C53411F0C536B9F7F701108260E070E04E
:10E310008091250C9091260C0E9442B0F701C08399
:10E3200004C060E070E00E9442B08B01D82FC92F7A
:10E3300020E030E040E050EC0E94B5AE87FD1DC00B
:10E3400020E030E040EA50E4B8018D2F9C2F0E947D
:10E35000B2AC181694F0C801AD2FBC2F80936A059B
:10E3600090936B05A0936C05B0936D05DF91CF91F1
:10E370001F910F91FF90EF9008950E94F6158DE385
:10E3800095E1DF91CF911F910F91FF90EF900C9449
:10E39000E5150E94F31540916A0550916B05609157
:10E3A0006C0570916D058CE295E10E9430168AE053
:10E3B000DF91CF911F910F91FF90EF900C94751802
:10E3C0000895CF92DF92EF92FF920F931F93CF9316
:10E3D000DF93C091270CD091280C80E529DA88239F
:10E3E000D1F08091250C9091260C009749F04AE0DD
:10E3F00050E060E070E00E94D0B26B017C0103C08D
:10E40000C12CD12C760111E0C114D104E104F10436
:10E4100031F410E004C010E0C12CD12C760183E56A
:10E4200007DA882309F486C08091250C9091260C88
:10E43000009701F1FC017F010191202F2F7D89F0D0
:10E44000053411F00536B9F7F701108260E070E08D
:10E450008091250C9091260C0E9442B0F701008318
:10E4600004C060E070E00E9442B0B62FA72FF82FE2
:10E47000E92F04C0B0E0A0E0F0E0E0E020E030E010
:10E480004AE754E46B2F7A2F8F2F9E2F0E94F0AE15
:10E490000E9426AD6B017C01111109C0672B682B0E
:10E4A000692B29F4209719F08881811102C010E0AE
:10E4B00001C011E00E94E15A112329F00E94F315D6
:10E4C000CE010E94CC1883E08093FA0B81E0809308
:10E4D000E60EC114D104E104F10429F10E9468118F
:10E4E000C60ED71EE81EF91E0E946811DC01CB0182
:10E4F0008C199D09AE09BF09B7FD0EC01092E60E3A
:10E5000081E08093FA0BDF91CF911F910F91FF90E3
:10E51000EF90DF90CF9008958091E60E882371F3FD
:10E520000E9440ABE1CF8091E60E882339F30E9430
:10E5300040ABF9CF1111BBCFB5CF1092280C109280
:10E54000270C8FE38093240C1092230C1092220C42
:10E5500010921E0C10921F0C1092200C1092210C85
:10E5600008953F924F925F926F927F928F929F9207
:10E57000AF92BF92CF92DF92EF92FF920F931F93D1
:10E58000CF93DF931F921F92CDB7DEB789839A8313
:10E59000D4DF8981282F9A81392FF90180812F5F5B
:10E5A0003F4F8032D1F38E34B1F4818190ED980FDA
:10E5B0009A3020F08D3211F08B3269F43296DF01FF
:10E5C00031962C9120532A30D0F3CD01FC010196D5
:10E5D00020812032D9F3F0932A0CE093290C8F018B
:10E5E0000F5F1F4F30806AE270E0C8010E9477B46D
:10E5F000009731F0FC01319780818032E1F3118284
:10E600008DE4381631F0E4E53E1619F0F7E43F12D8
:10E61000FFC0F80180810F5F1F4F8032D1F380531C
:10E620008A3008F0F5C03092240C1092230C10921E
:10E63000220C4AE02091220C3091230C429FC00111
:10E64000439F900D11249093230C8093220C3196BC
:10E65000DF0111972C91022E000C330B205331094E
:10E66000280F391F3093230C2093220C8081805374
:10E670008A3000F3DF0131968C918032D9F38DE43A
:10E6800038121AC02E31310591F03CF42731310592
:10E6900071F02C31310581F40AC02537310564F061
:10E6A0002737310524F0203AE3E03E0729F4B09300
:10E6B000280CA093270CACC01092280C1092270CA9
:10E6C0005091290CC12CD12C7601C394FD013196B7
:10E6D0004C91442309F49CC04132A9F48DE43812D2
:10E6E00012C02032310579F4F093280CE093270C06
:10E6F00063E270E0CF010E9477B4009709F488C00C
:10E70000FC01108285C041544A3108F055C0BF0158
:10E71000FB0180816F5F7F4F8032D1F390ED980FC6
:10E720009A3008F18E3211F481810CC08D3211F0D3
:10E730008B3259F4818190ED980F9A30A0F08E328F
:10E7400021F4828180538A3070F08091270C90915F
:10E75000280C892B09F059C0CF0101979093280C00
:10E760008093270C52C0CF01A42FB0E0460157017F
:10E7700004C0880C991CAA1CBB1C4A95D2F7409077
:10E780001E0C50901F0C6090200C7090210C84285F
:10E790009528A628B72880921E0C90921F0CA09254
:10E7A000200CB092210C009711F0851B01C080E075
:10E7B000AC5FB34F8C930AC08091270C9091280CCA
:10E7C000892B21F4B093280CA093270C80818154CD
:10E7D0008A3130F4DF017ACF80ED890F8A3040F43E
:10E7E0004E2F6F2F91919111F7CF842F962F07C045
:10E7F00083ED890F8230A0F39B3291F3F6CFFC01B9
:10E80000019640814032D9F3E5CF80E090E0ACCF73
:10E810000F900F90DF91CF911F910F91FF90EF908C
:10E82000DF90CF90BF90AF909F908F907F906F9030
:10E830005F904F903F9008950E94F3156091290CCE
:10E8400070912A0C8BE595E10E94F91588E595E118
:10E850000C94E5150C945F3E0C944E4B0C94EC41DB
:10E86000CF9383E50E94D16BC82F882331F080912C
:10E87000250C9091260C892B41F483E50E94D16BE5
:10E88000C1E08C2FCF910C942F4315D897FD0BC06E
:10E8900012D86F3F71058105910509F094F70BD8E7
:10E8A000C1E06111EECFC0E0ECCF0E94474B88235E
:10E8B00031F00E94F3158EE695E10C94E51508956C
:10E8C0000E945B6C97FD0CC00E945B6C6F3F7105F2
:10E8D0008105910509F034F40E945B6C862F089540
:10E8E00080E008958FEF08950F931F93CF9383E5F2
:10E8F0000E94D16B811104C001E513E0C0E00DC09E
:10E90000C0E0DEDF682F8C2F0E94D73CCF5FC53080
:10E91000C1F7F2CFCF5FC43069F0F80181918F0168
:10E920000E94D16B8823B1F3CBDF682F8C2F0E941C
:10E93000D73CF0CF82E40E94D16B882329F0C0DF5E
:10E94000682F84E00E94D73CCF911F910F910C94C7
:10E95000843D0F931F93CF9383E50E94186C882307
:10E9600009F465C0ADDF823029F1833009F43FC07E
:10E97000813009F05CC001E513E0C0E0F80181914D
:10E980008F010E94186C882339F09ADF2FEF4FEF28
:10E99000682F8C2F0E94803CCF5FC43079F782E4CF
:10E9A0000E94186C882309F442C08ADF2FEF4FEFD2
:10E9B000682F3AC001E513E0C0E0F80181918F01B2
:10E9C0000E94186C882339F07BDF2FEF482F6FEF00
:10E9D0008C2F0E94803CCF5FC43079F782E40E9484
:10E9E000186C882321F16CDF2FEF482F1CC001E544
:10E9F00013E0C0E0F80181918F010E94186C882318
:10EA000039F05EDF282F4FEF6FEF8C2F0E94803C94
:10EA1000CF5FC43079F782E40E94186C882339F004
:10EA20004FDF282F4FEF6FEF84E00E94803CCF91A3
:10EA30001F910F910C94843DCF93DF931F921F92EF
:10EA4000CDB7DEB769837A830E94D16B69817A8101
:10EA5000882361F08091250C9091260C009731F06D
:10EA60004AE050E060E070E00E94A8B1972F862F46
:10EA70000F900F90DF91CF9108951F93CF93DF9365
:10EA800080E50E94D16B882381F160E070E080E531
:10EA9000D3DF182F6FEF7FEF83E5CEDFEC01019618
:10EAA000039718F517FD21C00E94E15ACF3F8FEF61
:10EAB000D80729F0219771F4C1E0D0E00DC0812F73
:10EAC0000E94BC1331E020E0892B09F030E0C32F15
:10EAD000D22F02C0C0E0D0E0812F0E94BC138C175F
:10EAE0009D0719F00E9440ABF7CFDF91CF911F91A6
:10EAF00008950F931F93CF9383E50E94D16B8823D2
:10EB000009F43EC08091250C9091260C009701F1EC
:10EB1000FC018F01C1912C2F2F7D89F0C53411F09C
:10EB2000C536B9F7F801108260E070E08091250CDD
:10EB30009091260C0E9442B0F801C08304C060E0AE
:10EB400070E00E9442B0B62FA72FF82FE92F04C023
:10EB5000B0E0A0E0F0E0E0E020E030E04AE754E49C
:10EB60006B2F7A2F8F2F9E2F0E94F0AE0E9426AD22
:10EB70006093E10E7093E20E8093E30E9093E40EA7
:10EB8000CF911F910F91089520E040E050E0BA012D
:10EB90000C94C8310C9410AA0F931F93CF9383E564
:10EBA0000E94D16B882391F18091250C9091260CC5
:10EBB000009761F1FC018F01C1912C2F2F7D89F00D
:10EBC000C53411F0C536B9F7F801108260E070E085
:10EBD0008091250C9091260C0E9442B0F801C083D0
:10EBE00004C060E070E00E9442B020E030E04AE7FC
:10EBF00054E40E94F0AE0E9426AD60936B027093C5
:10EC00006C0280936D0290936E0246C088E50E946C
:10EC1000D16B811114C089E50E94D16B81110FC0A5
:10EC20008AE50E94D16B81110AC085E40E94D16BF4
:10EC3000811105C0CF911F910F910C94BC5A0E9475
:10EC4000E15A88E50E94D16B882331F0179A8091B0
:10EC500091058E7F8093910589E50E94D16B882371
:10EC600031F0169A809191058D7F809391058AE508
:10EC70000E94D16B882331F0159A809191058B7F8A
:10EC80008093910585E40E94D16B882329F0CF9170
:10EC90001F910F910C9415AACF911F910F91089578
:10ECA000FF920F931F93CF93DF9383E50E94D16B65
:10ECB0008823F1F083E50E94D16B811102C060E0EE
:10ECC00015C08091250C9091260C892BC1F30E94D0
:10ECD0005B6C97FDF4CF0E945B6C6F3F7105810503
:10ECE000910511F00CF03FC00E945B6C6093A9038A
:10ECF0000E94F3158DEA95E10E94E5158091A90324
:10ED0000882329F103EA15E1C0E0D0E020E08091FA
:10ED1000A90390E00C2E02C0959587950A94E2F71E
:10ED200080FF0EC0FF24F394F20E222319F08CE230
:10ED30000E947518F801859194910E94E5152F2D78
:10ED400021960E5F1F4FC530D10509F704C08FE92A
:10ED500095E10E94E5158AE0DF91CF911F910F9117
:10ED6000FF900C9475186FEFC1CF0E9474230E941E
:10ED700060A70E94BC5A60E070E080E00E940A1B1D
:10ED800068EE73E080E090E00C94A31581E080933E
:10ED9000700283E50E94D16B882331F08091250CAD
:10EDA0009091260C892B39F483E50E94D16B811157
:10EDB00012C00C94A09E0E945B6C97FDFACF0E943B
:10EDC0005B6C6F3F71058105910509F024F40E9489
:10EDD0005B6C662371F3089581E00C94663080E0EB
:10EDE0000C9466300C94E15ACF930E94F31584ED95
:10EDF00095E10E94E51583E50E94D16BC82F882319
:10EE0000D1F08091250C9091260C892B91F00E94D5
:10EE10005B6C97FD0DC00E945B6C6F3F71058105B7
:10EE2000910509F034F40E945B6CC1E0611101C0EE
:10EE3000C0E0C0934502809145020E946A168CECA6
:10EE400095E10E94E5154091390250913A02609196
:10EE50003B0270913C028AEC95E10E943016409191
:10EE60003D0250913E0260913F027091400287EC5A
:10EE700095E10E943016409141025091420260910A
:10EE800043027091440284EC95E10E9430168CEBB1
:10EE900095E10E94E51540912D0250912E0260915E
:10EEA0002F02709130028AEB95E10E94301640915A
:10EEB000310250913202609133027091340287EB3B
:10EEC00095E10E94301640913502509136026091D2
:10EED00037027091380284EB95E10E9430168AE087
:10EEE000CF910C9475180F931F93CF93DF9383E505
:10EEF0000E94186C882309F450C0E2DC182F80E5CA
:10EF00000E94186C81110AC081E0111101C080E0DB
:10EF1000DF91CF911F910F910C948D1580E50E9488
:10EF2000186C882331F00E945B6CEB0177FD35C0D3
:10EF300002C0CDE0D0E00C2F89E40E94186C882339
:10EF400051F08091250C9091260C892B49F0B8DC6A
:10EF5000811106C017C089E40E94D16B882391F00B
:10EF600061E08C2F0E945113612F8C2F0E948D1312
:10EF7000612F70E08C2F0E943412083071F41093CE
:10EF8000C7040BC0802F0E94D9A9882349F3DF91C1
:10EF9000CF911F910F910C9401AADF91CF911F91F6
:10EFA0000F9108950C94D9A70C9475A70C9460A7A1
:10EFB0004F925F926F927F92AF92BF92CF92DF9209
:10EFC000EF92FF92CF93DF93EB01FC01608171819F
:10EFD000828193812CE3C22ED12CE12CF12CA7014C
:10EFE00096010E94DDAFB62EA72ECA01B901A70176
:10EFF00096010E94DDAF6B017C01CA01B90128E1D5
:10F0000030E040E050E00E94DDAF2B013C01C9013F
:10F010006DE671E00E94C9AF61157105D9F0AF923C
:10F02000BF92DF92CF925F924F929F938F937F9385
:10F030006F938CE096E19F938F93DF93CF930E9421
:10F04000A2B48DB79EB70E960FB6F8949EBF0FBEB2
:10F050008DBF61C00097C9F0AF92BF92DF92CF928F
:10F060005F924F929F938F938CEF95E19F938F9335
:10F07000DF93CF930E94A2B4EDB7FEB73C960FB6D4
:10F08000F894FEBF0FBEEDBF46C0411451046104A9
:10F090007104B9F0AF92BF92DF92CF925F924F921C
:10F0A00080EF95E19F938F93DF93CF930E94A2B45B
:10F0B0008DB79EB70A960FB6F8949EBF0FBE8DBF50
:10F0C0002AC0C114D104E104F104A9F0AF92BF92A7
:10F0D000DF92CF9288EE95E19F938F93DF93CF934A
:10F0E0000E94A2B4EDB7FEB738960FB6F894FEBFF3
:10F0F0000FBEEDBF10C0AF92BF9284EE95E19F931B
:10F100008F93DF93CF930E94A2B40F900F900F9034
:10F110000F900F900F90DF91CF91FF90EF90DF90C5
:10F12000CF90BF90AF907F906F905F904F90089579
:10F13000CF93DF93CDB7DEB769970FB6F894DEBFF4
:10F140000FBECDBF0E94A5A76E8B7F8B888F998F36
:10F15000BE016F5F7F4FCE0146962ADF0E94F315F6
:10F16000BE016F5F7F4F80E296E10E94F9158AE051
:10F170000E94751869960FB6F894DEBF0FBECDBF1A
:10F18000DF91CF91089583E50E94D16B882331F000
:10F190008091250C9091260C892B71F40E94F31517
:10F1A0004091660250E060E070E08DE296E10E94DE
:10F1B0005A168AE00C9475180E945B6C97FD17C074
:10F1C0000E945B6C6F3F71058105910509F01CF48D
:10F1D0000E945B6C01C06FEF862F90E0CD971CF40E
:10F1E0006093660208958CE380936602089560E060
:10F1F000F3CF81E00E948D150E94CD3080E00C9409
:10F200008D150E94E15A0C94994E1F93CF93DF9372
:10F21000C091270CD091280C83E010E040E0815091
:10F22000C9F09881292F2B7F2134C9F729812133F7
:10F23000B1F7913421F0953419F441E001C011E0A7
:10F240009E012E5F3F4FE9012F5F3F4F9881903223
:10F25000D1F3E5CF41110E94F315112321F084E38E
:10F2600096E10E94E515CE01DF91CF911F910C949C
:10F27000CC180F931F93CF938C01C62F88E396E190
:10F280000E94E515C8010E94E5158AE30E947518E1
:10F290006AE070E08C2F90E0CF911F910F910C9459
:10F2A0006E198DE497E10E94E51560E08DE397E12A
:10F2B000E0DF60E088E297E1DCDF61E081E297E196
:10F2C000D8DF60E086E197E1D4DF61E086E097E196
:10F2D000D0DF60E08DEF96E1CCDF61E083EF96E177
:10F2E000C8DF61E089EE96E1C4DF61E081EE96E17E
:10F2F000C0DF61E083ED96E1BCDF60E085EC96E184
:10F30000B8DF60E086EB96E1B4DF60E088EA96E182
:10F31000B0DF60E082E996E1ACDF61E081E896E190
:10F32000A8DF60E082E796E1A4DF60E08DE596E18A
:10F33000A0DF61E08AE496E19CDF60E08DE396E186
:10F3400098CF8EE40E94D16B8823A1F08091250C88
:10F350009091260C009771F04AE050E060E070E078
:10F360000E94A8B16093C70E7093C80E8093C90E17
:10F370009093CA0E08954F925F926F927F929F92E0
:10F38000AF92BF92CF92DF92EF92FF920F931F93B3
:10F39000CF93DF9385E5E82E83E0F82E00E512E0B9
:10F3A000B12C912CA12CF70181917F010E94D16B8E
:10F3B000882309F450C08091250C9091260C009769
:10F3C00009F449C0FC013F01C1912C2F2F7D89F028
:10F3D000C53411F0C536B9F7F301108260E070E072
:10F3E0008091250C9091260C0E9442B0F301C083BD
:10F3F00004C060E070E00E9442B06B01D82FC92FBA
:10F40000F80120813181428153810E94D8AB2B01C8
:10F410003C012DEB37E346E855EB0E94B5AE87FD86
:10F420000AC02DEB37E346E855E3C301B2010E9461
:10F43000B2AC181684F4F3E0BF1619F09924939433
:10F4400002C0AA24A394A6016D2F7C2FF80140834B
:10F45000518362837383B3940C5F1F4FF4E0BF1238
:10F46000A2CF992019F00E94C14E03C0A1100E94A2
:10F47000CB4EDF91CF911F910F91FF90EF90DF90D6
:10F48000CF90BF90AF909F907F906F905F904F9084
:10F490000C94994EBF92CF92DF92EF92FF920F930E
:10F4A0001F93CF93DF9329E5E22E23E0F22E0BE2A8
:10F4B0001CE06701C0E0D0E0BB24B394F601819169
:10F4C0006F010E94D16B882351F10E94E15AF8012B
:10F4D0006081662389F070E080E090E00E9454AD86
:10F4E0009B01AC01FE01E25DF34F6081718182817D
:10F4F00093810E94B9AC03C060E070E0CB01209121
:10F50000250C3091260C232B11F00E94246CFE0157
:10F51000E25CF34F6083718382839383B12C2496E2
:10F520000F5F1F4FCC30D10549F686E40E94D16BA6
:10F53000882371F10E94E15A0E94246C8B01D82F1C
:10F54000C92F20E030E040E85FE30E94B5AE181616
:10F550007CF020E030E0A901B8018D2F9C2F0E94A3
:10F56000B2AC87FF09C000E010E0D0E0C0E004C00A
:10F5700000E010E0D0E8CFE3C801AD2FBC2F8093AE
:10F580003A0C90933B0CA0933C0CB0933D0CB12CE7
:10F5900083E50E94D16B882369F00E94E15A0E94A2
:10F5A000246C609367027093680280936902909361
:10F5B0006A02ABC0BB2009F4A8C085E199E10E94B2
:10F5C000E51520E030E0A90160913A0C70913B0C08
:10F5D00080913C0C90913D0C0E94B2AC811104C012
:10F5E00082E199E10E94E51589E099E10E94E51523
:10F5F00040913A0C50913B0C60913C0C70913D0C49
:10F6000085EE98E10E94301684EC98E10E94E515A1
:10F6100082EA98E10E94E5150EE31CE0C9E5D3E01B
:10F6200093E0D92EDE0C80E20E94751889910E9429
:10F630007518F80161917191819191918F0142E06A
:10F6400050E00E94F3198AE00E947518DC12EBCF9B
:10F6500040916702509168026091690270916A025C
:10F660008EE798E10E9430168AE00E9475188CE5BA
:10F6700098E10E94E5158EE2C82E8CE0D82ECBE2F0
:10F68000DCE013E01C0F88818823D1F080E20E9427
:10F690007518F70180810E947518688170E080E01C
:10F6A00090E00E9454AD9B01AC01F6016081718134
:10F6B000828193810E94B9AC42E050E00E94F3192C
:10F6C0002196FFEFEF1AFF0A84E0C80ED11C1C132D
:10F6D000DACF80912B0C81110CC080912C0C811100
:10F6E00008C080912D0C811104C088E498E10E942B
:10F6F000E5158AE0DF91CF911F910F91FF90EF9078
:10F70000DF90CF90BF900C947518DF91CF911F912F
:10F710000F91FF90EF90DF90CF90BF9008952F92C0
:10F720003F924F925F926F927F928F929F92AF9291
:10F73000BF92CF92DF92EF92FF920F931F93CF93DE
:10F74000DF93CDB7DEB76A970FB6F894DEBF0FBE72
:10F75000CDBF182F81E00E948D158FE40E94186C98
:10F760008823B9F08091250C9091260C892BB1F05B
:10F770000E945B6C97FD18C00E945B6C6F3F710527
:10F780008105910509F054F40E945B6C611106C07B
:10F790000BC08FE40E94D16B882331F090919205C9
:10F7A0009770973009F40FC20E94E15A2091150614
:10F7B000288F80E00E94691A0E94995081E00E947F
:10F7C0007930111119C088E50E94D16B382E89E576
:10F7D0000E94D16B182F8AE50E94D16B282E311020
:10F7E00006C0111110C081110EC0312E0AC01123A4
:10F7F00051F0312E082F08C011E033243394222415
:10F80000239401E001C000E080E1E0E5F2E0A0E83F
:10F81000B5E001900D928A95E1F7011102C0222016
:10F8200019F082E00E94935382E50E94186C8823AD
:10F8300071F18091250C9091260C009709F457C026
:10F84000FC015F012191322F3F7D99F0253411F0A9
:10F850002536B9F7D5011C9260E070E08091250C47
:10F860009091260C2A8F0E9442B02A8DF5012083A8
:10F8700004C060E070E00E9442B06B017C0120E0B7
:10F8800030E0A9010E94B2AC882389F106C0C12CE6
:10F89000D12C20E8E22E30E4F32E011105C0311006
:10F8A00003C0112309F410C1C601D7018093880554
:10F8B00090938905A0938A05B0938B0520915802F7
:10F8C0003091590240915A0250915B02B601C70132
:10F8D0000E94B5AE18165CF419821A821B821C8233
:10F8E000BE016F5F7F4F88E895E00E945A5001117A
:10F8F0000CC0332009F4FCC0111107C080E00E9445
:10F900009353002309F47EC1DCC01092540210927C
:10F910005502109256021092570210925002109205
:10F92000510210925202109253020E94C14EE6E31D
:10F93000F4E12491298FE5E4F4E185909590A59078
:10F94000B490E9E4F4E14590559065907490A3017A
:10F950009201C501B4010E94B5AE18162CF4A501A0
:10F960009401C301B20104C0A3019201C501B40115
:10F970000E94B9AC6B017C01EEE2F4E185919591B6
:10F98000A591B4918D879E87AF87B88BEAE2F4E1A9
:10F9900085919591A591B491898B9A8BAB8BBC8BFA
:10F9A0002D853E854F855889BC01CD010E94B2ACA2
:10F9B00087FD09C09D859D8BAE85AE8BBF85BF8BB6
:10F9C000E889ED8708C0F989FD8B2A892E8B8B8900
:10F9D0008F8B9C899D87A7019601C701B6010E9464
:10F9E000F0AE20E030E040E85FE30E94D9AB0E9437
:10F9F0005DAF9B01AC016D897E898F899D850E94D9
:10FA0000F0AE69877A878B879C87E7E3F4E1F4900F
:10FA100020E030E040EC5FE3C301B2010E94F0AEB1
:10FA20002B013C016F2DFF0C770B880B990B0E946B
:10FA300054AD9B01AC01C301B2010E94F0AE6983D9
:10FA40007A838B839C8320E030E040EC5FE3C50148
:10FA5000B4010E94F0AE6B017C01A98D6A2FAA0F40
:10FA6000770B880B990B0E9454AD9B01AC01C70129
:10FA7000B6010E94F0AE6D837E838F839887AE01BE
:10FA8000475F5F4FBE016F5F7F4FCE0105960E94BB
:10FA900078500E94403010925402109255021092F9
:10FAA0005602109257021092500210925102109278
:10FAB000520210925302011121CF3110A0C0112324
:10FAC00019F081E00E9493530E94C14EF090E70428
:10FAD00080E00E946630812C912C90EAA92E90E45F
:10FAE000B92E89829A82AB82BC82011115C0A8C04E
:10FAF0001111E7CF0E94C14EF090E70480E00E9410
:10FB0000663080E090E0A0EAB0E489839A83AB831A
:10FB1000BC83222009F48BC080E090E0ADE1B3E427
:10FB20008D839E83AF83B887BE016F5F7F4FCE0109
:10FB300005960E945A5080E090E0A0EAB0E48983E4
:10FB40009A83AB83BC8301110BC0111109C0809152
:10FB5000540290915502A0915602B091570204C0F0
:10FB600080E090E0A9E3B3E48D839E83AF83B88700
:10FB700001110BC0311009C08091500290915102C7
:10FB8000A0915202B091530204C080E090E0A0EA3C
:10FB9000B0E489879A87AB87BC87AE014F5F5F4F20
:10FBA000BE016B5F7F4FCE0109960E9478508F2D6A
:10FBB0000E9466300E943B30888D0E94691A0E9424
:10FBC000B8500E94994E80E00E948D156A960FB63B
:10FBD000F894DEBF0FBECDBFDF91CF911F910F9183
:10FBE000FF90EF90DF90CF90BF90AF909F908F905D
:10FBF0007F906F905F904F903F902F90089580E09E
:10FC00000E94935311115DCF0E94C14EF090E70402
:10FC100080E00E946630812C912C80EAA82E80E43E
:10FC2000B82E89829A82AB82BC8221101FC080913B
:10FC3000580290915902A0915A02B0915B0270CF84
:10FC40002220A9F380E090E0ADE1B3E48D839E83B0
:10FC5000AF83B887BE016F5F7F4FCE0105960E94CC
:10FC60005A5089829A82AB82BC826FCF80E090E04A
:10FC7000ADE1B3E48D839E83AF83B887BE016F5F30
:10FC80007F4FCE0105960E945A5089829A82AB829C
:10FC9000BC825DCF80E1E0E5F2E0A0E8B5E0019054
:10FCA0000D928A95E1F708954F925F926F927F923D
:10FCB0008F929F92AF92BF92CF92DF92EF92FF927C
:10FCC0000F931F93CF93DF93CDB7DEB72E970FB669
:10FCD000F894DEBF0FBECDBF270138012E874A87BB
:10FCE0005B876C877D878987D5DF89852E854A85E7
:10FCF0005B856C857D858F3F51F094E0899FF00195
:10FD00001124E058FA4F40835183628373832F3F5D
:10FD100051F0A4E02A9FF0011124E058FA4F4082EC
:10FD2000518262827382BFEFCB1651F084E0C89E8D
:10FD3000F0011124E058FA4F80829182A282B382AE
:10FD40008090800590908105A0908205B0908305F9
:10FD500020E030E042E253E4C501B4010E94B2ACBD
:10FD600087FF11C020E030E040E450ECC501B40151
:10FD70000E94B5AE18166CF0812C912C30E4A32EA5
:10FD800030ECB32E06C0812C912C22E2A22E23E46B
:10FD9000B22E8092800590928105A0928205B09249
:10FDA000830540908405509085056090860570908D
:10FDB000870520E030E04EE353E4C301B2010E9426
:10FDC000B2AC87FF11C020E030E040EE50ECC30140
:10FDD000B2010E94B5AE18166CF0412C512C90EE79
:10FDE000692E90EC792E06C0412C512C8EE3682EA2
:10FDF00083E4782E409284055092850560928605B2
:10FE0000709287058091880590918905A0918A0557
:10FE1000B0918B058D839E83AF83B88720E030E05F
:10FE20004FE153E4BC01CD010E94B2AC87FF11C089
:10FE300020E030E040E050EC6D817E818F8198853C
:10FE40000E94B5AE18166CF080E090E0A0E0B0EC37
:10FE500004C080E090E0AFE1B3E48D839E83AF8384
:10FE6000B8878D819E81AF81B885809388059093F6
:10FE70008905A0938A05B0938B0580E090E0A8E403
:10FE8000B2E489839A83AB83BC83DE0111966D0152
:10FE9000ED80FE800F811885A3019201C501B40198
:10FEA0000E94A64F2E960FB6F894DEBF0FBECDBFB0
:10FEB000DF91CF911F910F91FF90EF90DF90CF9046
:10FEC000BF90AF909F908F907F906F905F904F907A
:10FED00008958F929F92AF92BF92CF92DF92EF924E
:10FEE000FF920F931F93CF93DF93EC016A017B0185
:10FEF00020E030E040E45FE3688579858A859B8572
:10FF00000E94D9ABA70196010E94D9ABAB01BC01FD
:10FF1000812C912C5401CC24CA94850174012FEFBB
:10FF200082E0C2DEEC80FD800E811F814881598114
:10FF30006A817B8121E080E0B7DEDF91CF911F9164
:10FF40000F91FF90EF90DF90CF90BF90AF909F9078
:10FF50008F9008952F923F924F925F926F927F926F
:10FF60008F929F92AF92BF92CF92DF92EF92FF92C9
:10FF70000F931F93CF93DF93CDB7DEB72E970FB6B6
:10FF8000F894DEBF0FBECDBF89878B014A8722233D
:10FF900059F0812C912C90E8A92E9EE3B92E80E097
:10FFA00090E0A0EAB1E40CC08AE0882E87ED982E9C
:10FFB00083E2A82E8CE3B82E80E090E0A0E8BFE3B7
:10FFC00089839A83AB83BC83211105C080E090E0D4
:10FFD000A0EAB0E404C080E090E0A8E4B2E48D833D
:10FFE0009E83AF83B88756DE412C512C3201B985F0
:10FFF000A4E0BA9FC0011124FC01E058FA4F1F0190
:020000021000EC
:10000000C801110FAA0BBB0B8B879C87AD87BE87DE
:100010002D813E814F815885C301B2010E94B2AC4F
:1000200087FF3FC06B857C858D859E850E9454AD82
:10003000A50194010E94F0AE9B01AC01D1016D912C
:100040007D918D919C910E94D9ABF1016083718368
:1000500082839383E0908805F090890500918A055A
:1000600010918B052091840530918505409186057E
:10007000509187056091800570918105809182057E
:1000800090918305DE0111966D010E94A64F0E949A
:10009000E15A83B182958170B1E08B27EA858E1396
:1000A00024C0398524E0329FF0011124E058FA4F32
:1000B00060817181828193812E960FB6F894DEBFA4
:1000C0000FBECDBFDF91CF911F910F91FF90EF90A9
:1000D000DF90CF90BF90AF909F908F907F906F9068
:1000E0005F904F903F902F900895A5019401C30118
:1000F000B2010E94D9AB2B013C018ACF4F925F9293
:100100006F927F928F929F92AF92BF92CF92DF9227
:10011000EF92FF920F931F93CF93DF93CDB7DEB78C
:1001200028970FB6F894DEBF0FBECDBFB82E6B0177
:10013000A42E4901C801B701FF24F39420E030E068
:1001400040EA50E40E94B2AC8111F12CA3DD84E0BE
:10015000B89E80011124F801E058FA4F8081918106
:10016000A281B3818D839E83AF83B8872F2D4A2DC3
:10017000B6018B2DEFDE2B013C018114910411F1AE
:10018000F11020C041E04A25662777276C197D09C8
:1001900020E08B2DDFDEA30192010E94D8AB6B0122
:1001A0007C0120E030E0A9010E94B5AE87FF04C0C9
:1001B000F7FAF094F7F8F094D401CD92DD92ED9235
:1001C000FC921397F801E058FA4F8D819E81AF8120
:1001D000B88580839183A283B38380E090E0A8E414
:1001E000B2E489839A83AB83BC83E0908805F09066
:1001F000890500918A0510918B0520918405309125
:100200008505409186055091870560918005709124
:1002100081058091820590918305DE0111966D0123
:100220000E94A64FC301B20128960FB6F894DEBF14
:100230000FBECDBFDF91CF911F910F91FF90EF9037
:10024000DF90CF90BF90AF909F908F907F906F90F6
:100250005F904F9008952F923F924F925F926F92CE
:100260007F928F929F92AF92BF92CF92DF92EF9246
:10027000FF920F931F93CF93DF93CDB7DEB76997AC
:100280000FB6F894DEBF0FBECDBF3C014C8B5D8B2B
:100290006E8B7F8B2D878CE0E1E1F3E0DE01119620
:1002A00001900D928A95E1F74C895D896E897F896D
:1002B000C3010FDE2D852230D1F060F42223F1F04E
:1002C000213009F073C1212C312C60E8462E6FEBF0
:1002D000562E46C03D853330C9F1343009F066C131
:1002E000212C312C70E8472E7FEB572E36C0212C65
:1002F000312CF0E84F2EFFE35F2E2FC09301205EDC
:100300003F4FEC88FD880E891F8941E06FEF7FEF3A
:1003100082E0F4DE6B017C0120E030E040E05FE34E
:1003200069857A858B859C850E94F0AE9B01AC0126
:10033000C701B6010E94D8ABF3016087718782873D
:100340009387C486D586E686F78630C1212C312C6A
:10035000E0E84E2EEFE35E2E03C0DD24D39401C00F
:10036000D12C2D2D30E03F872E87002309F463C068
:10037000C901880F991F880F991F7301E80EF91E94
:10038000E1E0F0E0EC0FFD1FE80FF91F20E030E0A6
:1003900040E05FE360817181828193810E94F0AED1
:1003A000F701E05CFF4F20813181428153810E943F
:1003B000D8AB9B01AC01C201B10190580E94F0AED4
:1003C000F70120813181428153810E94D9ABAB0179
:1003D000BC01812C912C5401CC24CA948501740158
:1003E0002FEF8D2D61DCEC88FD880E891F8993012C
:1003F000205E3F4F41E06FEF7FEF82E07FDE4B01F9
:100400005C01F301648775878687978720E030E079
:1004100040E05FE369857A858B859C850E94F0AE1C
:100420009B01AC01C501B4010E94D8ABF301608708
:100430007187828793878E859F85880F991F880F84
:10044000991F9301280F391F3F872E87E1E0F0E0C5
:10045000EC0FFD1FE80FF91F20E030E040E05FE304
:1004600060817181828193810E94F0AE688B798B6B
:100470008A8B9B8B52014101B7FAB094B7F8B094C4
:100480008E859F85805C9F4F998F888F20E030E01C
:1004900040E05FE3FC0160817181828193810E9471
:1004A000F0AE9B01AC01688979898A899B890E9499
:1004B000D9AB2C893D894E895F890E94D9AB9B01BC
:1004C000AC01C501B4010E94F0AEEE85FF8520812C
:1004D0003181428153810E94D9ABAB01BC01812C97
:1004E000912C5401CC24CA94850174012FEF8D2DD9
:1004F000DBDB23E333E343E35FE3F30164857585EB
:10050000868597850E94D8ABAB01BC012FEF82E0B6
:10051000CBDBFD85AF2EB12C450128E0820E911C6E
:10052000880C991C880C991C860C971CC201B1017F
:100530000E9421ADEC88FD880E891F89940141E05D
:100540008D2DDCDD6B017C0120E030E040E05FE3DD
:10055000E88DF98D60817181828193810E94F0AE76
:100560009B01AC01688979898A899B890E94D9ABF2
:100570009B01AC01C201B1010E94F0AE9B01AC0134
:10058000C701B6010E94D9ABEE85FF8560837183F8
:1005900082839383F5013396EE0FFF1FEE0FFF1F4B
:1005A000E60DF71DC082D182E282F38269960FB612
:1005B000F894DEBF0FBECDBFDF91CF911F910F9199
:1005C000FF90EF90DF90CF90BF90AF909F908F9073
:1005D0007F906F905F904F903F902F900895CF92B3
:1005E000DF92EF92FF920F93CF93DF93EC016A01BA
:1005F0007B0100E020E02FDE22E0B701A601CE0162
:100600002ADE23E0B701A601CE0125DEB701A6014F
:10061000CE015FDC1CAA1DAA1EAA1FAA18AE19AE25
:100620001AAE1BAE288539854A855B8560E070E08F
:10063000CB010E94D8AB6CAF7DAF8EAF9FAFDF9187
:10064000CF910F91FF90EF90DF90CF9008958F9210
:100650009F92AF92BF92CF92DF92EF92FF920F9351
:100660001F93CF93DF93EC01C0903A0CD0903B0CDA
:10067000E0903C0CF0903D0C80E090E0A0E8BFE3FF
:1006800080933A0C90933B0CA0933C0CB0933D0CA0
:100690008090670290906802A0906902B0906A0210
:1006A00010926702109268021092690210926A0218
:1006B000CE0195DF0E94E15A00E512E02CAD3DAD80
:1006C0004EAD5FADF80160857185828593850E948E
:1006D000D9ABF8016087718782879387188619865E
:1006E0001A861B861CAE1DAE1EAE1FAE0E94C14EEA
:1006F0008092670290926802A0926902B0926A02A8
:10070000C0923A0CD0923B0CE0923C0CF0923D0C23
:10071000DF91CF911F910F91FF90EF90DF90CF90DD
:10072000BF90AF909F908F9008952F923F924F92DD
:100730005F926F927F928F929F92AF92BF92CF9271
:10074000EF92FF920F931F93CF93DF93CDB7DEB756
:1007500028970FB6F894DEBF0FBECDBF5C01809125
:100760003A0C90913B0CA0913C0CB0913D0C8D83C8
:100770009E83AF83B88710923A0C10923B0C109274
:100780003C0C10923D0C8091670290916802A09100
:100790006902B0916A0289839A83AB83BC83109209
:1007A0006702109268021092690210926A02C501F3
:1007B00016DFEEE3FCE0D5019C964D915D916D91C5
:1007C0007C919F97408351836283738398964D9168
:1007D0005D916D917C919B9744835583668377836C
:1007E00090964D915D916D917C9193974087518743
:1007F0006287738780E090E0A0E8BFE380933A0CC3
:1008000090933B0CA0933C0CB0933D0C109267026C
:10081000109268021092690210926A0280E5282EF6
:1008200082E0382E20E030E040E450E4F1016085C1
:100830007185828593850E94D9AB4B015C0120E0D4
:1008400030E040E450E4D10114966D917D918D919A
:100850009C9117970E94D9AB2B013C0120E030E01E
:1008600040E450E4F10160817181828193810E94B2
:10087000D9ABAB01BC0192E0C92E8301720121E02A
:1008800080E012DA20E030E040E450E4D101189634
:100890006D917D918D919C911B970E94D8AB4B01DE
:1008A0005C0120E030E040E450E4F10164817581B6
:1008B000868197810E94D8AB2B013C0120E030E07B
:1008C00040E450E4D1016D917D918D919C910E9405
:1008D000D8ABAB01BC018301720121E080E0E4D917
:1008E00089819A81AB81BC81809367029093680271
:1008F000A0936902B0936A028D819E81AF81B88511
:1009000080933A0C90933B0CA0933C0CB0933D0C1D
:1009100028960FB6F894DEBF0FBECDBFDF91CF9102
:100920001F910F91FF90EF90CF90BF90AF909F904D
:100930008F907F906F905F904F903F902F90089591
:100940008F929F92AF92BF92CF92DF92EF92FF92DF
:10095000C0903A0CD0903B0CE0903C0CF0903D0CD9
:10096000812C912C20E8A22E2FE3B22E80923A0CFB
:1009700090923B0CA0923C0CB0923D0C8090670290
:1009800090906802A0906902B0906A02109267028B
:10099000109268021092690210926A0258DE8092E8
:1009A000670290926802A0926902B0926A02C092B5
:1009B0003A0CD0923B0CE0923C0CF0923D0CFF9034
:1009C000EF90DF90CF90BF90AF909F908F90089561
:1009D0009C018CE0EDE1F3E0D90101900D928A9544
:1009E000E1F798E0E9E2F3E0D901A05CBF4F0190A4
:1009F0000D929A95E1F708954F925F926F927F92D0
:100A00008F929F92AF92BF92CF92EF92FF920F93ED
:100A10001F93CF93DF93CDB7DEB7CC54D1090FB678
:100A2000F894DEBF0FBECDBFCE010196D1DF40905E
:100A30003A0C50903B0C60903C0C70903D0C80E068
:100A400090E0A0E8BFE380933A0C90933B0CA09316
:100A50003C0CB0933D0C8091670290916802A0918C
:100A60006902B0916A022D968CAF9DAFAEAFBFAF59
:100A70002D971092670210926802109269021092EC
:100A80006A0240E050E060EA70E4CE01019658DF6F
:100A900040E050E060E87FE3CE01019646DE40E0B2
:100AA00050E060E87FE3CE0101964ADF812C912C73
:100AB0005401CC24CA94850174012FEF40E050E02A
:100AC00066E173E480E0F0D82D968CAD9DADAEADBF
:100AD000BFAD2D978093670290936802A09369023F
:100AE000B0936A0240923A0C50923B0C60923C0CDC
:100AF00070923D0CC45BDF4F0FB6F894DEBF0FBEA3
:100B0000CDBFDF91CF911F910F91FF90EF90CF90CC
:100B1000BF90AF909F908F907F906F905F904F901D
:100B200008959F92AF92BF92CF92DF92EF92FF9281
:100B30000F931F93CF93DF93CDB7DEB7C854D1097E
:100B40000FB6F894DEBF0FBECDBF81E00E948D15B9
:100B500000914502109245029090150680E00E9497
:100B6000691A41E061E081E00E9442528111EEC0C9
:100B7000CE0101962DDF85E50E94D16B882341F1DE
:100B80002091250C3091260C2115310509F1F90130
:100B90005F011191812F8F7D99F0153411F0153679
:100BA000B9F7F501108260E070E08091250C90911A
:100BB000260C0E9442B06B017C01F50110830EC02F
:100BC00060E070E0C9010E9442B06B017C0106C088
:100BD000C12CD12C80E8E82E8FE3F82E82E40E940D
:100BE000D16B882331F0B701A601CE0101969DDDBE
:100BF000ADC084E50E94D16B882391F08091250CD3
:100C00009091260C009731F04AE050E060E070E0EF
:100C10000E94A8B1B701A601CE01019618DD96C0C9
:100C200086E50E94D16B882309F48FC0B701A60125
:100C3000CE010196D4DC8AE00E9475188FEA99E112
:100C40000E94E5154D855E856F85788987EA99E173
:100C50000E9430168AE00E947518498D5A8D6B8D5E
:100C60007C8D8EE999E10E9430168AE00E94751809
:100C70004D895E896F89788D84E999E10E943016EB
:100C80008AE00E9475188AE00E9475188BE899E145
:100C90000E94E51549855A856B857C8588E899E130
:100CA0000E9430168AE00E9475188AE00E9475182A
:100CB0008DE799E10E94E5154DA55EA56FA578A980
:100CC00084E799E10E9430168AE00E94751849A5D0
:100CD0005AA56BA57CA58AE699E10E9430168AE0A8
:100CE0000E94751849A15AA16BA17CA182E699E1E5
:100CF0000E9430168AE00E9475188AE00E947518DA
:100D000084E499E10E94E5158AE00E94751884E563
:100D10000E9475186AE070E080E090E00E94681917
:100D200080E399E10E94E51521964CAD5DAD6EAD75
:100D30007FAD21978DE299E10E9430168AE00E94F2
:100D400075188AE00E94751801C056DE892D0E9430
:100D5000691A0093450280E00E948D15C85BDF4F41
:100D60000FB6F894DEBF0FBECDBFDF91CF911F91BC
:100D70000F91FF90EF90DF90CF90BF90AF909F903A
:100D800008951F93CF93DF93CDB7DEB72C970FB69F
:100D9000F894DEBF0FBECDBF83E50E94D16B8823E0
:100DA000B9F08091250C9091260C892BC9F00E94F6
:100DB0005B6C97FD10C00E945B6C6F3F71058105F5
:100DC000910509F06CF40E945B6C611109C003C0CD
:100DD0001091150606C080E00E94691A10E001C05B
:100DE00011E08091500290915102A0915202B09175
:100DF000530289839A83AB83BC8380915402909180
:100E00005502A0915602B09157028D839E83AF8305
:100E1000B8878091580290915902A0915A02B091DE
:100E20005B0289879A87AB87BC8786E50E94D16B76
:100E3000882331F064EE79E181EF95E00E948AA683
:100E4000812F0E94691A112351F08091150681119A
:100E500006C00E94F61585EC99E10E94E5150E94F6
:100E6000F31587EB99E10E94E515809115060E9424
:100E700072164CE050E060E572E0CE0101960E94EF
:100E80006AB4892B59F02C960FB6F894DEBF0FBECA
:100E9000CDBFDF91CF911F910C94994E2C960FB638
:100EA000F894DEBF0FBECDBFDF91CF911F910895A3
:100EB0008F929F92AF92BF92CF92DF92EF92FF926A
:100EC000CF934B015C0169017A0122ED30E040EEE5
:100ED00050ECC701B6010E94B5AE87FD33C027E0D4
:100EE00030E04EE353E4C701B6010E94B2AC1816DD
:100EF0004CF123EA31E040E450ECC501B4010E941A
:100F0000B5AE87FD1FC027E030E042E253E4C501E3
:100F1000B4010E94B2AC1816ACF027E030E041E218
:100F200053E4C501B4010E94B2AC18165CF0C1E0F4
:100F300027E030E041E253E4C701B6010E94B2ACC1
:100F400018160CF4C0E08C2FCF91FF90EF90DF903B
:100F5000CF90BF90AF909F908F900895CF93DF93E5
:100F6000D82FC62F0E94186C8823D1F08091250CB1
:100F70009091260C892B11F481E01AC00E945B6CC1
:100F800097FD15C00E945B6C6F3F7105810591054F
:100F900009F094F70E945B6C81E0611109C007C001
:100FA0008D2F0E94D16B8111E7CF8C2F01C080E083
:100FB000DF91CF9108952F923F924F925F926F925F
:100FC0007F928F929F92AF92BF92CF92DF92EF92D9
:100FD000FF920F931F93CF93DF93CDB7DEB7CB5123
:100FE000D1400FB6F894DEBF0FBECDBF81E00E94A6
:100FF0008D1541E061E081E00E94425281111AC0EA
:1010000080911506882329F060E08FE4A7DF811125
:1010100011C0FE0131968CE3DF011D928A95E9F73C
:10102000309015068AE40E94D16B982E882329F00F
:101030000E94881A912C0C94EC9160E070E086E597
:101040000E941C75C351DF4F99838883CD5ED040C9
:10105000059718F087EC9BE136C160E084E47EDF01
:10106000C950DF4F8883C75FD040C351DF4F28810D
:101070003981CD5ED040233031054CF460E084E509
:101080006DDFC450DF4F8883CC5FD04006C031E0B5
:10109000C450DF4F3883CC5FD04062E070E088E519
:1010A0000E941C75182F62E070E089E50E941C7593
:1010B000082F80E50E94186C811103C0612F802FDA
:1010C00003C00E945B6C862F623019F08EE99BE1B1
:1010D000FAC0823019F085E79BE1F5C083E50E94F4
:1010E000186C882319F00E94246C04C060E070E83A
:1010F0008BEB95E420E030E040E752E40E94B9AC8D
:10110000609346027093470280934802909349028D
:1011100088E40E94D16B882391F10E94246C0E9484
:1011200021AD8B0177FF02C00F5F1F4F159507950B
:10113000119501951109035B1F4F0E3F4FEF1407E7
:101140002CF44DEFA42EBB24BA9401C058016501C4
:10115000C60ED71E51EAC516D1041CF031EAC32EC3
:10116000D12C0A3FAFEF1A0714F409EF1FEF7801F3
:10117000E60EF71EB1EAEB16F104CCF135C08CE4B3
:101180000E94186C882331F00E94246C0E9421ADCB
:101190005B0104C02DEFA22EBB24BA9482E50E940D
:1011A000186C882331F00E94246C0E9421AD6B01E1
:1011B00003C091EAC92ED12C86E40E94186C8823C2
:1011C00031F00E94246C0E9421AD8B0102C009EF16
:1011D0001FEF82E40E94186C882331F00E94246C77
:1011E0000E9421AD7B0103C081EAE82EF12CB801F9
:1011F000012E000C880B990B0E9454ADC250DF4F9A
:10120000688379838A839B83CE5FD040B5010B2CA2
:10121000000C880B990B0E9454ADCE5FDE4F6883A3
:1012200079838A839B83C250D140C250DF4F28818B
:1012300039814A815B81CE5FD0403ADE882309F450
:1012400040C0B7010F2C000C880B990B0E9454ADC5
:101250009B01AC01B6010D2C000C880B990BC85EEC
:10126000DE4F2883C851D140C75EDE4F3883C95155
:10127000D140C65EDE4F4883CA51D140C55EDE4FC5
:101280005883CB51D1400E9454ADC85EDE4F2881B7
:10129000C851D140C75EDE4F3881C951D140C65ECA
:1012A000DE4F4881CA51D140C55EDE4F5881CB51D7
:1012B000D140FEDDCA50DF4F8883C65FD040811128
:1012C00006C089E59BE10E94E5150C94EC91B601FE
:1012D0006A197B09072E000C880B990B0E9454ADEC
:1012E000C65FDE4F688379838A839B83CA50D1406F
:1012F000B701601B710B072E000C880B990B0E9425
:1013000054ADC25FDE4F688379838A839B83CE505E
:10131000D140C351DF4FE881F981CD5ED040EF2B42
:1013200091F083E49BE10E94E515C950DF4FE8810D
:10133000C75FD040EE2321F089E39BE10E94E515D1
:101340008AE00E9475180E94E15A80E00E94691AA2
:1013500081E00E94554B882329F0832D0E94691A51
:101360000C94EC910E94995060E085E4F7DD8111C6
:1013700007C0F2E0C350DF4FF883CD5FD04006C016
:1013800021E0C350DF4F2883CD5FD040C151DF4FF4
:1013900019821882CF5ED040C752DF4F188219825F
:1013A0001A821B82C95DD040C850DF4F1882198253
:1013B0001A821B82C85FD040C751DF4F1882C95EB6
:1013C000D0404FEF5FEFC352DF4F59834883CD5D6D
:1013D000D0405FEFCB50DF4F5883C55FD0408FEFD9
:1013E000CD50DF4F8883C35FD04091E0CB52DF4FB9
:1013F0009883C55DD040C352DF4F88819981CD5D10
:10140000D0400196880F991F880F991F4DE350E037
:101410004C0F5D1F480F591FCB51DF4F5983488335
:10142000C55ED040DC011497C85FDE4FB983A88346
:10143000C850D1408CE0C352DF4F28813981CD5D47
:10144000D040829FF001839FF00D1124CA5FDE4FD0
:10145000F983E883C650D140CF51DF4F19821882FB
:10146000C15ED040C151DF4F88819981CF5ED040AD
:10147000092E000CAA0BBB0BCE5EDE4F888399832E
:10148000AA83BB83C251D140C151DF4FA881B9812A
:10149000CF5ED040AA0FBB1FCA5EDE4FB983A883C0
:1014A000C651D140CB52DF4F5881C55DD040CD50A1
:1014B000DF4F8881C35FD040581709F497C2CE5ED2
:1014C000DE4F688179818A819B81C251D1400E941F
:1014D00054AD9B01AC01C65FDE4F688179818A8182
:1014E0009B81CA50D1400E94F0AE9B01AC01CE5FFF
:1014F000DE4F688179818A819B81C250D1400E94F0
:10150000D9AB4B015C01CB52DF4FB881C55DD040F8
:101510006B2FBB0F770B880B990B0E9454AD9B016F
:10152000AC01C25FDE4F688179818A819B81CE5098
:10153000D1400E94F0AE9B01AC01C250DF4F6881E8
:1015400079818A819B81CE5FD0400E94D9AB6B01AB
:101550007C0120E030E0A901C501B4010E94B2ACD9
:1015600087FD05C020E030E040E05FE303C020E0FD
:1015700030E0A901C501B4010E94D9AB0E948FAD32
:10158000C355DF4F688379838A839B83CD5AD040CC
:1015900020E030E0A901C701B6010E94B2AC87FD8E
:1015A00005C020E030E040E05FE303C020E030E031
:1015B000A901C701B6010E94D9AB0E948FADC755E2
:1015C000DF4F688379838A839B83C95AD040C35293
:1015D000DF4FE881F981CD5DD0403196C352DF4FB6
:1015E000F983E883CD5DD040CA5EDE4FE881F981A2
:1015F000C651D140CB52DF4F2881C55DD040E20FAC
:10160000F11D27FDFA95EE0FFF1F41EA50E04C0F48
:101610005D1FE40FF51FC352DF4F88819981CD5DB7
:10162000D0409183808301E0C351DF4F2881CD5E9C
:10163000D040C350DF4F4881CD5FD040BE016755D9
:101640007F4FCE0183559F4F0E94F64BC752DF4F0D
:10165000688379838A839B83C95DD0409B01AC01F9
:101660000E949EAF882321F0832D0E94691AD5C164
:10167000C752DF4F288139814A815B81C95DD040E3
:10168000C850DF4F688179818A819B81C85FD040D3
:101690000E94D9ABC850DF4F688379838A839B83CC
:1016A000C85FD040CF51DF4FE881F981C15ED040A3
:1016B000C85FDE4FA881B981C850D140EA0FFB1F37
:1016C0002DE630E02C0F3D1FE20FF31FC752DF4F16
:1016D00088819981AA81BB81C95DD040848395832B
:1016E000A683B783C355DF4F488059806A807B80CB
:1016F000CD5AD040CB51DF4FA881B981C55ED040D3
:101700004D925D926D927D92CB51DF4FB983A8834C
:10171000C55ED040CF51DF4FE881F981C15ED04036
:101720003496CF51DF4FF983E883C15ED040C7556F
:10173000DF4F88809980AA80BB80C95AD0401C9610
:101740008D929D92AD92BC921F9720E030E040E8D0
:101750005FE35C962D933D934D935C935F97A3015C
:10176000920169817A818B819C810E94D9AB6983C6
:101770007A838B839C83A50194016D817E818F8107
:1017800098850E94D9AB6D837E838F839887C752DB
:10179000DF4F288139814A815B81C95DD0406985ED
:1017A0007A858B859C850E94D9AB69877A878B87E0
:1017B0009C87A3019201C301B2010E94F0AE9B017C
:1017C000AC016D857E858F8598890E94D9AB6D8728
:1017D0007E878F87988BA5019401C501B4010E9473
:1017E000F0AE9B01AC0169897A898B899C890E9442
:1017F000D9AB698B7A8B8B8B9C8BC752DF4F28813F
:1018000039814A815B81C95DD040CA01B9010E941A
:10181000F0AE9B01AC016D897E898F89988D0E9405
:10182000D9AB6D8B7E8B8F8B988FA5019401C301F3
:10183000B2010E94F0AE9B01AC01698D7A8D8B8D57
:101840009C8D0E94D9AB698F7A8F8B8F9C8FC752EA
:10185000DF4F288139814A815B81C95DD040C30156
:10186000B2010E94F0AE9B01AC016D8D7E8D8F8D1B
:1018700098A10E94D9AB6D8F7E8F8F8F98A3C7528E
:10188000DF4F288139814A815B81C95DD040C50124
:10189000B4010E94F0AE9B01AC0169A17AA18BA1B9
:1018A0009CA10E94D9AB69A37AA38BA39CA31DA181
:1018B0000EA13FA028A420E030E0A901C301B2019D
:1018C0000E94B5AE7301620187FF04C0F7FAF0947D
:1018D000F7F8F094212F302F432D522DC701B60178
:1018E0000E94B5AE181624F0C12ED02EE32CF22C97
:1018F000CDA2DEA2EFA2F8A619A50AA53BA42CA4AE
:1019000020E030E0A901C501B4010E94B5AE750127
:10191000640187FF04C0F7FAF094F7F8F094212FE0
:10192000302F432D522DC701B6010E94B5AE1816B7
:1019300024F0C12ED02EE32CF22CC9A6DAA6EBA6F9
:10194000FCA620E030E040E85FE369AD7AAD8BAD06
:101950009CAD0E94D9AB69AF7AAF8BAF9CAFC75239
:10196000DF4FC880D980EA80FB80C95DD0409501F7
:101970008401B301A201CE0183589F4F0E9418A297
:10198000CF51DF4FA881B981C15ED040AA0FBB1FE4
:10199000CF51DF4FE881F981C15ED040AE0FBF1F4C
:1019A000CA5FDE4F28813981C650D140A20FB31FD4
:1019B000A65BB34FFE01E358FF4F8CE001900D9200
:1019C0008A95E1F70E9440ABCB52DF4F3881C55D6D
:1019D000D040CB50DF4F4881C55FD040340FCB5251
:1019E000DF4F3883C55DD040312C5CCDC151DF4F16
:1019F000A881B981CF5ED040119779F0C752DF4FEF
:101A0000288139814A815B81C95DD040CA01B90111
:101A10000E949EAF882309F4A4C480E00E94554B25
:101A2000882381F0832D0E94691A20E030E040EC89
:101A30005FE7C752DF4F288339834A835B83C95DE1
:101A4000D04071C4C752DF4F288139814A815B8100
:101A5000C95DD040CA01B9010E949EAF811163C423
:101A6000CE0101960E94FBA78DA59EA5AFA5B8A9A2
:101A7000C352DF4F88839983AA83BB83CD5DD04057
:101A800029A93AA94BA95CA9CF51DF4F28833983F3
:101A90004A835B83C15ED0408DA99EA9AFA9B8AD32
:101AA000CB51DF4F88839983AA83BB83C55ED04027
:101AB00020E030E040E85EE3C850DF4F6881798184
:101AC0008A819B81C85FD0400E94F0AEC151DF4F38
:101AD000688379838A839B83CF5ED040C351DF4F75
:101AE000A881B981CD5ED040AB2B09F480C142E61C
:101AF0005CE066E57CE0CE0183589F4F0E94EAA23D
:101B000046E55CE06AE47CE0CE0187579F4F0E9487
:101B1000EAA2AE0143585F4FBE0167577F4FCE0127
:101B20008B569F4F0E9432A2CB56DF4F4880598080
:101B30006A807B80C559D040C756DF4F8880998026
:101B4000AA80BB80C959D040C356DF4F2881398154
:101B50004A815B81CD59D040CB52DF4F28833983F6
:101B60004A835B83C55DD04020916E0C30916F0C31
:101B70004091700C5091710CC301B2010E94F0AE03
:101B80006B017C012091720C3091730C4091740CAC
:101B90005091750CC501B4010E94F0AE9B01AC01DF
:101BA000C701B6010E94D9AB6B017C012091760C74
:101BB0003091770C4091780C5091790CCB52DF4FDB
:101BC000688179818A819B81C55DD0400E94F0AE99
:101BD0009B01AC01C701B6010E94D9AB6B017C012E
:101BE00080914A0C90914B0CA0914C0CB0914D0CF3
:101BF000BC01CD019058A30192010E94F0AEC751E3
:101C0000DF4F688379838A839B83C95ED0402091AC
